:020000040000FA
:040000006FD00400B9
:101000006F00907E00000000000000009020002093
:10101000AA220020A9BDF9F56C23002000000000E1
:10102000000000006C230020902000200000000041
:101030000000000090200020000000009020002010
:101040000000000090200020902000209020002030
:101050009020002090200020582F00209424002071
:101060000000000090200020902000201E2400207E
:1010700090200020D22300209020002090200020EB
:101080009020002090200020902000209020002020
:101090009020002001A04111B7170040985F3AC688
:1010A000945F3247E39CE6FE3245410182800111A4
:1010B00013078008F337078093F787083EC20100C3
:1010C0000100B7170040930570052380B70413068D
:1010D00080FA2380C7040100010083C6B70493F699
:1010E000F60DA385D704238007049246F3A6068055
:1010F0000100010093760502D5CEF336078093F602
:10110000860836C4010001002380B7042380C70489
:1011100001000100B70614007D89558D88C70100C4
:1011200001000100010023800704A246F3A6068007
:101130000100010073370780137787083AC6010062
:1011400001002380B7042380C704010001000100CF
:1011500001003727004093061005A303D7802380A2
:101160000704B247F3A70780010001009307800836
:10117000F3B7078093F787083ECE01000100B71749
:101180000040130770052380E704130780FA2380CB
:10119000E7040100010003C7B70413670708A3852C
:1011A000E70423800704F247F3A70780010001004A
:1011B0000561828093760504BDC6F336078093F6F9
:1011C000860836C8010001002380B7042380C704C5
:1011D00001000100B7061400938606047D89558D31
:1011E00088C7010001000100010023800704C246F6
:1011F000F3A6068001000100733707801377870884
:101200003ACA010001002380B7042380C70401000B
:1012100001003727004093062005A303D7802380D1
:101220000704D24781B773370780137787083ACC12
:10123000010001002380B7042380C70401000100DE
:1012400098471367070C98C723800704E24719BF24
:101250000111814601468145114506CE97000000E7
:10126000E780605893078008F3B7078093F78708F3
:101270003EC601000100B717004013077005238028
:10128000E704130780FA2380E7040100010003C785
:101290006704136717002383E70423800704B2471A
:1012A000F3A7078001000100F2400561828041112F
:1012B000814601468145114597000000E780A05214
:1012C00013078008F337078093F787083EC40100AF
:1012D0000100B7170040130670052380C70493066A
:1012E00080FA2380D70401000100FD552396B70240
:1012F00023800704A245F3A5058001000100733790
:101300000780137787083AC6010001002380C704CD
:101310002380D7040100010003C767041367170087
:101320002383E70423800704B247F3A70780010063
:10133000010001A0BD473305F50201007D1575FDD3
:101340008280411122C426C206C6AA8401446317C2
:101350009400B24022449244410182800504130566
:10136000803E420497000000E78000FD4180C5B741
:101370009305000273A04580824573901534924016
:101380002242B2424243D2436244F2440255925551
:101390002256B2564257D2576258F25806499649D9
:1013A000264AB64A464BD64B664CF64C065D965DD1
:1013B000265EB65E465FD65F09617300203041113C
:1013C000B7170040985F3AC6945F3247E39CE6FE49
:1013D000324541018280B71700401307000323887C
:1013E000E702854717170000232EF74673002030C9
:1013F000411122C42D6426C24AC006C637190040D6
:101400001304A4AAB704002023208900977000E0E9
:10141000E78020AA9C408297977000E0E78060A94F
:10142000E5B737370040834747009146BD8B639E41
:10143000D702B73600401306F00F973500009385AA
:10144000651E9737000083D7E72D03C7A6001377E3
:10145000F70F1DE3B7E70400BC4F09468945171590
:1014600000000345A5F7829731A099466394D70001
:10147000834757007300203003C786001377F70FA8
:10148000E365F6FC13851700AE9717380000231BA1
:10149000A8282380E70075B7B787004003C7670017
:1014A000098B6309071003C77700930600031377BE
:1014B0000703630DD708173800000348F87717367D
:1014C0000000130666740547B30606012380E60094
:1014D00083C577001737000013070775429793F508
:1014E000F50F2300B70003C58700973500009385EB
:1014F000A572C2951375F50F2380A5000347070059
:1015000089451377F703630CB70C63E7E50A6306B5
:10151000071A8545630CB7129737000083C7D77148
:101520003307F600034707001377F70F19CB85073A
:1015300093F7F70F3D476363F71A17370000A30DC2
:10154000F76EB787004009472383E700B78700405D
:1015500083C77700E207E18763DE0704973700005F
:1015600083C7976D173700001307076A3E978546B4
:101570002300D700173700001307076B3E97930629
:1015800000032300D700173700001307E7683E97D2
:10159000A14685072300D70093F7F70F3D47636403
:1015A000F71417370000A309F768B7870040094709
:1015B0002383E70073002030930610026300D70EE8
:1015C000930620026305D70693060002E316D7F4BC
:1015D00003C727021377C70F13672700D5A803C7D0
:1015E00067001377070465CB03C7A702173800000D
:1015F00013080843173500001305453A1347070839
:101600002385E70203C7A7021377370F1367870005
:101610002385E702814713070004B305F5008C41D9
:10162000B306F80091078CC2E399E7FEF5B503C74E
:10163000A702134707042385E70203C7A70213770E
:10164000C70F136727002385E702F9B503C76700B3
:101650001377070449C303C767021738000013084C
:10166000E82F1735000013052527134707082383A4
:10167000E70203C767021377370F136787002383D7
:10168000E702814713070004B305F5008C41B30658
:10169000F80091078CC2E399E7FEBDBD03C767025E
:1016A000134707042383E70203C767021377C70FB3
:1016B000136727002383E70285B503C76700137705
:1016C000070411CB03C727021377370F136787006F
:1016D0002381E70291B5238006003DBD97370000C6
:1016E000A38C0754B9BD97370000A387075475BD75
:1016F0002303048015472303E48001002302A48010
:10170000828083076480E3CE07FE23030480828007
:1017100083076480E3CE07FE03454480828083070D
:101720006480E3CE07FE2302A4808280411126C498
:101730004AC24EC006C61377F50BAD47AA892E895B
:101740009544630CF700194597000000E78080FA84
:1017500097000000E78020FB8D444E859700000035
:10176000E78040F9FD59FD1463983401B240A2446A
:101770001249824941018280135509011375F50F01
:1017800097000000E780E0F92209F1BF011126CCA3
:1017900006CEB704080097000000E780C0F61545A4
:1017A00097000000E78000F597000000E78080F6D2
:1017B00097000000E78000F62AC697000000E78047
:1017C00080F432459377150089EB13651500137586
:1017D000F50FF240E24405618280FD14E9F0014515
:1017E000CDBF397126DC4ADA4ED852D656D45AD2F9
:1017F0005ED006DE62CE66CCB7E700E07D5783AAF6
:10180000070022C603AA470023A0E71823A2E7186F
:10181000B7170040130770052380E704130780FA09
:101820002380E70483C74704930B75FFB684E20760
:1018300093FBFB0F8546AA892E8B32893724004003
:10184000E187015763FA76016308D50089461307DB
:1018500000026313D5000157D98F93F7F70FB71C18
:1018600000402382FC0411472303E4801305F00F9A
:1018700097000000E78000E8094C97000000E7802F
:1018800080E863657C15B7050700DA9537870700A0
:10189000795563FEE504B3879500636AF704370B57
:1018A0000800A94733EB65016395F90881E8814495
:1018B00097000000E78020E5268515A8DA85094510
:1018C00097000000E780C0E605090345F9FFFD1415
:1018D000050B97000000E780C0E481C49377FB0FFD
:1018E000E5F797000000E780A0EA69F17D55B7179A
:1018F0000040130770052380E704130780FA238054
:10190000E70403C74704418B2382E704F250B7E79B
:1019100000E023A0571123A24711E2543244525948
:10192000C259325AA25A125B825B724CE24C21615C
:101930008280A547639BF90685691309F00FB306FA
:101940009900B3742B01B6941349F9FFB37499004D
:10195000856B33796901416B9387F9FFB3F72701F1
:1019600099E363FC340193D94900C147E3E637FFAB
:101970003DBF0569C1697D19D9B71305800D63881D
:101980006901130500026384790113051008CA85F3
:1019900097000000E780C0D997000000E78040DF93
:1019A00031D54E99B38434416DBFDA852D4597000A
:1019B0000000E780E0D7CA94E30B99EE0509970091
:1019C0000000E78020D5A30FA9FEFDB79387F9FF9C
:1019D00093F7F70F636DFC0C83C71C0413073008E3
:1019E0006315F706370708006361EB06B3079B0032
:1019F000B706100063FBD704334BEB0089476399AC
:101A0000F9068980D549E38404EADA850945970017
:101A10000000E780E0D111090327C9FF9147232087
:101A2000E48003076480E34E07FE23033481FD173F
:101A3000EDFBFD14110B81C49377FB0FE9FF9700B9
:101A40000000E780E0D461F155B5B717004003C747
:101A50005704B70708001377070219E3B787070091
:101A60007955E376FBE833079B00E3F9E7F841B5E6
:101A70008547E380F9F0DA852D4597000000E7807F
:101A800020CB9389F4FFE38404E297000000E78011
:101A900060C893F7390091EB83260480032709007F
:101AA00093074900E396E6E03E89CE84D9BFB54767
:101AB0006399F9001305900B97000000E78080C33D
:101AC000FDB3B1471305B00AE388F9FE9947639760
:101AD000F904B7050800B365BB002D459700000069
:101AE000E78000C581448D4BA14997000000E78045
:101AF00060C263967401832704802320F900850463
:101B0000E39534FF8327048013172B0163550700E7
:101B10002312F90069BB2322F90051BB9D47639F43
:101B2000F90281451305B00497000000E78040C02A
:101B3000BD442320090023220900FD59970000001D
:101B4000E78040BD93F77400CA9703C70700FD14F0
:101B5000398D2380A700E39334FF91BBA14763979E
:101B6000F90697000000E780A0C28144630D0B00D6
:101B70008D479304C0036308FB00930400056304CE
:101B80008B01930440041375C507E30295D21945F0
:101B900097000000E78000B697000000E780A0B63D
:101BA000054597000000E780E0B426859700000017
:101BB000E78020B7094597000000E78080B69700CE
:101BC0000000E780E0BCE31405CE0DB39147639FAE
:101BD000F9001305600697000000E780A0B19700A8
:101BE0000000E78040B213059009F9B5E38109CC04
:101BF000F1547DB9BD660147173600001306063063
:101C0000938606A685458347060093F7F70F91C391
:101C100082800507E3F9E6FE973700002380B72EA0
:101C2000DDB77D166206618693178601E18763D46E
:101C3000070001458280931726003307F500AE9711
:101C400018439C4363E7E7007D16E37FF7FC7D556F
:101C5000828005458280FD15E205E18513978501A7
:101C6000618793F7F50F63480700FD15139725006B
:101C70002A97584365D713851700620561858280CE
:101C80003308B5021C4283A80600B335B502C297DB
:101C900033B50701AE98469585486367B5006394F0
:101CA000A50063E3070181480C43C6950CC388C2B5
:101CB0001CC2828081471397870161876343B70005
:101CC0008280139727002A97232007008507E5B70E
:101CD0008147014793968701E18663C5B6001335B6
:101CE0001700828093962700AA9694428507558F05
:101CF000D5B793D755408A07AA979C430545331516
:101D0000B5007D8D828017F3FFDFE702833D2A84D3
:101D100097000000E78060F405C5931725003E9406
:101D20000327C4FF814711EB7D1516053E9542053B
:101D3000418517F3FFDF6700033D05838507E5B79E
:101D40000145C5BF81471397870161876343C7007A
:101D5000828013972700B386E50094422A9785076F
:101D600014C3D5B77D1662066186014793178601B5
:101D7000E18763D50700133517008280931726008B
:101D8000B306F500AE9794429C437D16B58F5D8FE8
:101D9000F1BF8A05AA9501476363B500828083A6D7
:101DA000C5FFF11593D71600D98F9CC11397F60183
:101DB000E5B72A830148014701456343D700828084
:101DC000B387050183A80700B30706019C43C697A4
:101DD000AA976384F80033B517010507B308030118
:101DE000620723A0F80061871108C1BF2A83014759
:101DF0008147014563C3D70082803388E50083288B
:101E00000800330EE600032E0E003388A840330886
:101E1000C8416384080133B508018507B308E300AE
:101E2000E20723A00801E1871107E9B717F3FFDFF5
:101E3000E702232B0111B286B2842E86AA850A8579
:101E400097000000E780C0FA2A84A6850A859700DB
:101E50000000E78020E833348000060413351500C5
:101E6000018D056117F3FFDF6700E32917F3FFDF3B
:101E7000E702A3244111AA89AE8A328BB68402C23A
:101E800002C402C60144131C8401135C8C416349E3
:101E90009C02939B1400FD1B0549138CF4FFF15C1D
:101EA00033048901620461846340740792478E049D
:101EB000CE9423AEF4FE410117F3FFDF67006323E6
:101EC00013192400B30B2B01014A93172A00D6974C
:101ED00083A50B0088437800340050009700000071
:101EE000E78040DA050A93178A01E187F11BE35E78
:101EF000FCFC92474E9905042320F900A2473EC2FC
:101F0000B24702C63EC441B7131A8901135A8A4127
:101F1000131D240093178A01E18763CF970092472E
:101F20000A044E941CC0A24705091379F90F3EC25A
:101F3000B24702C63EC4ADB7B3079A0313152A00D1
:101F400056950841780034005000050AEA97DA9760
:101F50008C4397000000E780E0D26DBF197106C284
:101F600012C416C61AC81ECA22CC26CE2AD02ED219
:101F700032D436D63AD83EDA42DC46DECAC0CEC2C9
:101F8000D2C4D6C6DAC8DECAE2CCE6CEEAD0EED2F9
:101F9000F2D4F6D6FAD8FEDA971500009385058CB0
:101FA0008841E700050092402242B2424243D243B8
:101FB0006244F244025592552256B2564257D257C5
:101FC0006258F25806499649264AB64A464BD64BBD
:101FD000664CF64C065D965D265EB65E465FD65F45
:101FE0000961730020300000972100209381810156
:101FF000175100201301018117F5FFFF1305C500DC
:102000009705002093850500171600201306C6FDCE
:1020100063FAC5008322050023A055001105910530
:10202000E3EAC5FE17050200130545749715002065
:102030009385C5FB171600201306C66563FAC50015
:102040008322050023A0550011059105E3EAC5FE92
:102050001715002013050564974500209385053664
:102060006377B500232005001105E36DB5FEFD4241
:10207000739002BC8D4273904280B722000093821D
:10208000828873900230970200209382A2F793E235
:1020900032007390523097520000938222B57390B1
:1020A00012346FB0F47573002030397101436EC67D
:1020B00019A0397141536AC866CA62CC5ECE19A0B4
:1020C000397101535AD056D252D44ED64AD826DA54
:1020D00022DC06DE33016140828241114AC026C201
:1020E00022C406C68282B24D4101024D924C224C5E
:1020F000B24B4101024B924A224AB2494101024984
:1021000092442244B240410182803D432A87637356
:10211000C3029377F700BDEFADE5937606FF3D8AE6
:10212000BA960CC34CC30CC74CC74107E36BD7FE30
:1021300011E28280B306C3408A0697020000969699
:102140006780A6002307B700A306B7002306B700E1
:10215000A305B7002305B700A304B7002304B70005
:10216000A303B7002303B700A302B7002302B700FD
:10217000A301B7002301B700A300B7002300B700F5
:10218000828093F5F50F93968500D58D9396050182
:10219000D58D61B7939627009702000096968682A8
:1021A000E78086FA9680C1171D8F3E96E374C3F8C8
:1021B000A5B73367B500FD530D8B79E7B7877F7FF0
:1021C0009387F7F710419441B372F6003363F6003A
:1021D000BE92B3E262006397720C6318D606504158
:1021E000D441B372F6003363F600BE92B3E26200EC
:1021F0006398720A631BD60410459445B372F600C7
:102200003363F600BE92B3E262006391720A631E0A
:10221000D6025045D445B372F6003363F600BE9241
:10222000B3E26200639A72086311D60210499449BE
:10223000B372F6003363F600BE92B3E262006393BA
:1022400072085105D105E30FD6F6131706019397CF
:102250000601631CF7001357060193D706013305E7
:10226000F7409375F50F91E982804183C18333056F
:10227000F7409375F50F91E182801377F70F93F78D
:10228000F70F3305F74082800346050083C605003B
:10229000050585056313D60065FA3305D6408280AF
:1022A00011059105E312D6FE014582802105A105A5
:1022B000E31CD6FC014582803105B105E316D6FC4E
:1022C000014582804105C105E310D6FC01458280AD
:1022D000B717004003C777051377E70FA38BE70411
:1022E000130700F8A38DE7043D47238CE704130789
:1022F0005003A38CE70403C7A7051377D70F238DDB
:10230000E7048280B717004003C7E7020D89411137
:102310001377C70F498F93068008F3B6068093F6AC
:10232000860836C601000100930670052380D70495
:10233000930680FA2380D704010001002387E70277
:1023400023800704B247F3A7078001000100410181
:10235000828041112A83014E930E407E130F001993
:10236000930F400663E56E129308001913034006AD
:10237000B3781503854E0D4FA14F337365020D8958
:102380001335150063EFBE121308F6FF79467298F5
:102390004208135808013307C70213D61700BE07B7
:1023A00032976146B3F6C60213068070B386C60242
:1023B0003697A166F58F42075D8FB716004083C739
:1023C000F60293F70708A303F1000346710083C7E1
:1023D000F60293F70708E394C7FE83477100B71628
:1023E000004093F7F70F6388071293078008F3B74D
:1023F000078093F787083EC401000100B71700402B
:10240000930670052380D704930680FA2380D704AF
:102410000100010023AA070383C6170393E60608F9
:10242000A388D70223800704A247F3A707800100EF
:1024300001001166B71700407D16D45BC85F938515
:102440004703A98EF18EF5FA93068008F3B606804D
:1024500093F6860836C601000100930670052380B6
:10246000D704930680FA2380D7040100010098C1A5
:1024700003C7170313670704A388E7022380070431
:10248000B247F3A7078001000100410182807D135C
:102490003368E3039308E016630E08003368F30320
:1024A0009308D016630808009378330093B8180097
:1024B0009388D81633081E01131E0801135E0E01FF
:1024C00055B56393E5030548638608000148630337
:1024D00003002A8871087298FD15131E0801C205B1
:1024E000135E0E01C18179BD13F8150063F4BF00BE
:1024F0007908D5B713381800E5BF83C7F60293F7FC
:102500000708A303F1000346710083C7F60293F79F
:102510000708E394C7FE8347710093F7F70FF1DFD5
:10252000E9B531714AD966CB06DF22DD26DB4ED70D
:1025300052D556D35AD15ECF62CD6AC96EC7AA8C26
:1025400002D897100000E78020B12A8993078008FD
:10255000F3B7078093F787083EDA01000100B71749
:102560000040130770052380E704130780FA2380D7
:10257000E7040100010003C7F7021377770FA38771
:10258000E70203C7F70213678700A387E7022380E8
:102590000704D257F3A70780010001000545970003
:1025A0000000E78060D6130780C13347E902116A53
:1025B00093070AE893065002BD69930BA004814A71
:1025C000014B13048008930470057D1AB347F90288
:1025D0003307D7023EC0FD873ECC938709A69309F7
:1025E000803E3347F7023AC27D873AC43347390306
:1025F0008549B399990193D93940B306D702B30BF2
:102600007703B3C6F602B3CBFB0236C6FD8636C8E7
:1026100093D6FB4136CEB7460F0093860624334946
:10262000D9028566938606FAB3969601B389E902C4
:10263000130760553309D90293060010B389E902E4
:102640003349D902B3C9F9029316390036CA37198A
:102650000040FD8636D0930D090493D7F9413ED250
:10266000F336048093F6860836DC010001009307F8
:1026700070052380FD00930680FA2380DD000100B1
:1026800001008346390593F6860FA309D9048346D2
:10269000390593E61600A309D90423800D00E256FC
:1026A000F3A6068001000100130C80FA116DF336C9
:1026B000048093F6860836DE01000100930770055A
:1026C0002380FD0023808D01010001008346390530
:1026D000216693E60602A309D90483560905B3E6E9
:1026E000A6012318D90483560905D18E2318D904CD
:1026F00023800D00F256F3A60680010001008346F8
:10270000390593F606026381061A03463905218AC4
:102710006DDE081897100000E7800098733604807B
:1027200013768608B2C20100010023809D00238039
:102730008D0101000100B717004003C6370513766D
:10274000F60DA389C70403C6370513660602A389DD
:10275000C704835609052166B3E6A6012318D904E8
:1027600083560905D18E2318D90423800D0096467F
:10277000F3A60680010001008346390593F60602A0
:10278000638B061483463905A18AEDFE970000206D
:10279000E7806090AA8636D497000020E780A08F5B
:1027A000A256E30AD5FE835609054255B3E6A601B3
:1027B0002318D90497100000E780C08F834639059D
:1027C000A18AEDDE03560905834629058247337643
:1027D000CA00B306DA0293D5F641B296B388F64042
:1027E000E24733B8C6002E983308F840A247B3B684
:1027F00016013308D84063C70701631DF8009247EC
:1028000063FA1701C247634FF80E63950701B24799
:1028100063EAF80E894663E9660FF24693151800DD
:1028200013D3F8015E8613951800B365B30042D642
:1028300046D497C00100E78040513258050B137B06
:10284000FB0F63470001631A0838A25863870838F2
:1028500013081500B336A800B69513D6F5013298C3
:10286000B336C800AE9613581800FE06B3E606014C
:102870007336048013768608B2C6010001002380F7
:102880009D0023808D01010001000356C902B2960C
:10289000C206C1822316D90223800D00B646F3A6D4
:1028A00006800100010021B5F336048093F6860806
:1028B000B6C00100010023809D0023808D0101002E
:1028C00001008346390593E60602A309D904238053
:1028D0000D0086460DB5F336048093F68608B6C41F
:1028E0000100010023809D0023808D010100010073
:1028F0008346390593E60602A309D90423800D0017
:10290000A646BDB5E30B0BF0F336048093F68608BC
:10291000B6C801000100930680FA23809D00238041
:10292000DD00010001008346390593F5FC0F93F6A5
:10293000860FA309D90483463905CD8EA309D9048E
:1029400023800D00C646F3A6068001000100130592
:1029500080FA03463905930639051D8A631C9629BA
:102960007336048013768608B2CC0100010013068A
:1029700080FA23809D002380CD000100010003C662
:1029800006001376F60D2380C60003C60600136604
:1029900006022380C600835609051166D18E2318CE
:1029A000D904835609052166D18E2318D9042380C2
:1029B0000D00E646F3A6068001000100130680FA2A
:1029C0008346390593F60602638006268346390559
:1029D000130C3905A18AFDDA081897000000E7807A
:1029E000A06BF336048093F68608B6D00100010090
:1029F000930680FA23809D002380DD000100010002
:102A000083460C00116693F6F60D2300DC00834626
:102A10000C0093E606022300DC0083560905D18EE4
:102A20002318D904835609052166D18E2318D904A9
:102A300023800D008656F3A60680010001001306D0
:102A400080FA8346390593F60602638A0620834698
:102A50003905A18AEDFE97F0FF1FE780C0632A8C3D
:102A600097F0FF1FE7802063E30C85FF835609057D
:102A700011664255D18E2318D90497000000E780D3
:102A800060638346390513063905A18AFDDAF336FA
:102A9000048093F68608B6D401000100930680FAFC
:102AA00023809D002380DD00010001008346060095
:102AB00093F6F60D2300D60023800D00A656F3A64C
:102AC0000680010001008356090503462905D24707
:102AD000B376DA003306CA021305800C9355F6412B
:102AE0003696330DF6408257333CD6002E9C333653
:102AF000A601330CFC40330CCC40330885039256BE
:102B00004E86B335A5033305A503C29597C00100D2
:102B1000E780A02363468001631E0C16630C0D162C
:102B2000130615003335A6002E959356F5013696FB
:102B3000B335D600AA959396F50105828585D18E89
:102B40006346B000639D051A638B061A0356C902DB
:102B500015823305D6003336C500B2956348B00000
:102B6000639105241306F00F637DA622894663F363
:102B7000561593078008F3B7078093F78708BED6EA
:102B80000100010037170040930770052300F70488
:102B9000930780FA2300F704010001008356C7025F
:102BA00089678117D58FC207C1832316F7022300D7
:102BB0000704B657F3A7078001000100FA506A54D2
:102BC000DA544A59BA592A5A9A5A0A5BFA4B6A4C49
:102BD000DA4C4A4DBA4D296182801308F5FF33352E
:102BE000A800FD152E951356F5013298B336C8008E
:102BF000AA9695B9F336048093F68608B6CA010002
:102C0000010023809D002380AD0001000100834668
:102C10003905CD8EA309D90423800D00D646F3A62D
:102C200006800100010035B3F336048093F6860870
:102C3000B6CE0100010023809D002380CD0001005D
:102C400001008346390593E60602A309D9042380CF
:102C50000D00F646F3A606800100010095B3F33699
:102C6000048093F68608B6D20100010023809D00FF
:102C70002380CD00010001008346390593E606025A
:102C8000A309D90423800D009656F3A606800100FF
:102C9000010045BB9306F5FF33B5A600FD152E9543
:102CA0009355F501AE96B3B5B600AA951396F50106
:102CB000858269B5F336048093F68608B6D801009C
:102CC0000100930680FA23809D002380DD0001002F
:102CD00001008356C9020566011693F6F60FD18EE0
:102CE000C206C1822316D90223800D00C656F3A660
:102CF000068001000100850A93FAFA0F95B233E6C7
:102D0000B60045C20356C9023305D0403338A0008F
:102D1000B305B040B385054115826345B000D1E1EC
:102D20006371A608894663F0560593078008F3B7D8
:102D3000078093F78708BEDA01000100B71700404B
:102D4000130770052380E704130780FA2380E70444
:102D50000100010003D7C7027D8B2396E702238081
:102D60000704D65781BDF336048093F68608B6DC97
:102D700001000100930680FA23809D002380DD007E
:102D8000010001008356C9020566011693F6F60F8D
:102D9000D18EC206C1822316D90223800D00E656C9
:102DA000B9B793078008F3B7078093F78708BEDEAB
:102DB0000100010037170040930770052300F70456
:102DC000930780FA2300F704010001000356C702AD
:102DD00093975600B297C207C1832316F7022300C8
:102DE0000704F657C1BB914763EEB70217E701002E
:102DF000130707948A05BA959C41BA978287B7173B
:102E0000004003A7470B1345F5FF698F23AAE70A84
:102E100003A7070B698F23A8E70A03A7070A798D81
:102E200023A0A70A8280B717004083A6470B134749
:102E3000F5FFF98E23AAD70A83A6070B558D23A881
:102E4000A70A83A6070A758F23A0E70A8280B7170F
:102E5000004003A7470B498F23AAE70A03A7070BE4
:102E60001345F5FF45BFB717004083A6470B13472F
:102E7000F5FF758F23AAE70A03A7070A598D4DB7F7
:102E8000B717004003A7470B498FEDB7914763EE93
:102E9000B70217E701001307E78A8A05BA959C4134
:102EA000BA978287B717004003A7470D1345F5FF70
:102EB000698F23AAE70C03A7070D698F23A8E70CE6
:102EC00003A7070C798D23A0A70C8280B7170040B9
:102ED00083A6470D1347F5FFF98E23AAD70C83A6C7
:102EE000070D558D23A8A70C83A6070C758F23A06B
:102EF000E70C8280B717004003A7470D498F23AA2C
:102F0000E70C03A7070D1345F5FF45BFB7170040B2
:102F100083A6470D1347F5FF758F23AAE70C03A778
:102F2000070C598D4DB7B717004003A7470D498FC0
:102F3000EDB7797122D43714004026D24AD0035914
:102F400024028354040206D64209C2044ECE52CC57
:102F500056CA13590901C1802DE11379F9F793F489
:102F6000F49F4209C20413590901C18093078008E4
:102F7000F3B7078093F787083EC401000100930769
:102F800070052300F404930780FA2300F404010081
:102F90000100231124032310940223000404A247F8
:102FA000F3A7078001000100B25022549254025945
:102FB000F249624AD24A45618280B7F507008146EC
:102FC0003000B105194597000020E7808081A247B5
:102FD00013972701E34A07FC1369090893E40440A7
:102FE00093098008F3B7098093F787083EC0010072
:102FF0000100930A700523005405130A80FA230088
:10300000440501000100231124032310940223002E
:1030100004048247F3A7078001000100294597F0C7
:10302000FF1FE7802031F3B9098093F989084EC268
:1030300001000100230054052300440501000100A4
:103040008357040293E707202310F40223000404AB
:103050009247B9B7B7170040884742054181937737
:10306000050491EB9377F5013755E80113050580C9
:103070003345F50282809377050C130700046397AC
:10308000E7009377F50137459C1CCDB72165130503
:1030900005D0828037E700E01C435443A183E20659
:1030A000D58F1CC1FD572320F7182322F7188280E3
:1030B00013178500B7E700E023A0E710618123A282
:1030C000A7108280B7F700E08847CC47828081470D
:1030D00037370040A14663C4C7003285828003456C
:1030E000B740E38EA6FE3385F5000345050085074E
:1030F0002304A740CDB797070020938727EF9C4371
:10310000173700201307872B3E95636EE5001737AE
:1031100000201307273F6368A70017070020232715
:10312000A7EC3E858280FD57EDBF8280411122C40D
:1031300006C62A8497000000E78000F22947B307FB
:10314000E502B2408D83B3D7870222449507B3D7F7
:10315000E70237370040C207C1832316F700410159
:103160008280411137150E0006C697000000E780E7
:1031700020FCB7370040130770F82381E7000D47A4
:10318000A381E70013070004A380E7000547238716
:10319000E700B24041018280373700408347270073
:1031A0001A0593F7F703C98F93F7F70F2301F70079
:1031B0008280B737004003C7170019C9D98DA38093
:1031C000B70003C70700136787002380E7008280EA
:1031D00093C5F5FFF98DA380B7008280AE872A875B
:1031E000B736004021463738004089E71703000012
:1031F0006700E3F383C8B600E30916FF05078348B9
:10320000F7FFFD17C20723041801C183F9BF41115D
:1032100022C406C62A8497000000E780E0E329471D
:10322000B307E502B2408D83B3D7870222449507E6
:10323000B3D7E70237370040C207C1832316F740F0
:1032400041018280716541111305052006C6970072
:103250000000E78000FCB7370040130770F82381B7
:10326000E7400D47A381E74013070004A380E74030
:1032700005472387E740B24041018280CC4141119C
:1032800006C6328503C6150083C5050022064D8E8D
:1032900042068D654186138875A2630C0611634B47
:1032A000C804138845A26300060D634AC8009385CD
:1032B00035A26301B6082390060029464DA0138865
:1032C00055A26305060D938565A2E316B6FE8D45EE
:1032D0001D4663E6E5081146198E63F3C7003E8676
:1032E000B7E704002390C600FC4797D501009385FB
:1032F000A5479DA0138895A263030611634E060D92
:103300001388A5A263000613938505A5E315B6FAF5
:1033100099451D4663E5E504198E63F3C7003E86B3
:10332000B7E704002390C600FC479705002093856B
:1033300025D61DA09D451D4663E3E5022146198E55
:1033400063F3C7003E86B7E70400FC472390C6003E
:103350009705002093858534BA9582970146B2403F
:10336000328541018280AD451D46E3EAE5FE3146E6
:10337000198E63F3C7003E86B7E704002390C600AA
:10338000FC4797D501009385A540F9B7B1451D4687
:10339000E3E7E5FC3546198E63F3C7003E86B7E7E1
:1033A00004002390C600FC4797D501009385453F54
:1033B00065B78D451D46E3E4E5FA1146198E63F3C2
:1033C000C7003E86B7E704002390C600FC4797D5A8
:1033D00001009385253A49B78D451D46E3E1E5F89F
:1033E0001146198E63F3C7003E86B7E704002390A9
:1033F000C600FC4797D501009385453CB1BFA54564
:103400001D46E3EEE5F42946198E63F3C7003E86B8
:10341000B7E704002390C600FC4797D501009385C9
:1034200025361DBFB5451D46E3EBE5F23946198E3D
:1034300063F3C7003E86B7E704002390C600FC474D
:1034400097D501009385453101BFB7E7040003A379
:103450000713970600209386A6C24146A545170587
:1034600000201305E5B802832D455DE703C505007F
:103470000947631FE50803A84500411106C6034735
:10348000180032850346080022074168518F9308CF
:1034900028FE6307170563E9E800051863030703BF
:1034A00023900600294591A8130648FE630AC70425
:1034B0001518E31707FF15463E87637BF60015478F
:1034C00001A8130600023E876374F600130700028A
:1034D000B7E704002390E600FC471316070111A884
:1034E0003E8691C30546B7E70400FC472390C6001B
:1034F0004206CC45418282970145B240410182801B
:10350000130600083E87E375F6FC13070008C9B7E9
:103510002390060005458280828041677917630405
:10352000E504411122C406C685472A84639FF5003D
:10353000B7E7040022852244B24003A3871397050E
:1035400000209385E52F4101028389476399F500A7
:10355000B7E7040083A7070B8545829771D9B2406E
:103560002244410182808280797126D252CCAE847D
:103570002A8A97D501009385652617D50100130582
:10358000652806D63AC622D44AD0368432894ECE31
:1035900097C00100E780A0C6A28517D501001305DA
:1035A000652797C00100E78080C5294597C00100C5
:1035B000E780C0C983C7840093F70702F9E383C992
:1035C00004008947054532476396F908D44083C70C
:1035D000160083C60600A207D58FC166138616FEA5
:1035E000638CC7028D16638FD7068D6693862690EF
:1035F00029456391D706B7E70400A286225403A3A6
:103600004714B250F2494A86A6850259925452850F
:10361000624A8547456102832D450DEF93070002FD
:10362000354563E98702B7E70400FC47C844130641
:103630000002CA8582978149970700209387072156
:103640009C43014581CB9C4391C74E852286CA8508
:1036500082970145B250225492540259F249624A6B
:10366000456182802D457DF79307700F3545E3E373
:1036700087FEB7E70400FC47C8442286CA858297C4
:1036800065BF2145C1BF411122C437E4040083272F
:10369000841326C2AA84416506C697050020938537
:1036A000251A7D1582978327C40A17050000130584
:1036B00005E78588829795C0032304132244B2400E
:1036C000924497060020938626AE4146C5451705CD
:1036D00000201305659C41010283B24022449244BC
:1036E00001454101828019C59707002023A0A71634
:1036F00001458280454582801147636AA70A97D6B3
:1037000001009386660C0A0536951841411106C6DC
:103710003697AE87B2850287130700026145639D25
:10372000E700B7E70400FC47130600021705002076
:10373000130545F782970145B24041018280054754
:103740006145E39BE7FEB7E70400FC470546170524
:103750000020130525F7F9BF1307700F6145E39D9E
:10376000E7FCB7E70400FC471306700F17050020BD
:10377000130585F5C1B7130700086145E39EE7FA15
:10378000B7E70400FC4713060008170500201305DF
:1037900025034DB715476145E390E7FAB7E7040005
:1037A000FC471546170500201305C50961B70945F3
:1037B0008280411126C2B7E4040083A7C41322C447
:1037C0004AC006C62E8497050020938565072A897E
:1037D0008297058905C5970700209387E78B83D7D4
:1037E000A70BA28503A3440D2310F4002244B2408A
:1037F00092444A850249014641010283B240224473
:103800009244024949454101828097070020238163
:1038100007049707002023AF0702B717004003A74C
:10382000070CB706C0FFFD16758F23A0E70C03A792
:10383000070DB7064000558F23A8E70C03A7070C18
:103840003D9B23A0E70C03A7070D1367070123A8DF
:10385000E70C8280B717004003A5470C83A7470CED
:10386000598113451500C18B058999E3136525001E
:103870009707002083C7C7FD6380A7029707002032
:103880002388A7FC11C9970700209387A7FC03A3EF
:1038900007006303030002838280114517F3FFFFD3
:1038A000670063C8011122CC06CE3714004026CA37
:1038B0004AC84EC652C483447405034AB4058349BA
:1038C00084050349940597F0FFFFE780A0A0834794
:1038D000A40593F4F40F137AFA0F93E71700230D5E
:1038E000F40493F9F90F1379F90FB717004003C7E0
:1038F000A705058B6DFF03D5C705A38D4705238C51
:103900003705A38C2705A38B9704F2406244D24469
:103910004249B249224A05618280411193970501CB
:1039200022C406C626C2C1872E8463DC0700B7E422
:103930000400FC54829719C1BC5482972165218DE3
:1039400015A893F7150013C515008DE793F725000B
:103950009DC797000000E78020F0B7E70400BC4F48
:103960001306000A894517050020034525EF8297B5
:1039700013452400B240224492444101828093972F
:10398000250163D80702B7E4040083A7C41E829709
:1039900097000000E780A0F0BC4C375607001306E4
:1039A0000630896517050020034545EB82970965B8
:1039B00079B7939715010145E3DE07FA17D50100A2
:1039C000130545ED97C00100E780409BB7E7040071
:1039D000BC4F13060064916517050020034505E8F8
:1039E00082971165A9BF1D71A2CC37E404005C5C0D
:1039F000485886CE494697D50100938525E582979C
:103A000011E917D501001305A5E597C00100E7806E
:103A1000E09601A0B7F600E0795798CAFD57DCCAD6
:103A20000567B7E700E023A0E7101306F00290C295
:103A300023A0E718010001003707002018471306EC
:103A4000000481459706002023A8E6E04157A38A99
:103A5000E7403C4408088297970700209387077C3B
:103A60003EC8856713870740938757D1231AE10023
:103A70002312F1021307B00F97F7FFFF9387C76474
:103A80002310E1023ED81547970700009387C7E14E
:103A9000B7F50700A30FE1003EDC054797070000DC
:103AA0009387E7DF81463000E10519452301E102F4
:103AB0003EDE97F0FF1FE780C0D218088147994685
:103AC00030003E960346060085070507A30BC70096
:103AD000E398D7FEC24791C70357410185676373D7
:103AE000F70001A0B7E7040083A7470A08088297F8
:103AF000AA8511C917D501001305C5D797B00100D4
:103B0000E780E06F01A0F6406644256182804111A4
:103B100026C2B7E4040083A7040806C622C417051A
:103B200000001305C5DF829717040020130404D397
:103B30002300A40097000000E780800297000000A7
:103B4000E780E0CC03450400224403A38405B2408F
:103B5000924413060032896541010283797106D6C9
:103B600022D413078008F337078093F787083EC2F3
:103B700001000100B7170040930570052380B704CA
:103B8000130680FA2380C7040100010083C6F702F0
:103B900093F6A60FA387D702238007049246F3A6C5
:103BA00006800100010073370780137787083AC445
:103BB000010001002380B7042380C7040100010035
:103BC00003C7F70213672700A387E70223800704D0
:103BD000A247F3A7078001000100054597E0FFFF1A
:103BE000E780807297000000E78060CB0147814644
:103BF0008147054685451305407E97E0FFFFE78036
:103C0000807537E404003C44680051468145829742
:103C1000B707C0A83EC8B787E803938707D03ECA56
:103C200097E7FF1F9387A7793EC67C586800829765
:103C3000B250225445618280411197D5010093858D
:103C4000652A17D501001305E5BB06C697B001002C
:103C5000E780E05A17D501001305C54197B0010070
:103C6000E780E059B2402945410117B301006700E0
:103C7000E35D411197D501009385052817D5010013
:103C8000130545B806C697B00100E780405717D521
:103C900001001305E53C97B00100E7804056B240B3
:103CA0002945410117B301006700435A411122C45D
:103CB00006C6834705002A849DC797D501009385D2
:103CC000652917D501001305E5B397B00100E7801A
:103CD00000534C4017D501001305054F97B0010064
:103CE000E780E0513DA058410DEF97D50100938545
:103CF000652617D501001305E5B097B00100E780F0
:103D0000005017D501001305A54D97B00100E780BD
:103D1000004F2244B2402945410117B3010067001A
:103D2000E352A1679386D7036313D70297D50100A7
:103D30009385452217D501001305C5AC97B0010046
:103D4000E780E04B17D501001305854A7DBFED07DD
:103D500097D501009385052017D50100130585AA85
:103D6000631BF70097B00100E780604917D5010099
:103D70001305454959BF97B00100E78040484C40C2
:103D800017D501001305054A91BF411197D50100D0
:103D90009385C51717D501001305C5A606C697B0AC
:103DA0000100E780C045B2402945410117B3010039
:103DB0006700C349397122DC26DA4AD82E842A8961
:103DC0008145B2844808714636C606DE97E0FFFF9B
:103DD000E780E03397F7FF1F9387075EDC4783D7C1
:103DE0000700231C2101231BF10097500000E780EE
:103DF0006055B246230DA10091E285469307001954
:103E00003ECE2686FD57A2854808A30DD100230289
:103E1000F10297500000E780C055F2506254D2542E
:103E20004259216182808546170300006700C3F86C
:103E30004111972700202396078E97170020238F84
:103E4000077C06C6170700200347C72D9307F00A13
:103E50006315F7029307F0F889451705002013054D
:103E6000652C17070020230FF72A97070020A38B44
:103E7000072A97600000E780E01597600000E78060
:103E8000A04297600000E780E043814537050400C9
:103E90009707002023AE07269707002023890726CF
:103EA000970700202398071E970700202396071CDA
:103EB00097070020239B072497070020239C0724B3
:103EC00097400000E780E09F014597600000E78091
:103ED000601997D501009385E50517D501001305F5
:103EE0006592970700202393072297B00100E7808F
:103EF000003117D501001305253997B00100E7807F
:103F00000030B2402945410117B301006700033476
:103F10004111814617F6FF1F1306464785451705D1
:103F200000200355251506C697D00000E780E09EC7
:103F300015C997D501009385A50017D50100130574
:103F4000658C97B00100E780802B17D50100130521
:103F5000A52397B00100E780802A294597B001008A
:103F6000E780C02E97D50100938585FD17D5010008
:103F70001305458997B00100E780602817D5010037
:103F80001305C52197B00100E7806027294597B048
:103F90000100E780A02B97F7FF1F9387E741DC47DD
:103FA000054797D501009385A5F92390E70017D51C
:103FB00001001305258597B00100E780402417D53F
:103FC00001001305E51E97B00100E7804023B240D1
:103FD0002945410117B3010067004327411122C45D
:103FE00097D50100938545F82A8417D5010013055C
:103FF000658106C697B00100E78060204C4017D568
:1040000001001305E51597B00100E780401F294521
:1040100097B00100E7808023034704009307F00F67
:10402000631FF70297D50100938505F417C50100BA
:104030001305457D97B00100E780601C4C4017D503
:1040400001001305E51297B00100E780401B2244F0
:10405000B2402945410117B301006700231FB24058
:10406000224441018280411122C426C22A84AE84A6
:1040700017C501001305057997D50100938585EAD9
:1040800006C697B00100E780801717D50100130519
:10409000251E97B00100E7808016294597B00100E2
:1040A000E780C01A97D501009385C5E797070020E0
:1040B000239287FC17C501001305C57405449707B3
:1040C0000020239797FA97070020239487FA9717E1
:1040D00000202398976497B00100E780401297155D
:1040E000002083D5056417D501001305E51897B0A6
:1040F0000100E780C010294597B00100E780001556
:1041000097170020238C875097F7FF1F9387C72AA4
:10411000DC4717F5FF1F0345E57403D70700C167A8
:10412000FD17631EF700B7E7040003A38705130616
:10413000000A85452244B240924441010283B7E718
:10414000040003A387051306001493050010DDB7D0
:10415000B1C1411122C417C501001305A56A2E84FF
:1041600097D50100938545DB06C697B00100E7802F
:104170000009A28517D501001305C50E97B00100EF
:10418000E780E0072244B2402945410117B301000E
:104190006700C30B8280B7E70400FC471171A2DD02
:1041A000CAD986DFA6DBCED72E8432892E86AA8591
:1041B00017050020130505F782971707002013073E
:1041C00067F683470700930680029387E70793F714
:1041D000F70FE3ECF610BA898A0717C70100130737
:1041E000A76BBA979C43BA9782878D4797D50100F2
:1041F000938505DD17C501001305C560630FF40045
:1042000097B00100E780A0FF17D501001305059ABC
:1042100097B00100E780A0FEBDA497B00100E78041
:1042200000FE17D501001305E59997B00100E7805E
:1042300000FD294597B00100E7804001930720F871
:104240001146970500209385E5ED4A851707002064
:10425000230AF7EC97070020A38707EC97000000DC
:10426000E780A0BC2A841DC997D50100938545D558
:1042700017C501001305055997B00100E78020F824
:10428000A28517D501001305A59797B00100E78017
:1042900000F7294597B00100E78040FB97D5010062
:1042A000938505D217C501001305C55597B00100C8
:1042B000E780E0F417D501001305C59597B001001C
:1042C000E780E0F3294597B00100E78020F84165D9
:1042D000930730FA0546970500209385A5E47D15E0
:1042E000170700202300F7E497000000E780E0B301
:1042F0002A841DC997D50100938585CC17C5010077
:104300001305455097B00100E78060EFA28517D5EF
:1043100001001305E58E97B00100E78040EE2945C6
:1043200097B00100E78080F2B7E70400BC4F056654
:10433000130606C8A14517F5FF1F0345A55282972E
:10434000FE506E54DE544E59BE5911618280914721
:104350006303F40297D50100938585C617C5010054
:104360001305454A97B00100E78060E917D50100C1
:104370001305858D71BDB7E70400FC4F914517F516
:10438000FF1F0345254E829797D50100938545C3AE
:1043900017C501001305054797B00100E78020E627
:1043A00017D501001305058C97B00100E78020E5C3
:1043B000294597B00100E78060E997500000E78049
:1043C000600F914535A485476303F40297D501003A
:1043D000938505BF17C501001305C54297B00100BD
:1043E000E780E0E117D501001305458915B597076A
:1043F0000020239127CBB7E704000566BC4F1306C6
:1044000006C8C1450DBF8D476303F40297D501006F
:10441000938505BB17C501001305C53E97B0010084
:10442000E780E0DD17D5010013050587D5B39307B5
:1044300040F81146970500209385C5CE4A85170799
:1044400000202301F7CE97070020A38E07CC97000A
:104450000000E780809D2A84E30405EE97D50100E3
:10446000938505B617C501001305C53997B001003E
:10447000E780E0D8A28517C501001305657897B0DD
:104480000100E780C0D7294597B00100E78000DC34
:1044900045BD9147E31CF4F6B7E70400FC4F9305D4
:1044A000000217F5FF1F0345E53B829797D50100F2
:1044B000938505B117C501001305C53497B00100F8
:1044C000E780E0D317C501001305857EF1BD89475C
:1044D00063E3870297D50100938585AE17C5010078
:1044E0001305453297B00100E78060D117C5010080
:1044F0001305457D31BB9704002083C4C4C29707D0
:10450000002083C737C297D50100938565ABA2040D
:1045100017C501001305052FDD8C97B00100E7805A
:1045200000CEA28517C501001305057B97B00100D9
:10453000E780E0CCC204294597B00100E78000D1B4
:10454000C1849305D4FF93960401C1824A8693F5F2
:10455000F50F17050020130515BD97300000E78003
:10456000003AE35F90DC930750F817070020230B15
:10457000F7BA83C73900228697050020938585BA4C
:1045800085074A8517070020A30FF7B8970000009A
:10459000E780A0892A84E30505DA97D50100938591
:1045A00025A217C501001305E52597B00100E78096
:1045B00000C5A28517D501001305C5C9C9B589472E
:1045C00063E3870297D501009385859F17C5010096
:1045D0001305452397B00100E78060C217C50100AD
:1045E0001305457135B197500000E780A0ECA28516
:1045F00017050020130505B397600000E780809D34
:1046000081B38D476303F40297D501009385459BE1
:1046100017C501001305051F97B00100E78020BEF4
:1046200017C501001305C56EE5B6B7660200014661
:10463000B7750200054597E0FF1FE780801A9307D2
:1046400060F817070020230FF7AC97070020A38C12
:1046500007AC93070006170700202307F7AC89472C
:1046600017070020A302F7AC97070020238F07AAA3
:1046700097070020A38B07AAC1471707002023072D
:10468000F7AA930720F917070020A301F7AA3146DC
:1046900097070020A38DA7A897050020938585A8DC
:1046A0004A8597070020238407A897F0FFFFE7803B
:1046B000C0772A84E30605C897D501009385459005
:1046C00017C501001305051497B00100E78020B35A
:1046D000A28517C501001305256555B3B1476303CE
:1046E000F40297D501009385A58D17C50100130528
:1046F000651197B00100E78080B017C50100130570
:10470000656439B6B7E70400FC4F9305000417F55C
:10471000FF1F03452515829797500000E78080D939
:10472000B145F9B5914763E3870297D501009385B9
:10473000258917C501001305E50C97B00100E78036
:1047400000AC17C501001305A561D9B4970400207A
:1047500083C4849D9707002083C7F79CA204DD8C47
:104760008E04B77702006D14BE942286A68517C505
:1047700001001305256097B00100E78040A8B7E766
:104780000400FC472286970500209385F5992800B0
:10479000829793160401C1823000A685094597E0EF
:1047A000FF1FE78000042A8409C917C5010013050B
:1047B000255E97B00100E78060BC930770F819464A
:1047C00097050020938505964A8517070020230B3F
:1047D000F79497070020A389879497F0FFFFE7805D
:1047E000C0642A84E30E05B497C501009385457D16
:1047F00017C501001305050197B00100E78020A04F
:10480000A28517C501001305A55995B99947630BF2
:10481000F41297C501009385A57A17C50100130509
:1048200065FE97B00100E780809D17C50100130564
:10483000A558F9BA914763E3870297C501009385AC
:10484000257817C501001305E5FB97B00100E78047
:10485000009B17C501001305A5575DBA97040020FA
:1048600083C4848C9707002083C7F78BA204DD8C58
:104870008E04B77702006D14BE942286A68517C5F4
:1048800001001305255697B00100E7804097B7E770
:104890000400FC472286970500209385F5882800B0
:1048A000829793160401C1823000A6850D4597E0DA
:1048B000FF1FE78000F32A8409C917C5010013050B
:1048C000255497B00100E78060AB930780F8194644
:1048D00097050020938505854A8517070020230347
:1048E000F78497070020A381878497F0FFFFE78074
:1048F000C0532A84E30605A497C501009385456C3F
:1049000017C50100130505F097B00100E780208F5F
:10491000A28517C501001305E54F95B699476303B6
:10492000F40297C501009385A56917C50100130519
:1049300065ED97B00100E780808C17C50100130575
:10494000E54EF9B0B7E70400FC4F9305000417F5F6
:10495000FF1F034525F1829797500000E78080B53F
:10496000994579B18D476303F40297C5010093859A
:10497000256517C501001305E5E897B00100E7803C
:10498000008817C501001305E54B59B017C5010094
:104990001305454C97B00100E780409E1305C012F7
:1049A00097E0FF1FE780E099014597E0FFFFE78070
:1049B000A06E0D4597100000E780C038294597E0AC
:1049C000FF1FE780009897E0FF1FE78060888DBA9F
:1049D00099476303F40297C501009385655E17C587
:1049E0000100130525E297B00100E780408117C55B
:1049F00001001305E54629B817F7FF1F0347D772D3
:104A000097F7FF1F83C7477222075D8F9166BA969B
:104A1000C2061166C1821306F6EF8D476365D602A2
:104A200097F7FF1F938747999C4B17F6FF1F034685
:104A3000966F9386C7002DC203D6070069CA8907FF
:104A4000E39CD7FE89471307A0F8114697F5FF1F8F
:104A50009385456D4A8597F6FF1F2385E66C17F70A
:104A6000FF1FA302F76C97F0FFFFE780003C2A844A
:104A7000E308058C97C501009385855417C501008F
:104A8000130545D897A00100E7806077A28517C578
:104A900001001305253EE5B203D60700630EE60AC2
:104AA0008907E39BF6FE8D4779BF91476304F402C3
:104AB00097C501009385C55017C50100130585D41E
:104AC00097A00100E780A07317C501001305053CFE
:104AD0006FF00FF4B7E70400FC4F9305000817F5DB
:104AE000FF1F034525D88297C9B897C50100938554
:104AF000254D17C501001305E5D097A00100E780FB
:104B0000007017C501001305E5396FF06FF02390B1
:104B1000E70017F5FF1F1305258A97400100E7807E
:104B2000809A97C501009385A54917C50100130513
:104B300065CD97A00100E780806C17C501001305C3
:104B4000653797A00100E780806B294597A0010099
:104B5000E780C06F8147C5BD2390070017F5FF1F91
:104B60001305858597400100E780E09597C5010012
:104B70009385054517C501001305C5C897A0010019
:104B8000E780E06717C50100130545345DBF0111DB
:104B900022CC06CE26CA4AC8834705002A849DC770
:104BA00097C501009385853D17C50100130585C58F
:104BB00097A00100E780A0644C4017C501001305D1
:104BC000A57097A00100E7808063E1A05841B70776
:104BD000CF009387777D631DF7060359C50085478E
:104BE00004450356E5009716002083D686B363FC80
:104BF000270383C7040003C71400A207D98FC20785
:104C00007177C1871307C755639FE7006305D60C0B
:104C10006244F240CA8526854249D244056117E3C1
:104C2000FFFF6700E35B630AD600CA85268532C6AC
:104C300097E0FFFFE780C05A32466244F240CA85DF
:104C400026854249D244056117F3FFFF6700E3540C
:104C5000B707CC009387777D6317F70497C50100EA
:104C60009385C53117C501001305C5B997A001008B
:104C7000E780E0581C448356E4008355C40003C613
:104C8000070017C501001305A56597A00100E7807F
:104C900000576244F240D24442492945056117A3B6
:104CA00001006700A35AB707CE009387777D63049E
:104CB000F70297C501009385652C17C50100130500
:104CC00065B497A00100E78080534C4017C50100F0
:104CD00013054555FDB5F2406244D2444249056191
:104CE0008280B7E70400FC4741112E8606C622C425
:104CF00026C24AC02E842A89AA8517F5FF1F1305EC
:104D00006542829797C501009385452D17C501001F
:104D1000130545AF97A00100E780604E97F5FF1F90
:104D200083C5454017C50100130545D397A0010071
:104D3000E780E04C294597A00100E780205197F4D7
:104D4000FF1F9384243E83C70400414793870706CF
:104D500093F7F70F636AF75E17C70100130707BEE3
:104D60008A07BA979C43BA9782879D476307F402E4
:104D700097C501009385852617C50100130585A8F1
:104D800097A00100E780A04717C50100130585CD56
:104D900097A00100E780A04669AC97F7FF1F83C783
:104DA0007738DDCB17F7FF1F0347F73797F7FF1F5C
:104DB00083C7673722075D8F97F7FF1F83C7C73603
:104DC000C2075D8F97F7FF1F83C71736E207D98F9A
:104DD00017F7FF1F232EF73283C7640097C5010022
:104DE0009385C51F17C501001305C5A117F7FF1F40
:104DF000230FF73097A00100E780604097F7FF1F6F
:104E0000938707318C4317F6FF1F0346463017C5BB
:104E100001001305E5C697A00100E780403E294543
:104E200097A00100E780804297F7FF1FA38C072E11
:104E30002244B24092440249930700F817F7FF1F3B
:104E40002302F72E9D4517F5FF1F1305A52D4101E0
:104E5000175300006700031897700000E780C0E751
:104E600097F7FF1F2381A72C9357850017F7FF1F84
:104E7000A30BF72A935705012A8417F7FF1F230571
:104E8000F72A93578501014517F7FF1FA30EF7284F
:104E900097700000E780A0E897F7FF1F2387A728F7
:104EA00097C501009385851317C5010013058595E6
:104EB00097A00100E780A03417F6FF1F0346E626FF
:104EC000A28517C50100130525BDB1B7CD47630302
:104ED000F40297C501009385651017C501001305FD
:104EE000659297A00100E780803117C50100130586
:104EF00025BC79BD97F7FF1F83C7E72317F7FF1F6F
:104F000003475723A207D98FC207C18717F7FF1F8F
:104F1000231EF71E6345F004B7A71C81B7060001E6
:104F20000147938757DC17F5FF1F1305E593938619
:104F300036191946B305E50083C505000507AD8F91
:104F4000B387D702E318C7FE2167130707E0B3F75B
:104F5000E7029387072017F7FF1F2319F71AB7E710
:104F6000040003A387051306000A89452244B240C2
:104F70009244024917F5FF1F0345C58E4101028384
:104F80008D476303F40297C501009385250517C576
:104F900001001305258797A00100E780402617C56B
:104FA00001001305A5C0EDB317F4FF1F0344A417B8
:104FB00097F7FF1F83C7171797C501009385050251
:104FC000220417C501001305E5835D8C97A001003D
:104FD000E780E022A28517C501001305E5AE97A082
:104FE0000100E780C021294597A00100E780002645
:104FF0000D4697F5FF1F9385E512228597F0FFFF79
:10500000E780A0E2AA8421C197C50100938505FD30
:1050100017B501001305057F97A00100E780201E4A
:10502000A68517C50100130565AB97A00100E780B1
:10503000001D2244B240924402492945410117A370
:1050400001006700A32097F7FF1F23958704B7E7A8
:105050000400116603A38705130606E8914539B7D6
:105060008D476303F40297C50100938525F717B5B3
:1050700001001305257997A00100E780401817C5A6
:105080000100130565C129B317F4FF1F0344A409E8
:1050900097F7FF1F83C7170997C50100938505F48C
:1050A000220417B501001305E5755D8C97A001007A
:1050B000E780E014A28517C50100130565A397A03A
:1050C0000100E780C013294597A00100E780001880
:1050D0000D4697F5FF1F9385E504228597F0FFFFA6
:1050E000E780A0D4AA841DC197C50100938505EF70
:1050F00017B501001305057197A00100E780201086
:10510000A68517C501001305E59F05B797F7FF1F93
:10511000239487F6B7E70400116603A387051306F7
:1051200006E89305000299B5894763E3870297C5AE
:1051300001009385A5EA17B501001305A56C97A09A
:105140000100E780C00B17C501001305A5B789B1A1
:1051500097F4FF1F83C424FD97F7FF1F83C797FCB5
:1051600097C50100938585E7A20417B501001305D3
:105170006569DD8C97A00100E7806008A68517C5EA
:1051800001001305A59997A00100E7804007294574
:1051900097A00100E780800B228697F5FF1F93857B
:1051A00065F8268597F0FFFFE78020C82A84630E04
:1051B000051A97C50100938565E217B5010013052F
:1051C000656497A00100E7808003A28517C50100F0
:1051D0001305059699BD854763F98718834519001E
:1051E0002244B24092440249B335B00097F7FF1F02
:1051F000238CB7EA17C501001305C594410117A315
:1052000001006700C3FFA2852244B24092444A8550
:105210000249410117130000670003B9994763036E
:10522000F40297C50100938565DB17B501001305EE
:10523000655D97A00100E78080FC17C5010013059C
:1052400025C2B9B617F4FF1F0344E4ED97F7FF1F1B
:1052500083C757ED97C50100938545D8220417B53C
:1052600001001305255A5D8C97A00100E78020F905
:10527000A28517C501001305658E97A00100E78080
:1052800000F8294597A00100E78040FC194697F5F2
:10529000FF1F938525E9228597F0FFFFE780E0B89F
:1052A000AA841DC197C50100938545D317B5010098
:1052B0001305455597A00100E78060F4A68517C542
:1052C00001001305A58A95B397F7FF1F239487E480
:1052D000B7E70400116603A38705130606E89305E4
:1052E000000869B1854797C50100938525CF17B59B
:1052F000010013052551630BF40097A00100E7801E
:1053000000F017C501001305A58759B497A0010047
:10531000E780E0EE17C501001305058897A001009E
:10532000E780E0ED294597A00100E78020F22244C4
:10533000B2409244024997F7FF1F239907DC4101CD
:10534000177300006700C38997C50100938505C9DD
:1053500017B501001305054B97A00100E78020EA6F
:1053600017C50100130505B425B4B2402244924488
:10537000024941018280411106C622C426C239C1B8
:105380002A8497F00000E780C00DAA8411EDB7E7EA
:105390000400BC474146814522858297B2402244A1
:1053A000268592444101828041657D1597F0000079
:1053B000E780000CB7E7040001E9BC47414681459E
:1053C000228582978144D9BF0347E501FC479305B5
:1053D000900819E393050003AA9541462285829718
:1053E00085446DBF411106C622C426C24AC097F04B
:1053F0000000E780000755CD97700000E780808EA1
:105400002A8497100000E7804046AA8422856373AF
:1054100094002685B7D7B0009387F75E63F3A702A1
:10542000B7E7B000130514009387F74F63E3A708AD
:105430002244B240924402494101177300006700C0
:10544000238B8567938707F13E956364A40033053A
:10545000F40097700000E780A08997700000E78053
:1054600060882A8963F6A40097100000E780A042B4
:1054700097C50100938505B817B501001305853858
:1054800097A00100E780A0D7A6864A86A28517B517
:1054900001001305E54E97A00100E78040D62244A5
:1054A000B240924402492945410117A30100670017
:1054B000E3D9B24022449244024941018280011161
:1054C00022CC37E404005C5C06CE354697C501006B
:1054D000938585BB17D501001305058F829711E9C8
:1054E00017B501001305C53797A00100E78000E953
:1054F00001A097E7FF1F9387A7373EC4B7F50700C2
:10550000856793870780814617E6FF1F1306C63518
:10551000E10519453EC697D0FF1FE780802C7C44EB
:10552000194697E5FF1F9385253417F5FF1F1305CF
:10553000A5B68297340017E6FF1F1306E63297C51B
:105540000100938565FD17C50100130565FE976091
:105550000000E780002E2A841DCD97C501009385A9
:10556000E5A317B501001305E52997A00100E78021
:1055700000C9A28517C50100130505B297A0010057
:10558000E780E0C7294597A00100E78020CCF240E2
:1055900062440561828097E00000E780409317C570
:1055A0000100130565A697500000E7804022975040
:1055B0000100E780804C17E5FF1F130565DC97505D
:1055C0000100E780203517C501001305E5A49750B9
:1055D0000100E780004D2A8497600000E780008981
:1055E00097000100E780602497800100E78080BD7C
:1055F00097700000E780E0E497600000E78000FF1C
:1056000097300100E780C0E597C5010093850599B3
:1056100017B501001305051F19C897A00100E78001
:1056200000BEA28517C50100130545A981BF97A03B
:105630000100E780C0BC17C50100130565AA97A04B
:105640000100E780C0BB294597A00100E78000C0AA
:1056500097300100E780A0C197F00000E78060E08C
:1056600069CD97E7FF1F9387A7C483D707008545B8
:1056700037050400170700202315F70A97200000BC
:10568000E780202497C501009385459117B5010057
:105690001305451797A00100E78060B617C5010004
:1056A000130585A597A00100E78060B5294597A05F
:1056B0000100E780A0B98547170700202300F7F60F
:1056C00097E7FF1F938747CFDC4703D70700C167E2
:1056D000FD176316F70097F0FFFFE780A0839700A0
:1056E0000000E78060D097100000E78020EC1705ED
:1056F00000200355050397400000E780206305451F
:1057000097500000E780009697500000E78080BB2C
:1057100097C501009385858817B501001305850E8F
:1057200097A00100E780A0AD17C50100130505A2F1
:1057300097A00100E780A0ACB1B597C501009385A3
:10574000E58517B501001305E50B97F7FF1F239FAC
:10575000079A97A00100E78080AA97C5010093856A
:10576000E59B17C501001305E59B97A00100E780A5
:1057700000A9294597A00100E78040AD0145975059
:105780000000E780208E69B7411122C437E404008D
:105790008327041A06C6829797400000E780C05C02
:1057A000832704081705000013050503829797E770
:1057B000FF1F2389A70A17E5FF1F1305E5BF9740C1
:1057C0000000E780E0052244B240410117030000D9
:1057D000670023CF011122CC06CE26CA4AC84EC686
:1057E00093F715002E84B5CB97E0FFFFE78080721A
:1057F000930710F817F7FF1F2306F79297F7FF1F7D
:1058000083D7078717F7FF1FA30EF7909145A18352
:1058100017F5FF1F1305059117F7FF1F2305F790D5
:1058200097F7FF1FA381079097400000E780807AD9
:10583000B7E70400BC4F130600149305001017E5EA
:10584000FF1F03452502829713451400F24062446E
:10585000D2444249B2490561828093F70510B1C72D
:10586000054597400000E780E07F170500200355BD
:1058700045EB97400000E780604B97000000E78011
:10588000A0B697100000E78060D297F7FF1F83C78C
:10589000B79889E797500000E78000A19750000073
:1058A000E78040A21345041055B793F72500E9CFD0
:1058B00017F7FF1F0357878569C7AD64B719004005
:1058C0009384A4AA23A0990097F6FF1F9386468489
:1058D000944297C701009387279D17F6FF1F034641
:1058E0000683814517C501001305059D97600000DB
:1058F000E780201F23A0990097E7FF1F2392A79C12
:105900002A8941C197B501009385456A17B5010001
:10591000130545EF97A00100E780608ECA8517B593
:1059200001001305A50897A00100E780408D2945D7
:1059300097A00100E780809197E7FF1F2398077CDD
:10594000930710F817E7FF1F230EF77C97E7FF1F59
:1059500083D7077217E7FF1FA306F77CA18317E71A
:10596000FF1F2302F77C91458D4717E5FF1F1305A5
:10597000657B17E7FF1FA308F77A97400000E780D1
:10598000606513452400D9B593F74500D1C397B599
:1059900001009385A56117B501001305A5E697A041
:1059A0000100E780C08517B501001305E50197A048
:1059B0000100E780C084294597A00100E7800089A5
:1059C000930720F817E7FF1F230EF77497E7FF1FD1
:1059D00083D7476C17E7FF1FA306F774A18317E768
:1059E000FF1F2302F774854717E7FF1FA30DF77208
:1059F00097400000E78000AC17E5FF1F1305857294
:105A0000914597400000E780E05C134544003DBDB0
:105A100093F78500A9C797B501009385255917B558
:105A20000100130525DE97900100E780407D17B542
:105A300001001305A5FA97900100E780407C2945F5
:105A400097A00100E780808097E7FF1F2390076CF5
:105A500097600000E780C01813458400C5BB93F72A
:105A60000501D1C3854517E5FF1F0355A562975072
:105A70000100E780C0CD97B501009385255317B588
:105A80000100130525D897900100E780407717B5EE
:105A900001001305E5F597900100E7804076294560
:105AA00097900100E780807A930730F817E7FF1F8F
:105AB000230AF76697E7FF1F83D7C75D17E7FF1F26
:105AC000A302F76617E5FF1F1305C565A1838D4582
:105AD00017E7FF1F2309F76497400000E780804F16
:105AE00013450401A5B393F70502D1C797B501008B
:105AF0009385C54B17B501001305C5D097900100DC
:105B0000E780E06F17B501001305C5F0979001001D
:105B1000E780E06E294597900100E78020739307A6
:105B200040F817E7FF1F230FF75E97E7FF1F83D7A4
:105B3000A75417E7FF1FA307F75EA18317E7FF1F0F
:105B40002303F75E854717E7FF1FA30EF75C97E770
:105B5000FF1F2393075297400000E780A09517E5A9
:105B6000FF1F1305255C914597400000E7808046A4
:105B700013450402E1B993F70504FDC397B501008D
:105B80009385C54217B501001305C5C7979001005D
:105B9000E780E06617B50100130545E9979001001D
:105BA000E780E065294597900100E780206A97E744
:105BB000FF1F83C727571307700A6386E70613077B
:105BC000800A638CE7081307600A6393E70493076E
:105BD00060F817E7FF1F2307F75497E7FF1F83D7E6
:105BE000C75217E7FF1FA30FF752A18317E7FF1F45
:105BF000230BF752854717E7FF1FA30AF752B1455A
:105C000017E5FF1F1305055297400000E780803C11
:105C100097400000E780008A1345040497E7FF1FC0
:105C20002395074E25B1930770F817E7FF1F230B45
:105C3000F74E97E7FF1F83D7474D17E7FF1FA303D3
:105C4000F74EA18317E7FF1F230FF74C854717E790
:105C5000FF1FA30BF74C994565B7930780F8F1B781
:105C600093F705080145E38307BE97B501009385C7
:105C7000E53317B501001305E5B897900100E780FB
:105C8000005817B501001305E5DB97900100E78088
:105C90000057294597900100E780405B9307A0F8E3
:105CA00017E7FF1F2300F74897E7FF1F83D78746B3
:105CB00017E7FF1FA308F746A18317E7FF1F230479
:105CC000F746854717E7FF1FA30FF74497E7FF1F26
:105CD0002392074497300000E780C07D17E5FF1F3F
:105CE00013054544914597400000E780A02E1345D9
:105CF0000408A9BE411106C697E0FFFFE780C00B6C
:105D00000DC197E7FF1F83D7473A850717E7FF1FA6
:105D1000231DF73897E7FF1F239AA738B2404101A8
:105D2000828097E7FF1F83D78738850717E7FF1F14
:105D3000231FF736E5B78546170300006700C3FB4E
:105D4000411122C491462A8417E6FF1F1306864B91
:105D50009D652D4506C697D0FF1FE78080A8B7F741
:105D6000070003C70701A5476313F70001A09306C7
:105D7000001001469D65254597D0FF1FE78060A66E
:105D800097E7FF1F238087482244B240914617E6D9
:105D9000FF1F130626479D652945410117D3FF1FA5
:105DA000670023A41171CED7B7E9040083A7C90403
:105DB000CAD917E9FF1F1309E936A2DD2E8686DF4F
:105DC000A6DB2E84AA854A85829797E7FF1F83C7A3
:105DD00067351307700A6385E710636DF7001307D3
:105DE000600A6385E704FE506E54DE544E59BE5976
:105DF000116182801307800A6385E7161307900AF2
:105E0000E393E7FE8D476306F41C97B50100938585
:105E1000A55817B501001305E59E97900100E7808E
:105E2000003E17B501001305655425A08D47630C8E
:105E3000F40297B501009385255617B501001305A7
:105E4000659C97900100E780803B17B50100130522
:105E5000254B97900100E780803A294597900100F3
:105E6000E780C03E49B7854717B501001305054BCC
:105E700017E7FF1F230AF72297900100E7800050E1
:105E8000B7750200B76602000146054597D0FF1FAF
:105E9000E7802095930760F817E7FF1F2304F72892
:105EA00097E7FF1FA38107289307002617E7FF1F27
:105EB000232CF726E5779387072117E7FF1F231782
:105EC000F726B14597E7FF1F2383072697E7FF1FB4
:105ED000A38FA7244A8597000000E780E01621B72A
:105EE000914763E3870297B501009385E54A17B5AB
:105EF00001001305259197900100E780403017B508
:105F000001001305A543B1B797E4FF1F83C4C42163
:105F100097E7FF1F83C73721A204DD8C83A7C9043D
:105F20006D14228697E5FF1F938515202800829720
:105F30008E0493160401B7750200C1823000A69545
:105F4000094597D0FF1FE780C089930770F817E7CE
:105F5000FF1F2309F71C994597E7FF1FA386A71C7E
:105F600095BF914763E3870297B501009385C542CA
:105F700017B501001305058997900100E7802028D7
:105F800017B501001305053DE9B597E4FF1F83C46C
:105F9000A41997E7FF1F83C71719A204DD8C83A7F5
:105FA000C9046D14228697E5FF1F9385F517280015
:105FB00082978E0493160401B7750200C1823000E7
:105FC000A6950D4597D0FF1FE780A081930780F825
:105FD000BDBF17B501001305A53A97900100E780F2
:105FE000E039930790F82304F100834719008D45A9
:105FF0002800A304F100834729002305F10097003E
:106000000000E78060041305C01297C0FF1FE780FF
:106010004033014597D0FFFFE78000080D4597000A
:106020000000E78020D2294597C0FF1FE78060313C
:1060300097C0FF1FE780C0217DB397E7FF1F23AB09
:10604000A71C828097E7FF1F9387C71C03A3070045
:10605000630303000283174300006700A3F74111A5
:106060004AC097F6FF1F83D6C66B328917D6FF1F2B
:106070000356A63622C426C206C62A84AE849700DA
:106080000000E780E06929C921C8994763F69704B1
:106090008347140003470400A207D98F1397870092
:1060A000A183D98FC2073167C1831307C755639591
:1060B000E70297D7FF1F83D74732A301F400A183DC
:1060C0002302F40097F7FF1F83D7A76591C7A302A8
:1060D000F400A1832303F40097F7FF1F83C707543D
:1060E000A1CB2686A28517D5FF1F0355052F970044
:1060F0000000E78080C4630F090297F7FF1F83C782
:10610000E7518DEB97E7FF1F83C7071185C79DC038
:1061100097E7FF1F83C747F991EF22852244B240DA
:106120000249A6859244410117430000670083EAB3
:10613000E31A09FCB24022449244024941018280A0
:106140000145828097A701009387475C9C4301111A
:106150006800914506CE3EC697000000E780C0EE7D
:10616000F240056182808D4763F6B708011126CAA7
:1061700006CE22CC0344350097E4FF1F83C4D40924
:1061800097B5010093850523B337800017E7FF1FFC
:10619000A304F70809C497B501009385652217B5D4
:1061A00001001305652297900100E780400597E7FD
:1061B000FF1F83C777066386970097000000E7807C
:1061C000404697400000E780E00F9967938757EEBD
:1061D0002316F100680085479145A3078100230736
:1061E000F10097000000E78020E6F2406244D244CC
:1061F000056182808280894763F7B708011122CC4C
:1062000006CE26CA8344250085472A84639DF4046C
:10621000914763F5B70403454500834734002205E1
:106220005D8D97D7FF1F239AA71A97000000E7807C
:1062300000589967938767EE2314F1008347340071
:1062400023059100A305F1008347440095452800EC
:106250002306F10097000000E78000DFF24062446F
:10626000D24405618280FDF89967938767EE231415
:10627000F10097D7FF1F83D74716A305F100230529
:106280000100A183E1B782800111996722CCD51763
:1062900017F4FF1F130484382314F100834704000C
:1062A00026CA97F4FF1F9384C4472305F10083D7C0
:1062B000040028009545A305F100A18306CE23061E
:1062C000F10097000000E78020D803D60400834542
:1062D000040017B501001305251097900100E78011
:1062E00000F2F2406244D244056182809D67797178
:1062F000D9172316F10097F7FF1F9387273283C71B
:1063000007001305F10006D62307F10097F0FFFF01
:10631000E780A00609E9B7E70400BC47414681458C
:106320001305F10082976800CD4597000000E780D3
:10633000A0D197F5FF1F83C5652E17B50100130582
:10634000A50C97900100E78080EBB25045618280F8
:1063500063080516411126C206C622C44AC097E743
:10636000FF1F83C777EB97F4FF1F83C4242B99C3C8
:1063700093E424002A8497100000E780C00119C12B
:1063800093E4040137E90400832789042285130676
:10639000200381458297930750FA2300F400930766
:1063A000A005A300F4008D472301F4009147A30149
:1063B000F4009307E005A302F40097F7FF1F83D7CB
:1063C00047362304F400A183A304F40097D7FF1FEA
:1063D00083D7A700230394002305F4009304C4008B
:1063E000A18323020400A305F400268597F0FFFF94
:1063F000E780A0F819E58327890441468145268571
:10640000829797D7FF1F83D7E7FA230EF400A18363
:10641000A30EF40093070002230FF400930710FA71
:10642000A30FF4009D472300F402A3000402B7E782
:106430000400FC4713052402194697D5FF1F9385D6
:10644000A542829797E7FF1F83D767C62304F4020C
:10645000A183A304F40297E7FF1F83D707C5230591
:10646000F402A183A305F40297E7FF1F938707C4F3
:10647000839707002285930500032306F402C207D1
:10648000C183A183A306F40297D7FF1F938747E335
:10649000839707002307F402C207C183A183A307E0
:1064A000F40297000000E780A0232308A4022181C2
:1064B000A308A402B24022449244024941018280CE
:1064C00082805D71E17793C777FF1305E10086C68F
:1064D0002316F10097000000E780C0E768009305ED
:1064E000400397000000E78020B6B64061618280DB
:1064F0005DC9411122C426C206C6930750FA230083
:10650000F5009307A005A300F50089472301F500D6
:106510009147A301F5009307E005A302F50097F763
:10652000FF1F9387A70F83C707009304C5002A8422
:106530002303F50097E7FF1F938717CE83C7070054
:1065400023020500A303F50097F7FF1F83D7671DFC
:106550002304F500A183A304F50097D7FF1F83D779
:10656000C7E72305F500A183A305F500268597F06D
:10657000FFFFE78080E001E9B7E70400BC47414640
:106580008145268582972285F14597000000E780A6
:106590002015230EA4002181A30EA400B2402244A2
:1065A00092444101828082805D710A8586C6A2C4C0
:1065B00097000000E78000F437E404007C448A85FB
:1065C0000810794682973C441305E103094681454A
:1065D0008297101093050002014597D0FFFFE780D6
:1065E000E011B640264461618280411122C426C276
:1065F0002A84AE848566AA850146254506C697C0CD
:10660000FF1FE780001EA2852244B24026869244E6
:10661000A1462945410117C3FF1F6700831C0111D3
:10662000B7C7A55A22CC9387C73317E4FF1F1304BB
:10663000B4BE3EC4834704002C00196506CE3EC696
:1066400097000000E780A0FA8345040017B5010019
:10665000130505E697900100E78060BAF2406244B6
:10666000056182800111A146300099652D4522CC3B
:1066700006CE97C0FF1FE780C016A24737C4A55AB1
:106680001304C43363958702B24517B5010013059F
:10669000E5D9B335B00097E7FF1FA38FB7B6979042
:1066A0000100E780C0B5F2406244056182809165D7
:1066B000A1463000938505F02D4597C0FF1FE78068
:1066C0004012A247E38287FC97E7FF1FA38607B427
:1066D000814517B501001305A5D7D1B7C167697604
:1066E0008146FD1705061397060141836364B700D1
:1066F0003E8582803307D50003470700B98F2147C5
:1067000013F81700858363050800B18FC207C183A2
:106710007D171377F70F6DF78506F1B741C5A547CC
:10672000054763F2B7088347150003470500316842
:10673000A207D98F13978700A183D98FC207C1837E
:106740001308C855054763900707411106C622C4C0
:1067500026C203442500914763F087049307540041
:1067600063ECF502A301C50021822302C500930456
:10677000340091C6A302D500A1822303D5002A8448
:10678000A68597000000E780A0F526942300A400CA
:106790002181A300A4000147B240224492443A85DB
:1067A0004101828005473A8582800111B7C7A55A09
:1067B00022CC9387E7342A842AC62C00156506CE9E
:1067C0003EC497000000E78080E2A28517B5010073
:1067D000130505D097900100E78060A297000000A4
:1067E000E780C0DCF2406244056182800111A1466D
:1067F000300095652D4522CC06CE97C0FF1FE7805F
:1068000040FEA24737C4A55A1304E43463958702B7
:10681000B24517B501001305A5C597D7FF1F239EE5
:10682000B7BAC205C18197900100E780409DF24050
:106830006244056182809165A1463000938505EE32
:106840002D4597C0FF1FE780C0F9A247E38287FC70
:10685000D14717D7FF1F2312F7B8D14517B501004D
:10686000130505C3C9B70111A146300091652D4537
:1068700006CE97C0FF1FE780C0F62247B7C7A55ACC
:106880009387073501456313F7003245F2400561F0
:1068900082800111B7C7A55A2AC6938707352C00F5
:1068A000116506CE3EC497000000E78040D4F24058
:1068B000056182804DC5411126C206C622C4AE8440
:1068C000D1C92A8497100000E78080AD97E7FF1FA9
:1068D00083C7879499C7A685228597300000E780F3
:1068E000606F97F7FF1F83C767D3ADC7954763F303
:1068F00097068347040013073005639DE70483462A
:106900001400130750046397E6048346240013071A
:1069100010046391E60403473400631DF702034744
:1069200044009307B0046317F7020347540093072A
:1069300090056311F702A2852244B2402686924454
:1069400017D5FF1F035565A98D46410117F3FFFFBA
:106950006700833AB240224492444101828082809F
:1069600001114EC606CE22CC26CA4AC893F715009E
:10697000AE899DCBAD67371700409387A7AA1CC38C
:10698000B7E70400BC4F13060019854517D5FF1F54
:10699000034585A4829713C51900F2406244D2448E
:1069A0004249B2490561828093F725000145F5D738
:1069B00017F7FF1F0357C7D6954763F9E70C014444
:1069C00017F6FF1F1306C6C59306300513055004BE
:1069D000130810049308B004130390059307640090
:1069E0006374F7043A847D5997F4FF1F83C444C34A
:1069F00097F7FF1F83C7D7C2A204DD8CAD679387CB
:106A0000B755638BF41463E3970AA9679387A75577
:106A1000638EF414A28517F5FF1F130565C0970058
:106A20000000E78060E9E9A0B307860083C507009E
:106A3000639AD50483C517006396A50483C5270010
:106A40006392050583C53700639ED50283C5470061
:106A5000639A150383C757006396670222890DE87E
:106A600097F5FF1F83D5C5CBB3852541C20517F523
:106A7000FF1F1305E5BAC1814A9597000000E78022
:106A8000A0E3E1A005044204418089BF3A847D5916
:106A90008547E3EB87F45DC4854517F5FF1F1305B4
:106AA00025B897000000E78020E169A8B1679387C7
:106AB000C7556389F404B5679387D755E39CF4F40D
:106AC000A28517F5FF1F1305A5B597300000E780D5
:106AD00060508947630EF4009305E4FFC205C1814D
:106AE00017F5FF1F1305E5B397100000E780408BF3
:106AF000A68517B501001305659F97800100E78003
:106B0000007089A097200000E780603A971000008D
:106B1000E780608811C9A28517F5FF1F130545B0EE
:106B200097100000E780C0870546A28517F5FF1F74
:106B3000130505AF97F0FFFFE780A05297200000F4
:106B4000E780E036FD57E31DF9F097F7FF1F239923
:106B500007BC13C5290091B5A28517F5FF1F1305C2
:106B600025AC97F0FFFFE780E05D59B7A28517F5E8
:106B7000FF1F1305E5AA97F0FFFFE780E05C8DBFDC
:106B8000411122C437E404005C5C06C6354697A573
:106B900001009385654F17B501001305E522829723
:106BA00011E917B501001305A59597800100E7804D
:106BB000E07C01A08327041C82972A84054597C0A6
:106BC0000000E780203097700100E78040B59770A3
:106BD0000100E780408A97B00000E780A04122854D
:106BE000B2402244410182804111054506C622C4BB
:106BF00026C297C0FFFFE78000341305A00497B0BA
:106C0000FF1FE780C04A757585457D1597C0FFFF5A
:106C1000E780A01D7D7585451305F53697C0FFFFFC
:106C2000E7800027371400408327840A8D45130529
:106C3000002093E707202324F40A97C0FFFFE78092
:106C4000C01AB7E4040097C0FFFFE780E05FC858B0
:106C500097800100E780807217B501001305C51603
:106C600097800100E78080718327840C854541452A
:106C700093E707082324F40C97C0FFFFE780402127
:106C80008D451305000897C0FFFFE780602097C07F
:106C9000FFFFE780404D37A507001305051297C099
:106CA000FFFFE780E048014597C0FFFFE780004F06
:106CB00095450545894717F7FF1F2305F7A697C098
:106CC000FFFFE780404FB7E700E013070006238D82
:106CD000E7403707000423A0E71097D0FFFFE780C5
:106CE000C0D097D0FFFFE780C0E297000000E780A8
:106CF00060E997000000E780209797000000E78098
:106D000020AF97F0FFFFE78060A897000000E780C2
:106D1000606A97000000E780801083A704081705C9
:106D20000000130525C4829797C7FF1F2386A76A13
:106D3000BC4C130600648545829797B0FF1FE7801F
:106D4000206B01458280AD67371700409387A7AA63
:106D50001CC3B7E700E03707400023A0E718010095
:106D60000100B7F7070003C70701A5476316F7003F
:106D70009397450191C301A04111AE860146AA85B2
:106D8000254506C697C0FF1FE780A0A5B240B7E71C
:106D900000E03707400023A0E71041018280411145
:106DA000B2862E86AA852D4506C697C0FF1FE780AE
:106DB00040A3B2400145410182809307000463EC87
:106DC000C7041D71A2CC2A840808A6CACAC886CEE8
:106DD00032C697800100E7802037AD673717004043
:106DE0009387A7AA1CC3B7E400E03709400023A09B
:106DF000241901000100B2461008A285294597C058
:106E0000FF1FE780009EF640664423A02411D6446D
:106E10004649256182803955828041110D658D4535
:106E200006C697C0FFFFE78040FCB71700408D669D
:106E300023A6D70A17F5FF1F1305058F1387C70A67
:106E40009387870A1CC15CC5856689675CC958C180
:106E500014C518C9B7E70400B24003A3871E410157
:106E600002838145B307B5008387070089E71723AD
:106E700000006700630A8505C205C181E5B74111BD
:106E800006C6B94763EEB70017A501001305C57F15
:106E900097000000E78020FDB24005454101828057
:106EA0008347E500130710036390E702854717F750
:106EB000FF1F230DF79617A501001305257F97F7F0
:106EC000FF1F23940796E9B713070003E39EE7FA31
:106ED00097F7FF1F238C079497F7FF1F23970794BB
:106EE00017A501001305057E65B7411126C2E97794
:106EF00097F4FF1F9384C49322C49387A7552E84CD
:106F00002381B4002E86AA8517F5FF1F13058592ED
:106F100006C62390F400A381040097800100E78057
:106F2000A02293052400C205C18117F5FF1F130598
:106F3000459097F0FFFFE780A07AB3878400238213
:106F4000A7002181A382A700930564002244B240D8
:106F500026859244C205C1814101172300006700C4
:106F6000A3FB09C99307000463E6B70017030000F9
:106F70006700E3F782809306F00F0307060019E726
:106F80009307F00F63F0B7022E8582809387150078
:106F9000C207C183E3E6F6FEAA952380E500050655
:106FA000BE85E1BF2E9523000500F9BF01111C0825
:106FB000B69706CE238A07FE5C00BE9617A801008E
:106FC0001308487C1377F600429703470700FD1625
:106FD00011822380E600E397D7FE3E8697000000EB
:106FE000E780A0F9F240056182800111580006CEC9
:106FF00023070100A947BA8829482543B376060329
:10700000FD1793F7F70F93860603A304D700B35633
:1070100006036375C3007D173686EDF33386F800EB
:1070200097000000E78060F5F240056182803971C9
:1070300017A601001306866D06DE22DC26DA2A84F6
:107040004AD84ED697000000E78020F3AA8517E6BD
:10705000FF1F0356066D9146228597000000E780CA
:1070600020F597E7FF1F83C7675BAA8517A6010076
:107070001306466789C717A60100130626662285F0
:1070800097000000E78060EFAA8517A601001306AD
:107090002668228597000000E78020EEAA8517A6C3
:1070A000010013066667228597000000E780E0EC88
:1070B000AA851146228597000000E78040F3AA8543
:1070C00017B60100130646C4228597000000E7802A
:1070D000C0EAAA8517A601001306866422859700D8
:1070E0000000E78080E9AA8517B601001306C6C133
:1070F000228597000000E78040E8AA851306E00596
:10710000228597000000E78080EE97D7FF1F83C796
:10711000B710AA8517A601001306465D89E717A6D2
:1071200001001306265D228597000000E780E0E459
:10713000AA8517A601001306E65E228597000000C7
:10714000E780A0E337A60700AA851306061222856A
:1071500097000000E780A0E9AA8517A601001306A2
:10716000E65C228597000000E78020E197E7FF1F9B
:1071700083C7075DAA8517A601001306265889E76D
:1071800017A6010013060658228597000000E78025
:10719000C0DEAA8517A601001306065A22859700AD
:1071A0000000E78080DDAA8517A601001306465976
:1071B000228597000000E78040DCAA8517A6010021
:1071C00013068658228597000000E78000DB914671
:1071D000AA8517C6FF1F0356E61D228597000000EB
:1071E000E78000DD2AC697500000E780A0AFB245D7
:1071F000AA8417A601001306665522859700000091
:10720000E780A0D713D60401AA8589461376F60F26
:10721000228597000000E780A0D9139604019146CB
:10722000AA854182228597000000E78060D8AA8560
:1072300017A6010013060652228597000000E7807A
:10724000C0D39146AA8517C6FF1F0356061922858B
:1072500097000000E780C0D5AA8517A60100130695
:10726000E64F228597000000E78020D19146AA854D
:1072700017D6FF1F0356A6E3228597000000E7807C
:1072800020D3AA8517A601001306C64D22859700B4
:107290000000E78080CE9146AA8517D6FF1F0356CF
:1072A000C6E0228597000000E78080D0AA8517A657
:1072B00001001306A64B228597000000E780E0CB73
:1072C0009146AA8517D6FF1F035646DE22859700F2
:1072D0000000E780E0CDAA8517A601001306464905
:1072E000228597000000E78040C9AA85914617C60D
:1072F000FF1F0356E6FC228597000000E78040CB85
:10730000AA8517A6010013062647228597000000CC
:10731000E780A0C6AA85814497C9FF1F9389C954F5
:107320001949B387340103C60700894622859700AF
:107330000000E780E0C78504AA85E39424FF17A630
:1073400001001306E643228597000000E780E0C2B3
:107350002AC6080897E0FFFFE7802002B24504082C
:107360001309010283C7040003C614009146A20753
:107370005D8E228597000000E78080C38904AA857E
:10738000E31299FEF2506254D2544259B25921612B
:10739000828017E5FF1F0345A53A828097E7FF1F0C
:1073A00083C7C74889E7172300006700E3B68280D8
:1073B00097E7FF1F83C7274C99EF411106C6972017
:1073C0000000E78040ADB240854717E7FF1F230468
:1073D000F74A4101828082806302054E6380054E38
:1073E0002971B7064000232E1112232C8112232A63
:1073F00091122328211323263113232441132322FE
:10740000511323206113232E7111232C8111232A60
:1074100091112328A1112326B11101475948A5062E
:107420009319070193D9090163F1B902B307E50084
:1074300083C70700D91793F7F70F6368F800B3D72E
:10744000F600858B13061700A1E3B3893541C20905
:1074500093D90901B9472E89AA8463F93703330404
:10746000E500394697A50100938545102285978050
:107470000100E78000CB19E9CE8522859700000046
:10748000E78020A025E5F1A4328759BF97E7FF1FC9
:1074900083C7C739638F0724BD6A396C014A17EB6C
:1074A000FF1F130B2B2A938BFA55938CFA66130D3F
:1074B000EC5505A8B387440183C6070097E7FF1F73
:1074C00083D7A736A5E39307A005639BF6008547FE
:1074D00017E7FF1F231BF73497E7FF1F2384D726E7
:1074E000050A93170A01C183E3E627FD8320C11330
:1074F0000324811383244113032901138329C11217
:10750000032A8112832A4112032B0112832BC111FA
:10751000032C8111832C4111032D0111832DC110E6
:1075200031618280854D639BB7039307500A639E48
:10753000F600894717E7FF1F2319F72E930750FA24
:1075400017E7FF1FA300F72061BF9307A005E3899A
:10755000F6F897E7FF1F239A072C59B713871700F0
:107560004207DA9741832380D70017E6FF1F231EC7
:10757000E62A8D47E3F6E7F617E4FF1F0344B41C41
:1075800097E7FF1F83C7271C22045D8C9307F4FF36
:10759000C207C1839306F00DE3EDF6FA930764008A
:1075A000C207C183E31EF7F293052400C205C1811F
:1075B00017E5FF1F1305251997F0FFFFE78040121D
:1075C00033078B008347570003474700A207D98F33
:1075D00017E7FF1F231B07246312F5108149630D72
:1075E000B40197E9FF1F83C92916A20997E7FF1F76
:1075F00083C79715B3E9F900170500001305A59691
:1076000097F0FFFFE780A0A36385790963EF3B0351
:107610006388A9059307EC656383F90697E7FF1F65
:1076200083C7871205476380E70881CB1387A705C7
:107630001377F70F8D4663F9E6081307F007230069
:10764000E100A300F100894595A863899905938716
:10765000FA77E395F9FC97F0FFFFE780C0E611A801
:10766000A28517E5FF1F1305250E97F0FFFFE780A2
:10767000C0AF014597F0FFFFE780609C95B5A285FC
:1076800017E5FF1F1305450C97F0FFFFE780E0B6F5
:10769000CDB797F0FFFFE78060BFE1BF97F0FFFF36
:1076A000E78000C5F9B7930710F813051100230010
:1076B000F10097F0FFFFE780E0E3FD450A859700C2
:1076C0000000E780C08275B7A28517E5FF1F13058C
:1076D000A50797E0FFFFE780206D61BF9307F007E4
:1076E00089450A852310F10097000000E78020807B
:1076F000C5BB15476375270503C604009306500BE9
:107700000147631FD60203C614009306B0053E87E7
:107710006318D602CA85268597F0FFFFE78080A20E
:1077200011C917A50100130565E597F0FFFFE78074
:1077300080736DBB17A50100130585E5FDB70147F3
:10774000B70640005946A506131407014180636936
:107750002401CA85268597C0FFFFE78060A879B31A
:10776000B389E40083C70900D91793F7F70F63675C
:10777000F600B3D7F600858B0507F9F73304894087
:1077800042044180BD4763FD8706414697A501003D
:10779000938505E24E8597800100E780809817A6C3
:1077A0000100130626E205C13D4697A50100938519
:1077B000A5E24E8597800100E780A09621E917A6F3
:1077C0000100130666E281450A8597F0FFFFE78016
:1077D000C07AAA850A8597000000E7808085AA857F
:1077E00017960100130686610A8597F0FFFFE78070
:1077F000C078AA850A8597100000E780E071FDB186
:10780000E304F4FAB547E3F687F439A8C147E3FB8C
:1078100087FE454697A50100938545DE4E859780F6
:107820000100E780009015D5394697A501009385A2
:10783000E5D34E8597800100E780A08E01E5A28503
:107840004E852DB9394697A50100938565DC4E8597
:1078500097800100E780E08CE30D05EEC147E3FA75
:1078600087EE414697A50100938585DB4E8597807D
:107870000100E780008BE31E05EC83C709011307B5
:107880001003639CE700854717E7FF1F230AF7EA09
:1078900017A50100130505DA49BD1307000317A555
:1078A0000100130525DCE392E7E897E7FF1F238932
:1078B00007E817A50100130565D985BD8280411130
:1078C00026C2AE848D4522C406C62A8497B0FFFF27
:1078D000E780005CB717004099C803A5C70C418D2D
:1078E00023A6A70CB240224492444101828003A502
:1078F000870C418D23A4A70CF5B7834705000347E8
:107900001500A207D98FC2076177C1871307272007
:10791000639AE7008345250037050400170300003C
:10792000670023FA828017E6FF1F130626F58147BA
:10793000B2861303F00FA9483308F6000348080085
:1079400013F7F70F6307A80C630668008507E39534
:1079500017FF2947B387E6002380A70097E7FF1F9B
:10796000938787F25DA8411113D76500134717006D
:1079700006C693F63500058B954791CA054699478B
:107980006387C60009469D476383C600A14713F677
:1079900045003336C00093F68503050685C2A14530
:1079A000638BB604E145638AB6049305800263885D
:1079B000B604930580036393B600914697E5FF1FD5
:1079C0002389F51297E5FF1F2384C51297E5FF1F52
:1079D000A380D512BE8517A501001305A5DE9780EB
:1079E0000100E780C081B240854717E7FF1FA3026F
:1079F000F710410182808546D1B78946C1B78D46CF
:107A000075BF17A50100130565DE17730100670038
:107A1000037F17E7FF1F130727E7BA972380B700F5
:107A2000E147E302F5F493077002E30CF5FC828072
:107A30002A8723800500814717E5FF1F130505E40A
:107A40001308F00F2946B306F50083C606006396B7
:107A5000E60297E6FF1F938626E3B69783C70700E3
:107A600005452380F5009947636EF7029D4763FD46
:107A7000E700E147630DF700828063850601850713
:107A8000E393C7FC0145C5B7238005008280B73763
:107A9000004003C7370083C7050093F70704D98F59
:107AA0002380F50082805D7152DC56DA5ED6716A01
:107AB00097EBFF1F938B0B158D6AA6C24EDE62D427
:107AC00086C6A2C4CAC05AD866D26AD06ECEC14990
:107AD0005E8C97E4FF1F9384E4DB130A0A20938AE9
:107AE0007ADC17E9FF1F0349E914B3872B0183C729
:107AF000070093F7F70FC9EFB787004003C7670088
:107B0000058BE310077C03C76700118BE30D077E2D
:107B100083C75700918B99E36F10200317E7FF1F6E
:107B20000347671185476304F7006F10400197E72B
:107B3000FF1FA380E7FC97E7FF1F238D07E097E770
:107B4000FF1F238B07EC97E7FF1F238907F897E7B1
:107B5000FF1F238607F897E7FF1FA38D07DE97E730
:107B6000FF1FA38B07EA97E7FF1FA38907F697E795
:107B7000FF1FA38607F697E7FF1FA38D07F697E77A
:107B8000FF1FA38A070AB787004011476F0070776D
:107B90009307190093F7F70F3D476364F70617E75C
:107BA000FF1F2309F70897E7FF1F9387A707CA97C7
:107BB00083C707001307100293F7F703638EE71ECE
:107BC0006366F70405446385871CE38C07620947F5
:107BD000638EE71013070002E384E74EB7E700E087
:107BE0003707400023A0E718010001006299230035
:107BF0000900FD1923A0E71093F9F90FE39309EEAB
:107C0000E5BD97E7FF1F2387070271BF1307300207
:107C10006388E70C63E8E71613074002638CE70A02
:107C200013070003E39CE7FA97E7FF1F938787FE9C
:107C3000CA9703C70700A1471377F70FE31BF71491
:107C400083C7640097E6FF1F238CF6E897E7FF1FC2
:107C500083C7B7C491C7FD5797E6FF1F2382F6E895
:107C600097E5FF1F83C515C397E7FF1FA38AB7E6F4
:107C700097E7FF1F83C707C213FB0708930600049B
:107C800093F70706639FD74C9307A009638DF516FA
:107C900063EAB7129307F0056386F54A9307500924
:107CA0006384F52A014497E7FF1F83C777E31547ED
:107CB000E392E736B7E700E03707400023A0E71874
:107CC00001000100B786004023808602130680FC75
:107CD0006F00500EFD5717E7FF1F2302F7E0FDBDB1
:107CE000FD5717E7FF1F230BF7DECDBD17A50100DA
:107CF000130545C197700100E780406897E7FF1FB3
:107D0000938747F1CA9703C40700014B97ECFF1F05
:107D1000938CCCD01374F40F17AD0100130D0DBF6D
:107D200063478B04294597700100E78020528547FF
:107D300017E7FF1FA302F7CE17E7FF1F230F87CC1C
:107D400017E7FF1F2308F7DA37E700E0B706400020
:107D50002320D71801000100378600408347A60280
:107D600093F7370F2305F6022320D71085BDB3877D
:107D70006C0183C507006A85050B97700100E780D9
:107D8000004879BF854717E7FF1F2307F7C8B9B534
:107D900017E7FF1F130707E84A970347070097E60F
:107DA000FF1FA389F6BA97E6FF1F2386E6BA17E7F7
:107DB000FF1F2301F7D41DB5854717E7FF1F230BCE
:107DC000F7B829BD9307400A6389F5349307200B60
:107DD0006384F5369307100AE396F5EC8387240055
:107DE0000144E3D207EC97E7FF1F83C7D7AA93F6B6
:107DF0003700638A061A0546638AC62209466395D8
:107E0000C61A1D4755A217E5FF1F0345C5A8C94758
:107E100097ECFF1F83CC3CA897E5FF1F83C5C5A740
:107E200017E4FF1F034454A76315F510CD47639271
:107E3000FC1093077008639CF5021307300FB71707
:107E40000E006308E4001307900DB7B70400631435
:107E5000E40817E7FF1F232BF7C8BE8517A501000D
:107E6000130545AB97700100E780603925BD930786
:107E70008008639DF500B307804013F4F70FB777D0
:107E80004600938787CDB3D78702E1B79307900861
:107E9000639AF500B307804013F4F70F9167938757
:107EA000C766D5B79307A008639BF500B30780406A
:107EB00013F4F70FB7173D0093870790E9B79307BF
:107EC000B008639AF500B307804013F4F70F916789
:107ED000938797D04DBF93F5F5078D47639BF500CA
:107EE000B307804013F4F70FB7975B00938707D869
:107EF00059BF8947639BF500B307804013F4F70F20
:107F0000B7770B009387071BBDBF8547639AF500C2
:107F1000B307804013F4F70FDD67938767E3A5B7D6
:107F2000D28785F9B307804093F7F70FB3D7FA02EA
:107F30000DB797000000E780409FA28566859700F7
:107F40000000E780809EB9BB9305610017E5FF1F25
:107F50000345659417E4FF1F0344F4939700000062
:107F6000E78040AD93057100228597000000E7800F
:107F700060AC3C0017E7FF1F2324F7C8834761006C
:107F80002304F10083477100A304F100894717E738
:107F9000FF1F2307F7B48357810017E7FF1F231B39
:107FA000F78E094409B3154793F64700B336D0005E
:107FB00093F78703850685C32146638BC706614611
:107FC000638AC706130680026388C7061306800308
:107FD0006393C700914717E6FF1F230BD6B097E6C0
:107FE000FF1FA387F6B097E7FF1F2384E7B017E7CB
:107FF000FF1F0347678A9376070497E7FF1F83C72E
:10800000B7898DEE1377770C93067008630CD7024F
:108010001377F7078D466312D70CB307F040B79577
:108020005B0093F7F70F938505D849A81947ADBFB3
:10803000854755B7894745B78D4771BF9306700887
:108040006311D7021307300FB7150E006389E702DB
:108050001307900DB7B504006383E7021307700898
:1080600045BF9306800C6311D702B307F040B77584
:10807000460013F7F70F938785CDB3D5E70297E74F
:10808000FF1F23A5B7A6D9BB9306900C631CD7008E
:10809000B307F04093F5F70F91679387C766B3D5A1
:1080A000B702F1BF9306A00C631DD700B307F040E1
:1080B000B7153D0093F7F70F93850590B3D5F502FB
:1080C0007DBF9306B00CE315D7F4B307F04093F5EA
:1080D000F70F9167938797D0D9B78946631BD7006D
:1080E000B307F040B7750B0093F7F70F9385051BA7
:1080F000F1B78546631AD700B307F040DD6593F703
:10810000F70F938565E35DBFD28535FBB305F0407E
:1081100093F5F50FB3D5BA029DB783C72400C18B81
:1081200099C7854717E7FF1F230FF79AA5BE97E763
:10813000FF1F238A079ABDB6854717E7FF1FA30ACB
:10814000F79A8DB63C0017E7FF1F232BF7AA0947C4
:10815000930700032314F10097E6FF1F2382E6989C
:108160002DBD63940756A94763E5B74217970100F1
:10817000130787628A05BA959C41BA97828717D4FC
:10818000FF1F03445471894C6306940D63E68C060B
:1081900085476303F4089307F00F17E7FF1F0347B2
:1081A000279463F6E70017E7FF1F230BF79297EC7E
:1081B000FF1F83CCEC929307000413F4FC0F63F4CD
:1081C00097011304000497E7FF1F938767A303AD8C
:1081D000070022862685EA85B38C8C40229D977005
:1081E0000100E78060F697E7FF1F238B978F97E7E3
:1081F000FF1F23A7A7A145BC8D47630CF40A99472D
:10820000E31BF4F8979701009387875F17E7FF1F39
:108210002328F79EA94751B717E7FF1F0347A7A1D8
:1082200097E7FF1F9387C78D494697950100938570
:1082300025666306870097950100938565613E85F5
:1082400097700100E78040F017E7FF1F232AA79AE5
:10825000C947A1B797E6FF1F83C6E69D054797E785
:10826000FF1F9387E7896394E6023E851306700239
:10827000979501009385455F97700100E780C0ECFA
:1082800017E7FF1F232EA7969307700239B73E8585
:1082900013063004979501009385455797700100A8
:1082A000E78080EA17E7FF1F232CA7949307300489
:1082B000EDB597D5FF1F83C5055E17950100130522
:1082C000A56697700100E78080F3054D97EDFF1FCD
:1082D00083CD6D9697D5FF1F83C5E55B179501008C
:1082E000130585646398AD0B97700100E78020F15A
:1082F00097D7FF1F83C7275AB5CBE36EF4E81794CF
:1083000001001304245D638CB7011794010013046A
:10831000E45C63869701179401001304A45D228531
:1083200097700100E780C0061375F50F93071500DD
:10833000860717D7FF1F2305F77C8D4717D7FF1F29
:10834000A300F77C97D7FF1F9387877B0147BE86E3
:108350001376F70F89076365A60297E7FF1F23A12E
:10836000D78A97D7FF1F83C7A77905BD97970100C5
:108370009387474F17E7FF1F2324F788914731BDA5
:108380003306E40003460600A380070005072380A8
:10839000C7007DBF97700100E78060E697D7FF1F99
:1083A00083C7674FE1D7E368F4DE17940100130435
:1083B000644F638CA701179401001304244F638654
:1083C0009701179401001304E44F22859770010070
:1083D000E78000FC1375F50F93071500860717D784
:1083E000FF1F230FF7708D4717D7FF1FA30AF770E2
:1083F00097D7FF1F9387C7700147BE861376F70F85
:108400008907E37CA6F43306E40003460600A38054
:10841000070005072380C700D5B797D5FF1F83C581
:108420008547179501001305E55097700100E78017
:1084300000DD97D7FF1F83C7776C93E7470017D7F7
:10844000FF1FA30DF76A83C7240017D7FF1FA305DB
:10845000F76A89B8179501001305054F9770010059
:10846000E780C0F197D7FF1F9387076983C707008D
:1084700017D7FF1F2300F74217D4FF1F034444669A
:10848000333480000DB0179501001305254D97700A
:108490000100E780A0EE97D7FF1F83C7376693E7F9
:1084A000070117D7FF1FA30BF76483C7240017D753
:1084B000FF1F2303F7646FF0EFFE1795010013050C
:1084C000254B97700100E78060EB03C704007D8BAC
:1084D00051EFB787004003C767021377C70B1367D5
:1084E00027002383E70203C7A7021377C70B13678D
:1084F00027002385E70203C7E7021377C70B13673B
:1085000027002387E70203C727031377C70B1367E7
:1085100027002389E702854717D7FF1F230CF7425F
:1085200017D7FF1F230AF74E17D7FF1F2308F75A45
:1085300017D7FF1F2305F75A97D7FF1FA38C0740B4
:1085400097D7FF1FA38A074C97D7FF1FA388075809
:1085500097D7FF1FA385075897D7FF1FA38C0758EE
:1085600097D7FF1FA389076C6FF0CFF3894763127A
:10857000F70297D7FF1F83C727329146638CD7082E
:1085800063E0F604638EE70C6369F70A05476380CE
:10859000E70EFD5717D7FF1FA304F7543707400016
:1085A000B7E700E023A0E71801000100B78600400C
:1085B0001306F0FC2381C60223A0E7106FF00FE240
:1085C000130720086382E7086362F70213071008A5
:1085D000E391E7FC378700408347670293F7C70BB7
:1085E00093E727002303F7026FF0CFEB1307300860
:1085F0006389E70213074008E39DE7F837870040E7
:108600008347270393F7C70B93E727002309F70254
:108610006FF04FE9378700408347270393F7370709
:10862000F5B7378700408347E70293F7C70B93E717
:1086300027002307F7026FF0EFE6378700408347F4
:10864000E70293F73707F5B7378700408347A7025C
:1086500093F7C70B93E727002305F7026FF08FE42A
:10866000378700408347A70293F73707F5B7378767
:1086700000408347670293F73707ADB717950100AE
:108680001305053097700100E78040CF97D7FF1F93
:1086900023820720D5B3179501001305652F977026
:1086A0000100E780A0CD97D7FF1F2395071E97D71E
:1086B000FF1F9387E74203C40700894763F38700DE
:1086C00009441374F40F6FF00FDE13070002E392F6
:1086D000E7EC631B0B0A638FF500930720026383AB
:1086E000F508179501001305252E97700100E78006
:1086F00000B145B5179501001305452A9770010093
:10870000E780C0C70144179D0100130D6D2AA14CDD
:10871000B387840083C507006A850504977001004C
:10872000E780E0ADE31694FF17850100130505739C
:1087300097700100E78080C417D4FF1F0344C4155D
:1087400001E897D7FF1F23890712014B6FF0AFD5C0
:108750008947E310F4E4854717D7FF1F230EF7106E
:108760006FF04FD417D6FF1F0346F61297D5FF1FA1
:1087700083C5651217950100130505249770010044
:10878000E780E0A76FF00FD26380F5069307100231
:10879000E399F5F497D5FF1F83C5051017950100E0
:1087A0001305852397700100E78060A597D7FF1F09
:1087B00023A8974497D7FF1F93874733944383D7C2
:1087C000470017D7FF1F0347C73217D6FF1F2323C2
:1087D000D60C1D4497D6FF1F2390F60C97D7FF1F8A
:1087E000238DE70A6FF02FCC97D5FF1F83C5C50AED
:1087F000179501001305C51F97700100E78020A0A1
:1088000097D7FF1F238A070697D7FF1F23940708D0
:108810006FF02FF92547638FE7C8994637870040E7
:108820006394D70223008702B7E700E0B706400051
:1088300023A0D71801000100130600FC2301C70282
:1088400023A0D7106FF08FB99306100A639FD7004B
:1088500023008702B7E700E0B706400023A0D7183F
:1088600001000100130680FCD1BF9306A009E3813B
:10887000D7FE9306400AE38DD7FC93062002639D42
:10888000D700B7E700E0B706400023A0D7180100E3
:10889000010023008702F9B78546E384D7FE9307DA
:1088A0000008E300FBFEB7E700E0B706400023A0A6
:1088B000D71801000100130620FC23008702BDBF6A
:1088C00017D7FF1F0347D7216302F71E63E7E702AD
:1088D00095476300F7109947630AF704B78600408D
:1088E00023800602B7E700E03707400023A0E7181F
:1088F000010001001306A0FC75B99307F005630A97
:10890000F700930750096306F70093071002E31777
:10891000F7FCB7E700E03707400023A0E7180100A5
:108920000100B7860040130620FC69B117DBFF1F6A
:10893000034B0B1B930700045A8D63F46701130D5F
:10894000000497D7FF1F9387A72B83AC07001374EE
:10895000FD0F2286E685268597600100E780C07EB0
:10896000B3078B40669417D7FF1F230BF71697D7D3
:10897000FF1F23A78728B7870040630C0B022380C3
:10898000A703B7E600E03706400023A0C6180100A1
:10899000010003C72702134707042381E70203C727
:1089A00027021377C70F2381E70223A0C6106FF0B9
:1089B000EFA22380070237E700E0B706400023203C
:1089C000D71801000100130620FC2381C7026FF0B5
:1089D000AFB9378700408347370097D6FF1F83C65C
:1089E000B61193F70708D58FA301F700B70640002B
:1089F000B7E700E023A0D718010001001306A0FC90
:108A000035BD97D7FF1F9387E720CA9783C7070015
:108A100093F7F70FC1CF97D7FF1F83C7C721D9E7B8
:108A200017D7FF1F0347D70B930700026310F70800
:108A300083AD040017DDFF1F034D0DE697DCFF1F1C
:108A400083CC9CE517DBFF1F034B2BE5E6876A878A
:108A5000DA866E8697D5FF1F83C505E2179501005C
:108A6000130585FA97600100E780607997D7FF1FAB
:108A700023AEB70797D7FF1F238CA70797D7FF1FF2
:108A8000A388970797D7FF1F2385670797D7FF1FEF
:108A9000A38387DEB7E700E03707400023A0E7188D
:108AA00001000100B78600406FF04FA2B7E700E079
:108AB0003707400023A0E71801000100B7860040F7
:108AC00015BD97D6FF1F83C606170547639CE604AE
:108AD00029472381E70209472383E7022385E70229
:108AE00097D7FF1FA388070097D7FF1FA3850714F9
:108AF000B7870040A381070017D7FF1FA30E07FE0B
:108B000005472383E700B640264496440649F259B8
:108B1000625AD25A425BB25B225C925C025DF24DB9
:108B20006161828029472381E70209472383E702A5
:108B30002385E7022387E7022389E70255B717D782
:108B4000FF1FA30AF7D26FE01FFF854717D7FF1F4C
:108B50002302F7E017D7FF1F2300F7EC17D7FF1FFB
:108B6000230EF7F617D7FF1F230BF7F66FE0BFFEB4
:108B7000854717D7FF1F230FF7DC17D7FF1F230DDC
:108B8000F7E817D7FF1F230BF7F417D7FF1F2308AA
:108B9000F7F417D7FF1FA30F07DA17D7FF1FA30D8F
:108BA00007E617D7FF1FA30B07F297D7FF1FA3886E
:108BB00007F28280411106C697000000E78080FB23
:108BC000B787004023800700130740FC2386E70097
:108BD0001307C004A386E70017D7FF1F130787CB2F
:108BE0002398E70017D7FF1F1307C7CE239AE70084
:108BF00017D7FF1F130747DA239CE70017D7FF1F7C
:108C00001307C7E5239EE70029472381E7020947A9
:108C10002383E7022385E7022387E7022389E7020C
:108C2000A3810700930600F8A380D7009306900263
:108C30002380D700FD562383D7002381E7009306C6
:108C4000000537E700E0230BD740B706400023209C
:108C5000D71003C7170013671700A380E700B240BF
:108C600097D7FF1F239A07E841018280411106C66A
:108C700097000000E78000F0B787004023800700DE
:108C8000130700FC2386E7003147A386E70017D7C8
:108C9000FF1F130727C02398E70017D7FF1F1307ED
:108CA00067C3239AE70017D7FF1F1307E7CE239C5C
:108CB000E70029472381E70209472383E702238549
:108CC000E702A3810700930600F8A380D70093066C
:108CD00090022380D700FD562383D7002381E7002D
:108CE0009306000537E700E0230BD740B7064000A6
:108CF0002320D71003C7170013671700A380E700CE
:108D0000B24097D7FF1F239907DE41018280F167A8
:108D10009387072017D7FF1F232AF7DC854717D72C
:108D2000FF1F2317F7DCA14717D7FF1F2303F7DC2B
:108D300097D7FF1FA38F07DA97D7FF1F238C07DA78
:108D400097D7FF1F238A07B297D7FF1FA38507B2C4
:108D5000814717D5FF1F130565B2FD5517D6FF1FB5
:108D6000130686B22947B306F5002380B600B30682
:108D7000F600238006008507E397E7FE97D7FF1FDD
:108D8000A38107D697D7FF1FA38F07D497D7FF1FBD
:108D9000238A07D497D7FF1F238507D497D7FF1FB0
:108DA000238407D497D7FF1FA38E07D297D7FF1F1F
:108DB000238B07D2814717D6FF1F1306A6E441472E
:108DC000B306F600238006008507E39BE7FE82805A
:108DD00017D7FF1F034727E685476316F7001703DA
:108DE00000006700E3E8170300006700E3DC4111BF
:108DF00022C406C617D7FF1F0347E7E385472E8621
:108E000013F4F50FAA856317F70417D5FF1F130591
:108E1000A5BC97600100E780203397D7FF1F238D03
:108E200007BEB787004023848702B7E600E0370615
:108E3000400023A0C6180100010003C7A702137752
:108E4000C70F2385E702B240224423A0C610014584
:108E50004101828017D5FF1F1305C5AB9760010044
:108E6000E780802E97D7FF1F238607AEB787004085
:108E700023828702B7E600E03706400023A0C61829
:108E80000100010003C767021377C70F2383E702BE
:108E90005DBF411106C697000000E78080E7B24041
:108EA0004101170300006700E3F2411106C697F085
:108EB000FFFFE78080BF97D7FF1F83C7B7A9A1CB6C
:108EC00097D5FF1F83C525A989C917D5FF1F13058E
:108ED000A5A897E0FFFFE780605097D7FF1FA38BFF
:108EE00007A697D7FF1F238707C037E700E0B7061D
:108EF00040002320D7180100010037860040834737
:108F0000660293F7370F2303F6022320D710B240EF
:108F10004101828041C9D9C597D7FF1F83C7C7BD0B
:108F2000D1C3011122CC4AC84EC656C25AC006CE81
:108F300026CA52C42E89AA890144930A0004371B09
:108F4000030063772403B3078940C207C183BE844B
:108F500063F4FA0093040004C204C180130A1BD412
:108F600097D7FF1F83C7079F9DE37D1A631C0A00E5
:108F7000F2406244D2444249B249224A924A024BE8
:108F80000561828097F0FFFFE78020B2D1BF338573
:108F900089002694A685420497000000E78060E5DA
:108FA000418045B7828097D7FF1F938727DB184200
:108FB0009C4383D645000345070083C5C70003567D
:108FC00046006396A50083D5E700638DD5020111A5
:108FD00006CE2386A7002397D700B705CF00DC4B2A
:108FE0009385757D05077D162EC2230001003AC4C6
:108FF0002316C1002317D10099C30A858297F24036
:10900000056182808280411122C417A4FF1F1304CE
:10901000243F5C4C06C691CBC84B01C9B7E704009E
:10902000BC5782975C4C23AA0700B24022444101FE
:109030008280DC4DDC4B81CFB7E70400904503A371
:109040008705914517D5FF1F034585D1028382808F
:10905000B7E7040003A30705A14517D5FF1F034584
:1090600025D002836D713C083EC6B707E500232278
:1090700091103EC8AA843C083285232611103ECAAE
:1090800023248110232021112E8997300000E780AE
:1090900020622A84979501009385859A17750100AF
:1090A0001305457697600100E7806015A285179546
:1090B00001001305A5A597600100E780401429452C
:1090C00097600100E7808018B705CB009385757D18
:1090D000680097100000E780A067A28568009730BD
:1090E0000000E780404F014781467000CA85268511
:1090F00097200000E780208B05CD2A8497950100FA
:1091000093850594177501001305C56F97600100DD
:10911000E780E00EA285179501001305E59F976093
:109120000100E780C00D294597600100E78000122B
:109130008320C110032481108324411003290110CE
:109140005161828097D7FF1F938747C118429C4384
:10915000797122D406D60348070083C807012A8400
:1091600083D64500035546006396080183D827013E
:10917000638DD8022388070105072399D700370894
:10918000CC00DC4B1308787D3ACC1307F5FF42CABC
:1091900023080100231EE100231FD10099C70808FE
:1091A00032C62EC482973246A2452285970000001F
:1091B000E78080EBB250225445618280797131465C
:1091C000977501009385C554280006D69760010065
:1091D000E78080F797A7FF1F83D78722231B010013
:1091E000231C0100231D0100231E0100231F010079
:1091F00099E3C167FD17231AF10097A7FF1F83D7D3
:10920000472091EB97D7FF1F938747B59C439C431B
:10921000DC4783D7070097A6FF1F9386661E231B94
:10922000F100D84E83D74600231CF1005C4B91CB54
:1092300097A7FF1F83C7371D81EB97000000E780CA
:10924000C0DCB25045618280FD1717A6FF1FA30C3A
:10925000F61A0356070183C706014C472800230F5F
:10926000F10097300000E780203497D7FF1F9387E5
:10927000E7AE9C430147979601009386E6858843B5
:1092800030004C0897100000E780E0715DD975B799
:1092900099C9B7E7040003A30705A14517D5FF1F28
:1092A000034505AC028382805C4EDC4BB9CFB1CD67
:1092B000411122C4177501001305C5542E849785EA
:1092C00001009385257D06C697600100E78020F3A5
:1092D000A285178501001305257E97600100E780B0
:1092E00000F2294597600100E78040F6B7E70400E7
:1092F0002244B24003A3870517D5FF1F034545A6A7
:10930000130640069145410102838280411122C427
:1093100017A4FF1F1304840C1C4C06C689C7DC432A
:1093200099C34C488297584CB7E70400BC57484B48
:1093300082975C4CB240224423AA070041018280FC
:1093400017A7FF1F1307870B834707009306F00B30
:10935000850793F7F70F63E9F60097A6FF1F238FA2
:10936000F608034507008280930700F8FDB783578E
:10937000450099E37D558280011122CC17A4FF1F7F
:10938000130404085C4C4AC84EC6DC4B52C406CEDB
:1093900026CA56C2B2892E8A2A898DC7B7E7040029
:1093A000FC5F829797D7FF1F938747999C431307CA
:1093B000301FB307F54071556375F706970000003D
:1093C000E780A0C49307D00D7D5563EC3705B7E463
:1093D000040093878900B858832AC40113950701B4
:1093E0004181029723AAAA00484C584921E7978552
:1093F000010093852568177501001305A540976046
:109400000100E780C0DF178501001305A573976091
:109410000100E780C0DE294597600100E78000E396
:109420005D55F2406244D2444249B249224A924ACE
:109430000561828013874900B705CF002319E50035
:109440009385757D310597100000E7806030484CAA
:1094500083456900310597300000E780C017484C0C
:109460004E86D285310597300000E780E0137146C3
:10947000CA8517A5FF1F1305A5F897600100E780AF
:10948000A0CCFC5C82970326C90097D7FF1F23A7B7
:10949000A78A11CABC4C854517D5FF1F0345458CCB
:1094A00082970145BDBF97000000E78060D1D5BF1E
:1094B000411106C622C426C217D4FF1F1304448AD2
:1094C00097000000E78060B4B7E40400FC4C03455B
:1094D00004008545829703450400224403A3C40584
:1094E000B2409244A14541010283411126C297D462
:1094F000FF1F9384A4869C4006C622C44AC0D5C3DD
:10950000DC43C5C35CC12300B5002A8497850100F4
:1095100093858551177501001305C52E97600100CD
:10952000E780E0CD294597600100E78020D29C408C
:1095300023A4070023A2070097A7FF1F938707EA2A
:10954000DC4FDC4B91C7295597000000E78040DCD9
:1095500097A7FF1F9387C7EADC4FDC4B89C79700AB
:109560000000E78020F537E904008327C905894515
:1095700017C5FF1F0345C57E82978327C9059145FF
:1095800017C5FF1F0345C57D82979C4003A3470174
:109590006309030022852244B240924402494101FA
:1095A0000283B24022449244024941018280011167
:1095B000328506CE22CC26CA2E8497300000E78062
:1095C000200FAA84978501009385454917750100EE
:1095D0001305452397600100E78060C203078400FC
:1095E0000356640083554400A686178501001305C1
:1095F000254F97600100E78080C0294597600100F2
:10960000E780C0C497A7FF1F83C7A7DD639D9700AE
:10961000014597000000E780A0CF81450A859700AB
:109620000000E780C0ECF2406244D24405618280D1
:109630006D7123248110232611102322911093F79A
:1096400045002E84638707143C083EC0B707E50039
:109650003EC23C083EC42317010023180100231911
:109660000100231A0100231B010097A7FF1F83D7C6
:10967000E7D699E3C167FD172316F10097A7FF1FEF
:1096800083D7E7D591EB97C7FF1F9387276D9C433F
:109690009C43DC4783D7070017A7FF1F130707D496
:1096A0002317F100544F835747002318F100DC4A79
:1096B000A1E7978501009385A53E17750100130565
:1096C000651497600100E78080B3178501001305DA
:1096D000E54D97600100E78080B229459760010061
:1096E000E780C0B6134544008320C11003248110D5
:1096F000832441105161828097A7FF1F83C777CED3
:109700002555D9C3FD1717A6FF1FA30CF6CC03D60A
:10971000060183470701CC460A85230BF1009730E9
:109720000000E78060E897C7FF1F938727639C438B
:1097300017A7FF1F130787CA97860100938646372E
:1097400088430A866C0097100000E780C025AA8431
:1097500051D9978501009385A5341775010013052C
:10976000650A97600100E78080A9A685178501003A
:109770001305854497600100E78060A8294597603C
:109780000100E780A0AC268597000000E78040B884
:1097900091BF93F725009DC7B7E70400BC4741463A
:1097A000814528088297255597000000E78040B63C
:1097B00028089305F00F97000000E78040D3134579
:1097C00024001DB793F7150081CB97000000E780B8
:1097D000209F1345140009BF93F78500014589D7E1
:1097E00017A7FF1F034737C297A7FF1F938747C1DC
:1097F0000DC3D84F584B11CF37E70400384F90476F
:10980000854517C5FF1F0345A555029713458400DD
:10981000E1BD97F0FFFFE780407FCDBF5C4D411178
:1098200006C688C317C7FF1F232AF752B7E70400ED
:1098300083A70708170500001305C5DF8297B2400C
:1098400097C7FF1F238EA750014541018280011158
:109850003335A000A307A100B7E7040083A747178B
:1098600006CE1306F1008545130550308297F2406D
:1098700005618280B7E7040003A387051306000A89
:10988000914517A5FF1F0345A5BA028382804111A8
:1098900006C622C497B7FF1F83C7179881EF97C7E3
:1098A000FF1F83C7A7D7014481EF97B7FF1F83C767
:1098B000A79699E7014597000000E78080F90544E5
:1098C000228597000000E780C0F817850100130586
:1098D000653509E4178501001305C5352244B240FA
:1098E00041011763010067008391797122D4A30FAE
:1098F000010037E404008327841726D24AD006D615
:10990000AA842E89130550309305F10132C682973F
:1099100032468347F10193150601C18185CB01458C
:109920002EC697000000E780C0F283274417B24597
:109930004A8626858297054597000000E78060F1FA
:10994000B2502254925402594561828083274417B1
:109950004A8626858297EDB741119397050122C467
:1099600006C626C2C1872E8463D40702B7E404006A
:10997000FC5417A5FF1F0345A5AB829719C1BC5422
:1099800082972165218DB240224492444101828018
:1099900093F715008DC7B7E7040083A7471A17A6EA
:1099A000FF1F1306E6A797C5FF1F9385253C17A544
:1099B000FF1F0345E5A7829713451400E9B793F706
:1099C000250085CF97C7FF1F83C7C73B85E7B7E74C
:1099D000040003A8871A1307401F97A7FF1F83C718
:1099E00027A5814613064006994517C5FF1F035555
:1099F000E53802981345240079B793F745000145EF
:109A0000D9D397000000E780C0E813454400A5BF04
:109A100097C7FF1F83D787366398A70217C7FF1F13
:109A2000231FB73417C7FF1F231CC73417C7FF1FD7
:109A30002319D7342E861785010013052526BE85E8
:109A4000175301006700A37B1785010013058526C6
:109A500017630100670083920357450097C7FF1FF4
:109A600083D7C7316319F704C167F91717C7FF1FF9
:109A70002326F73097C7FF1F2386073097C7FF1F9E
:109A800023A0073097C7FF1F2388072E97A7FF1F24
:109A900023840778B7E70400FC4F411106C68945C7
:109AA00017A5FF1F0345C5988297B24041011703D0
:109AB0000000670063DC178501001305A51F17630D
:109AC00001006700A38B7D15954763E5A71E1787E7
:109AD00001001307A7130A053A951C41011122CC76
:109AE00006CEBA972E848287178501001305051DBF
:109AF00097600100E7808088F240624405618280BF
:109B000003C725009947631AF7022E8597A7FF1F01
:109B10002384077097000000E78040F483456400C9
:109B2000178501001305851A97500100E780206D05
:109B3000178501001305451B65BF97A7FF1F238DE0
:109B4000076CFDB703C7250095476319F702C16786
:109B500017C7FF1F03578722F91703D5A50063090D
:109B6000F702B7E7040083A7C7178297178501009C
:109B70001305851897600100E7804080854717A787
:109B8000FF1F230BF76817850100130565198DB7B3
:109B900097C7FF1F2394A71E83D7E50097C6FF1F13
:109BA000239FF61C83D7050197C6FF1F239AF61C37
:109BB00083D7250197C6FF1F2395F61C97C7FF1F64
:109BC000238C071A631FE5000356E4008355A400A5
:109BD000178501001305851397500100E780206267
:109BE00071BF9307700F2316F100B7E7040083A736
:109BF000870D17A6FF1F0346A6836C00829769F5A1
:109C0000854717C7FF1F2309F7167DBF178501007A
:109C10001305C511F1BD83C5250091476393F50276
:109C2000178501001305051297500100E7800075A4
:109C300097A7FF1F2382075E97000000E780C0C33D
:109C400065BD99476396F502228597A7FF1F238577
:109C5000075C97000000E78060E08345640017859B
:109C600001001305A50697500100E780405969B52A
:109C70009547639AF50083471400DDFB17850100C3
:109C80001305850EB5B5178501001305650EE1BFF7
:109C9000178501001305450D97500100E780006E00
:109CA00097A7FF1F238A0756F95717C7FF1F2317C8
:109CB000F70C59B782803757315F9797FF1F93870B
:109CC0006778130777D598C39356C50017870100A7
:109CD000130787F9BA9683C5060093568500BD8A97
:109CE000BA9603C6060093564500BD8A3D89BA96CA
:109CF0002A9783C6060003470700238407002383AF
:109D0000D700A383E7002382B700A382C7009797F9
:109D1000FF1F938727742383B700A383C70023847F
:109D2000D700A384E7008280411106C69700000097
:109D3000E780A0F8B7E7040083A787141796FF1FF2
:109D400013064670D54501458297B2404D4697951A
:109D5000FF1F938525701305703041011703000024
:109D60006700E3B861712324811A37E40400832774
:109D700004082326111A2322911A2320211B232EA3
:109D8000311917050000130565BD82971799FF1F4C
:109D90001309096A994785442300A900231CF1008F
:109DA00097850100938545EB9307400617750100E1
:109DB000130545A5231CF1082308910097C9FF1F2F
:109DC0009389299697500100E780604383D5090065
:109DD00017850100130545E797500100E7802042F1
:109DE000294597500100E780604603D50900970098
:109DF0000000E78080EC8327441710088545130591
:109E000050308297832744171796FF1F13068664E6
:109E1000CD45130570308297832744171796FF1F8F
:109E200013064661B54513056030829783274417B2
:109E3000300889451305103182978327441730096C
:109E40008945130520318297832744159305000A1D
:109E50000D458297832744159305000A1145829783
:109E6000A30591002306910002CD23080100230CD5
:109E700001008327841630099145130570408297AD
:109E8000832784161306B100854513050040829789
:109E90008327841670008545130510408297832719
:109EA0008416300885451305204082978327841641
:109EB00010088545130550408297832704157D556A
:109EC0008297832744137D5582977D559790FFFF96
:109ED000E780A07B8327440C82979790FFFFE78061
:109EE0000057832784141796FF1F1306A655D545E0
:109EF0000145829789471306700F8145280923067B
:109F0000F1009780FFFFE78080208D47130600084F
:109F100081452808230CF1089780FFFFE780201F68
:109F20009147230CF100976701009387277F98439F
:109F300083C747003AC8230AF10097C0FFFFE780B4
:109F4000E0667000854505459790FFFFE780007B40
:109F500030099305700F09459790FFFFE780007A5D
:109F60003008930500080D459790FFFFE7800079C2
:109F70001008954511459790FFFFE7802078C1674D
:109F800017C7FF1F130787DFF9171CC3232207001A
:109F90001795FF1F130585499790FFFFE780E07431
:109FA0008327C41D17C5FF1F1305C5DB82973C48D7
:109FB00003450900854582978320C11A0324811A2D
:109FC0008324411A0329011A8329C1195D61828002
:109FD000C16717C8FF1F035868DAF9176301F8084B
:109FE0003DCDB5CD011126CAB7E4040083A7841284
:109FF00022CC2E862315B10006CE2A840147814645
:10A00000ED45428582972AC611ED1785010013059B
:10A01000E5C697500100E7806036F2406244D244C2
:10A0200005618280FC440356A100A28582972C0022
:10A0300017C5FF1F035585D49790FFFFE780A077D2
:10A0400069DD178501001305A5C497500100E7805D
:10A05000E03283A7C412ED45280082977DBF82803D
:10A060000DC585471797FF1FA30BF73C9797FF1F59
:10A070002388073C35469795FF1F9385A53B13051D
:10A08000603017030000670083869797FF1FA3883F
:10A09000073AE9BF97C7FF1F83C7C7CEA9EFC167BC
:10A0A00017C7FF1F035787CDF9176306F704411140
:10A0B000854722C417C7FF1F2306F7CC37E40400E7
:10A0C0007C4C06C689451795FF1F03456536829768
:10A0D0000323841A2244B2409797FF1F83C7473552
:10A0E00017C5FF1F035585C91307401F8146314619
:10A0F00099454101028382806D71232481102326BA
:10A10000111023229110328401CD8947630AF50290
:10A110008320C11003248110832441105161828067
:10A1200017850100130585C5AE8497500100E780AF
:10A13000E024A285268597B0FFFFE780C0BAC9BF9B
:10A14000B7E70400FC472800829717850100130534
:10A15000A5C397500100E78060228347810039C47E
:10A160001307000B6380E7021387A7051377F70F28
:10A170008D4663EDE602A285280097C0FFFFE780C9
:10A18000A0C279B78547E3F587F883459100177535
:10A1900001001305259BB335B00097A7FF1F23854A
:10A1A000B7F097500100E78080059DB70347910005
:10A1B000A207B966D98F1387E6556384E70C636DF0
:10A1C000F7042D671307B755638FE708636AF70035
:10A1D00029671307A755638FE708A2852800A1BF49
:10A1E00031671307C7556388E70635671307D755E7
:10A1F000E395E7FE8947E3FD87F097000000E780DD
:10A20000A0E99305E4FFC205C1811305A100979061
:10A21000FFFFE780E0FCEDBD3D671306F75563895E
:10A22000C706636DF6009386E665E398D7FAA285C4
:10A23000280097C0FFFFE78040FCD9BD9306F76672
:10A24000638DD7041307F777E399E7F897C0FFFF0B
:10A25000E780602775BD0146A285280097C0FFFFF3
:10A26000E78020E075B5A285280097C0FFFFE78052
:10A2700060ED79BDA285280097C0FFFFE780C0ECA4
:10A2800041BDA285280097C0FFFFE78000EE49B5D9
:10A2900097C0FFFFE78080FFA5BD97C0FFFFE78065
:10A2A0002005BDB5C16717C5FF1F035525ADF917BB
:10A2B0006307F500B7E7040003A3C7170283828092
:10A2C00017F3FFFF6700E35C1783FFFFE70283DFFD
:10A2D0002A8408452E89B28919C900C19715000042
:10A2E0009385A586610597300100E780600481446D
:10A2F0007D5A97100000E780E03963C7A4048144C9
:10A3000097100000E780003A63C8A40497C7FF1FB6
:10A31000938787A79C43DC47B307F94091872302C3
:10A32000F400638309048327C900B307F4409587C9
:10A33000A302F4001C4C89C79C4799C322858297CD
:10A340001783FFFF670043DB5C4413971400850409
:10A35000BA972390470171BF1C48139714008504D6
:10A36000BA972390070069BF832789000547B30781
:10A37000F4409587A302F40083570400638EE7023C
:10A380008DC309476384E7040D47E395E7FA978790
:10A390000100938727F21CCC97870100938787F2EF
:10A3A00011A897870100938767B81CCC9787010095
:10A3B0009387C7B85CC8BDBF97870100938707A480
:10A3C0001CCC97870100938767A4EDB7978701009E
:10A3D000938707F31CCC97870100938767F3D9BF56
:10A3E00095E51783FFFFE70283CF004618448347B4
:10A3F000940075839D8B6317F70097100000E7802A
:10A4000060B448C41783FFFF6700A3CF828017831F
:10A41000FFFFE70223CB13893500C16442094111D4
:10A42000AA890144F11413590901054A2EC697104F
:10A430000000E7802026B2456348A40001454101A1
:10A440001783FFFF670043CB83A70900131714008E
:10A45000BA9783D707006388B70063949700637443
:10A460002A010504E1B70545D9BF1783FFFFE702BD
:10A4700083C4AA892E89328BB6843A8ABE8A97A071
:10A480000000E78000FE71C9268597200000E78064
:10A49000C00C8D4763E7A7007D551783FFFF67005A
:10A4A00003C583DB440097100000E780A0242A84C2
:10A4B00097100000E780402593077400314433056E
:10A4C000850263CDA70297100000E780A0229710B5
:10A4D0000000E78020222A8497100000E780C02235
:10A4E0009307740031443305850263C3A7049710B2
:10A4F0000000E78020209307450029A8971000005E
:10A50000E7808020330585021307F0179307C017F3
:10A51000E35FA7FA2D55E3C277F963040B02D686F1
:10A520005286A6854A8597200100E78000BDB5B711
:10A5300097100000E780401D330585029307C5FF93
:10A54000D1BF832749001385C90083D52700970011
:10A550000000E78000EC61F581B769553DBF97C702
:10A56000FF1F2395A78297C7FF1F9387E78190431B
:10A5700081470C463307F500420741836393B700D8
:10A5800082805446139847008507C2962390E600C0
:10A59000D5B797B7FF1F9387277F9C4303C58700D5
:10A5A000828017B5FF1F0355657E82801783FFFFEA
:10A5B000E702E3B2C1671387D7FF630BE502636A63
:10A5C000A700F1176300F50201451783FFFF67003D
:10A5D00043B31387E7FF6302E502FD171D8D1335B3
:10A5E0001500E5B797500000E780A0297D15C5BF8D
:10A5F00097500000E78020FED5BF97500000E7800D
:10A6000040FCEDB71783FFFFE70263AD4111AA8459
:10A6100001442EC697100000E780C008B245634889
:10A62000A400014541011783FFFF670083AD9C48EB
:10A63000131514003E9583570500E385B7FE050406
:10A64000C9BF03485500814693F7F60F63E507013C
:10A6500081473E858280584593975600BA9703D725
:10A6600027006316B70003D70700E304C7FE85067B
:10A67000E1BF8346450001479377F70F63E4D700B6
:10A68000814711A81C45131657000507B29703D63A
:10A690000700E313B6FE3E8582801783FFFFE702C3
:10A6A00063A293170501C18797BAFF1F938ACA6DEA
:10A6B000635BF00883A70A00C0479C470357040068
:10A6C000198D420541816368F50001442285178395
:10A6D000FFFF670063A212052A94CDBFDC471394E5
:10A6E0004900014A3E94834744006341FA02014A0B
:10A6F000834754006349FA028509C20993D90901C5
:10A7000083A70A009847E3EBE9FCC1B71C4413197F
:10A710005A00A6853E994A8597000000E780C0EE62
:10A7200005E1050AC9B75C4413195A00A6853E998C
:10A730004A8597000000E78020ED19E1050A4DBF2A
:10A74000E30C09FA61B7AA8481495DBF1783FFFF53
:10A75000E702E3981C452A8481E79307C5001CC5DE
:10A760001C44231204001CC09307F00F63EDB700D4
:10A7700093F5F50F228597200000E780C0E5178349
:10A78000FFFF6700039893940501C167C18063F9D7
:10A79000F500A685228597200000E780E0E8C5B790
:10A7A000C18193F5F50F228597200000E780A0E294
:10A7B000A685228597200000E780E0E3C9B797B718
:10A7C000FF1F9387675C884382801C4599C797B7B2
:10A7D000FF1F23ABA75A014582807D55828097B722
:10A7E000FF1F9387675A984383474500484792075E
:10A7F0003E9582801783FFFFE702638E61710045FB
:10A800001C183EC6B70780013EC81C183ECA8357B5
:10A81000440002CE02D002CC231EF1008347840004
:10A820002A8902D22301F1023C083ED402D69700C5
:10A830000000E78000FB835705002316F1029750C4
:10A840000000E78040C72307A1025C400355640075
:10A85000F18313F717008347F10252055181F99BE9
:10A86000D98FA307F10297100100E780607839CDF6
:10A87000AA840355050097A00000E78060BF83D736
:10A8800004002AD26800231CF10083D72400231D72
:10A89000F1001C4803D647008C4397200000E78056
:10A8A000A0D08347B400CA86177601001306864EEF
:10A8B0008117A305F4006C00481097200100E78081
:10A8C000C0835D611783FFFF6700A3832155D5BF58
:10A8D0001C45B1CF03C5A700894613576500630B1C
:10A8E000D7028D46630ED70285466300D702130751
:10A8F00040063305E50203C7B700418B15CB83C77C
:10A90000B700BD8B3355F54082801375F5031307EF
:10A91000803EC5B709671375F50313070771D1BFEB
:10A92000372709001375F5031307077CD9B70145CD
:10A9300082801773FFFFE702837A03A98500630C07
:10A9400009048347B900AE8493F7070E85C3034516
:10A950009900930520030D810505B305B5028844D0
:10A96000610597300100E780C0AC35A02E859700C7
:10A970000000E78020F62A8419CD97000000E780C8
:10A98000605C8325C900B307B54063FA87002E9445
:10A99000B305A440E9F51773FFFF6700837685458B
:10A9A0007DBF1773FFFFE70283732A8403D5050079
:10A9B000011132C636C43AC22EC002CA02CC02CE3F
:10A9C00097A00000E780C0AA82452ACA22852ECC23
:10A9D00097000000E780E0E003570500231EE10038
:10A9E00097500000E78020ADA24632469247230FE1
:10A9F000A10036874C08B2862285014697000000E8
:10AA0000E780E0A605611773FFFF6700836F177388
:10AA1000FFFFE702C36C61711C183EC6B7078001D7
:10AA20003EC81C183ECA3C0800453ED4AA8402CC4D
:10AA300002CE02D002D202D697000000E78060DA90
:10AA40008357050035592316F10297500000E7801F
:10AA500080A62307A10209C48357440081EB215932
:10AA60004A855D611773FFFF6700A36903556400A2
:10AA70005205518197100100E78080572A8965D1DE
:10AA80008347B40093F7070E99C7130584019730E5
:10AA90000100E780409C83574400231EF100834758
:10AAA00084002301F1025C4003550900D98313F7A8
:10AAB000070883471102231CA10093F7F707D98FDA
:10AAC000A300F10283572900231DF1005C40F183AC
:10AAD00013F717008347F102F99BD98FA307F102FF
:10AAE00097A00000E780C0982AD235D98347940008
:10AAF0006800139757008347B400FD8BD98FA305D7
:10AB0000F4001C4803D647008C4397200000E780E0
:10AB1000A0A9A687177701001307C7277400054669
:10AB20004C10268597000000E78060942A890DD993
:10AB30008347B400A685FD8BA305F40097000000B1
:10AB4000E78060DF31BF1773FFFFE70243598324BB
:10AB500085FE2A844111268597000000E78080D772
:10AB6000834734FF93F7070E8DCB2AC626859700BF
:10AB70000000E78060C809CD834734FFB245FD8BF4
:10AB8000A309F4FE91C5228597300100E780608A11
:10AB900041011773FFFF6700C3567DD98327C4FFA8
:10ABA0002685829775F5834734FF93F7070E91C783
:10ABB000228597300100E780008A032584FE9700F4
:10ABC0000000E78000E5E9B71773FFFFE702234EB7
:10ABD0009C4141112A8903C7070089472E84935657
:10ABE00067006380F6040D466388C6049307F00788
:10ABF0006304F7022E8597200000E78060ABAA84EB
:10AC00008149C16B130C490097B7FF1F9387C71782
:10AC10009C43984763E4E90441011773FFFF670011
:10AC2000C34C03D745008547E3F8E7FE2E85972000
:10AC30000000E78040ADE1B703D74500E3FEE7FC45
:10AC40002E8597200000E780A0A6AA842285972061
:10AC50000000E78000A8C204C98C5DB7DC4703553B
:10AC6000A900139A49003E9A93170501C187635DB5
:10AC7000F00083570A006397A70263E774038327F2
:10AC8000CA00034D5A002DA0A1672167A98F1307A1
:10AC9000F7EFE374F7FE6397090097000000E78081
:10ACA000209161FD85098DB783278A00034D4A00F5
:10ACB000835DA90003576900216A138BC7003AC658
:10ACC000814A33CA4D01631E5D0197B7FF1F938709
:10ACD000270C9C43E1DBA28662868145268582970C
:10ACE000D1B7A1679387F7EF930C4BFF63F247034C
:10ACF000B2455A8597F0FFFFE780A0710DC1032789
:10AD00008B00104709CE10436382C4023107D5BFC0
:10AD1000EE85668597000000E780008F71F99386C5
:10AD20001A0093FAF60F130B0B0271BF83564400FF
:10AD30005C43E3E9F6F622853AC697200000E780F7
:10AD40002081A1679387D7042A8A035D4400324794
:10AD500063E897008347D90093E707F8A306F90053
:10AD60001C4766852286E2858297C1670844FD17E5
:10AD7000337AFA00529508C02312A40125B797B779
:10AD8000FF1F938767009843814715C31447814786
:10AD900063FFD500939745004C47BE9519C903C77B
:10ADA000550081476375E600DC451606B2973E857F
:10ADB000828003C745008147E37BE6FE16069C457B
:10ADC000F5B71773FFFFE702E32FAA892E8A8144A4
:10ADD00097BAFF1F938A4AFB83A70A00984763E646
:10ADE000E4001773FFFF67002331DC47139444002E
:10ADF00001493E9413BB140083474400634BF900A0
:10AE0000014913BB140083475400634FF9008504C4
:10AE1000E1B70844931759005287DA860146A285A4
:10AE20003E9582990509C9BF484493175900528736
:10AE3000DA860546A2853E9582990509E9B717731A
:10AE4000FFFFE702C329814517F5FFFF13050548FA
:10AE500097B7FF1F239C07F297000000E780A0F63A
:10AE60001773FFFF6700E32997B7FF1F9387C7F1A9
:10AE70009C4395C31773FFFFE7026326814517F5CF
:10AE8000FFFF1305A54497000000E780C0F3177388
:10AE9000FFFF6700032782801773FFFFE70283220B
:10AEA00037E404008327841241112315E100AE89A1
:10AEB0003289368A3A8681460147ED45AA848297CF
:10AEC0002AC621C90356A100D28597400100E78018
:10AED000A0278327C413CE8526858297058905C9B7
:10AEE0008327440D2314210101462C0026858297D7
:10AEF0002A8401C9B7E7040083A7C712ED452800DB
:10AF00008297228541011773FFFF6700E31E4944C2
:10AF1000D5B76554FDB75C41FD175CC182801773DE
:10AF2000FFFFE702C31BB7E70400FC5F829795476A
:10AF30003305F50281450D811773FFFF6700631C20
:10AF40001773FFFFE702A319B7E70400FC5F8297BE
:10AF500095473305F5020D811773FFFF6700631AEC
:10AF60001773FFFFE702A317B7E7040083A7870B58
:10AF70000355050082971773FFFF67008318177347
:10AF8000FFFFE702C315035505003287AE8617861B
:10AF9000FF1F0356465297B5FF1F9385A5DF970005
:10AFA0000000E780A0EF1773FFFF6700831517739A
:10AFB000FFFFE702C312B7E7040083A7C717829712
:10AFC0001773FFFF6700E3131773FFFFE7022311F7
:10AFD000B7E7040083A7871397B5FF1F938585DB29
:10AFE000829701451773FFFF6700A3111773FFFFD7
:10AFF000E702E30EB7E7040083A7C71F8145178563
:10B00000FF1F0355454782971773FFFF6700630FC4
:10B010001773FFFFE702A30CB7E7040083A78713AA
:10B0200097B5FF1F938505D8829701451773FFFFDA
:10B030006700230D1773FFFFE702630AB7E70400F9
:10B0400083A7C71F81451785FF1F0355C5488297F2
:10B050001773FFFF6700E30A1773FFFFE702230878
:10B060002E8597800000E780C0B297800000E780BF
:10B07000C0EF1773FFFF6700C3081773FFFFE702F6
:10B08000030697800000E780C0F91773FFFF670091
:10B0900043075C49E1175CC95CC583572501A107DB
:10B0A0002319F50083570501A1072318F5008280B5
:10B0B000F1473305F50297B7FF1F9387A7D09C434D
:10B0C0003E9582808D476315F60803D74600854775
:10B0D00063F0E7081773FFFFE702630036853684E5
:10B0E0002E8997100000E780A05C29C9835744008F
:10B0F00093140501C18063E3970422859710000033
:10B10000E780005BFD14231294009307A002630004
:10B11000F5029307B0026307F50293079002631FDD
:10B12000F500228597000100E780A08801A801466C
:10B13000CA85228597A00000E78040B31773FFFF00
:10B14000670023FC228597100000E7806007FDB7A9
:10B15000828097B6FF1F938626C79C42014599CFF0
:10B160009843D44217B6FF1F2320E6C66396D70044
:10B1700097B6FF1F23ACE6C41385C7FE8280177302
:10B18000FFFFE702C3F597000000E780A04B714482
:10B1900033058502914597900000E78000EC11E5AA
:10B1A00065551773FFFF6700C3F597B7FF1F23A906
:10B1B000A7C097000000E780E0483305850291456D
:10B1C00097900000E78060E961DD97B7FF1F23AB30
:10B1D000A7BE97000000E780E04697B7FF1F239BBC
:10B1E000A7BC97000000E780E04597B7FF1F2394B6
:10B1F000A7BC97770100938727BF17B7FF1F232F9F
:10B20000F7BA97070000938707E917B7FF1F2325B1
:10B21000F7BA014579B71773FFFFE70243ECAA8538
:10B2200017B5FF1F130505B997100000E780605F91
:10B230001773FFFF6700E3EC1773FFFFE70223EAD2
:10B2400097000000E78060FD97100000E780E05E57
:10B2500097B7FF1F938747B79C4391CF1387C7FECC
:10B2600019CB83D5C7FF17B5FF1F130565B6972008
:10B270000100E780001C1773FFFF670083E8177366
:10B28000FFFFE702C3E597000000E780C0EC09CDAF
:10B29000834785002A8493F7070499EB0355E5005B
:10B2A00097000000E78080F91773FFFF670063E5F0
:10B2B0008347C5009304450117B9FF1F1309C9B09F
:10B2C00085E3832709005CC997B7FF1F23AE97AEBC
:10B2D00083274900F1FB97B7FF1F23A997AEE9B772
:10B2E000FD172306F500610597800000E780A0D9CF
:10B2F0008307840063CB07048347840093E707F840
:10B300002304F400B7E704009C5F82974205A94735
:10B3100041813375F5028347840093F707FCC98F99
:10B320002304F4008347D4003E951C402318A40056
:10B3300089CF984319CB8347C40050408145850786
:10B340003305F502420541810297832709005CC855
:10B3500097B7FF1F23AA97A68327490089E797B7C6
:10B36000FF1F23A597A68347C4009DDF83550401D3
:10B3700017B5FF1F1305C5A597200100E780600BD7
:10B3800025B71773FFFFE70283D597B7FF1F938792
:10B3900067C99C4701448583858B85E3AE84B2856C
:10B3A0003A8697100000E780204F2A8419C597102D
:10B3B0000000E7806045829408CC22851773FFFF68
:10B3C000670023D41773FFFFE702C3CF41112E8913
:10B3D00032C6AA8997000000E780C03132471306C1
:10B3E0000502CA86970500009385C5CC17B5FF1FD7
:10B3F0001305459C97000000E780E0F82A8425C9E2
:10B400009304C50097000000E780E0411946AA8533
:10B41000268597100000E78020198545268597101E
:10B420000000E7800015177501001305A5994E95DA
:10B4300083450500268597100000E780C0195C4809
:10B4400031468145A1075CC85CC483572401E117DC
:10B450002319F40083570401E1172318F4001C4C4E
:10B460003E859770FFFFE78080CAA30425012285EF
:10B4700041011773FFFF670023C81773FFFFE7023F
:10B4800003C64111AA842EC632C497100000E7807B
:10B49000003A004DB2452246834784000CC050C09C
:10B4A00093F7F70393E707042304F4002318040039
:10B4B000268597100000E780203583479400A94631
:10B4C0002317A40013D7370005073307D7029D8B36
:10B4D00085072306F400A306E40083C70401D848C7
:10B4E0008507230FF7FE17B7FF1F1307E78D584394
:10B4F000232A04009307440129E317B7FF1F2327DA
:10B50000F78C17B7FF1F2321F78C17B4FF1F130405
:10B51000248C228597200100E780E0E31C44858B82
:10B520005D8D19E58145228597200100E78060F057
:10B5300041011773FFFF6700C3BC1CC317B7FF1F90
:10B540002326F788D9B71773FFFFE70243B997059A
:10B550000000938565B7014597000000E78000B0C3
:10B5600001451773FFFF6700C3B91773FFFFE702B9
:10B5700003B797000000E78080B01773FFFF6700F4
:10B5800043B88347C500A5E31773FFFFE70223B560
:10B590002A840355E50097000000E78000C821C118
:10B5A0008347840093F7F7FB2304F4001C4091C702
:10B5B000DC4381C74C400145829797000000E7803B
:10B5C00080B917B5FF1F1305A58097200100E780FC
:10B5D00080E80355E40097000000E78020C6177359
:10B5E000FFFF670003B282801773FFFFE70223AFFC
:10B5F00097A7FF1F9387477D97050000938565C830
:10B6000017A5FF1F1305C57C23A0070023A2070071
:10B6100097200100E780C0D11773FFFF670063AE7A
:10B620001C4D91CFDC4381CF1773FFFFE70223ABA3
:10B630008345070082971773FFFF670083AC828002
:10B6400097A7FF1F9387077B9C4303C50700828052
:10B6500097A7FF1F9387077A9C4303C51700828033
:10B6600097A7FF1F938707799C4303C52700828014
:10B6700097A7FF1F938707789C4303C547008280E5
:10B6800097A7FF1F938707779C4303C537008280E6
:10B6900097A7FF1F938707769C4303C557008280B7
:10B6A00097A7FF1F938707759C4303C56700828098
:10B6B00097A7FF1F938707749C4303C57700828079
:10B6C00097A7FF1F938707739C4303C5870082805A
:10B6D00097A7FF1F938707729C4303C5970082803B
:10B6E00097A7FF1F938707719C4303C5A70082801C
:10B6F00097A7FF1F938707709C4303C5B70011E10D
:10B700001D45828097A7FF1F9387C76E9C4303C583
:10B71000C700828097A7FF1F9387C76D9C4303C50F
:10B72000D700828097A7FF1F9387C76C9C4303C5F0
:10B73000E700828097A7FF1F9387C76B9C4303D5C1
:10B740000701828097A7FF1F9387C76A9C4303C5A1
:10B750002701828097A7FF1F9387C7699C4303D562
:10B760004701828097A7FF1F9387C7689C4303D533
:10B770006701828097A7FF1F9387C7679C4303D504
:10B780008701828097A7FF1F9387C7669C4303C5E5
:10B79000A701828097A7FF1F9387C7659C4303C5B6
:10B7A000B701828097A7FF1F9387C7649C4303C597
:10B7B000C701828097A7FF1F9387C7639C4303C578
:10B7C000D701828097A7FF1F9387C7629C43885742
:10B7D000828097A7FF1F9387E7619C4303D5C70229
:10B7E000828097A7FF1F9387E7609C4303D5E702FA
:10B7F00019E11305800C828097A7FF1F9387875F4D
:10B800009C4303C50703828097A7FF1F9387875E2A
:10B810009C43C85B828097A7FF1F9387275D88435F
:10B82000828097A7FF1F9387A75C8843828019E1D6
:10B830007D558280F5DE984265DFFDD917A7FF1F91
:10B840001307477E1847AA877155058B631D072488
:10B8500003C507001547E37DA7FC03C737001305A1
:10B86000F0057D171377F70FE364E5FC03C357007A
:10B87000E30003FC83C86700E38C08FA03C7770082
:10B88000494579171377F70FE364E5FA03C7A70073
:10B8900011481305F7FF1375F50FE36BA8F803CEF6
:10B8A00097000D481305FEFF1375F50FE362A8F826
:10B8B00003C8B7006309080065181378F80F13056B
:10B8C000600DE36705F703C5C7007948791513755F
:10B8D000F50FE36FA8F403C8D7000D457D18137862
:10B8E000F80FE36705F503D80701930E40175118C9
:10B8F000420813580801E3ED0EF303C8E7007D1872
:10B900001378F80FE36605F303C827017D18137851
:10B91000F80FE36F05F103C88700C54E751813785B
:10B92000F80FE3E70EF103D86701856E938EBEE052
:10B930006D18420813580801E3EC0EEF03D84701D5
:10B940006D18420813580801E3E40EEF03D887018D
:10B950007918420813580801E36C05ED03C8A701E4
:10B960007D181378F80FE36505ED03C5B7011D4891
:10B970007D151375F50FE36DA8EA03C5D70171486E
:10B9800079151375F50FE365A8EA03D5E7011308E8
:10B99000E00F7D1542054181E36CA8E803C507026D
:10B9A000494879151375F50FE364A8E8C85301C930
:10B9B00037C834005915130858BFE36BA8E603A82D
:10B9C000870237C53400130555BF5918E36205E7F0
:10B9D00017A5FF1F232EC54003C6050117A5FF1F8E
:10B9E000232AF5400545E375C5E403D82501D04970
:10B9F00033760603E31E06E203C61501E30A06E2F8
:10BA000017A6FF1F2324B63E83C527000146638780
:10BA1000A50003C61700F1453306B60283C7070326
:10BA20009305C00272971A071307C70516031A97E2
:10BA300096084697B387B70241553E97329742071B
:10BA400041836362E8061763FFFFE70243693685B7
:10BA500097800000E780806B97000100E780004B33
:10BA60002A8497A00000E780605D2A9497F0000088
:10BA7000E78040292A9497900000E78080842A94E8
:10BA800097F0FFFFE780E06F2A9497400000E7807F
:10BA900000972A9497700000E780809F2295176393
:10BAA000FFFF6700036682801763FFFFE7022363DF
:10BAB0004111A307A10097A00000E78080C893056B
:10BAC000F100170500001305E5B597F0FFFFE780CB
:10BAD000802F014541011763FFFF670083621763F1
:10BAE000FFFFE702435D17A4FF1F1304A4530328BD
:10BAF000840079599368180097A4FF1F23A8145352
:10BB00001378180063100802BA84BE89368B328A13
:10BB10002E89AA8A97F0FFFFE780E0A77D1526957A
:10BB200019E531594A851763FFFF6700435C97F0B9
:10BB3000FFFFE78040A67D152695A167E353F5FE3C
:10BB400097B7FF1F9387078598433E8C814B01CBA6
:10BB5000014597F00000E7800047933B15004A85B8
:10BB6000DA865686D28597900000E780A0502A8911
:10BB700011CD1C44F99B17A7FF1F2329F74A8327E0
:10BB80000C00CDD3E3800BFA829769BF268597A777
:10BB9000FF1F23AB074897F0FFFFE780809C4146DB
:10BBA000CE8517A5FF1F1305655197300100E7806B
:10BBB000A05997D00000E780209C0325040B97D064
:10BBC0000000E780E09F054597D00000E780E0A6F1
:10BBD000054597000000E78060EDA9B797A7FF1F14
:10BBE000938747449C47858BEDC71763FFFFE702A8
:10BBF000034F17A5FF1F1305A54A97A7FF1F23A3F0
:10BC0000074297A7FF1F23A1074297A7FF1F23AF54
:10BC1000074097200100E780008497500000E780EC
:10BC2000C0F897100100E780804F97100100E7806F
:10BC3000805597A7FF1F9387673D9C4391C7054594
:10BC400097800000E780202397A7FF1F9387C725D1
:10BC50009C4399C741657D1597700000E78020A53A
:10BC600097F00000E780C04097D00000E780609226
:10BC700097A7FF1F938707509C431397170163569D
:10BC8000070097F00000E780E0AF97A7FF1F23A70A
:10BC9000074297A7FF1F23A5074297A7FF1F23A3CC
:10BCA000074297A7FF1F23A1074297000000E780E4
:10BCB000008C97000000E780A07597F0FFFFE780F9
:10BCC000401897F00000E78020D91763FFFF670056
:10BCD0004343828097A7FF1F9387C734884382809E
:10BCE00097A7FF1F93870734C8438280B7E7B00048
:10BCF0009387075063E1A70297A7FF1F93878732B7
:10BD0000D843FD576367E50097A7FF1F23AEA73011
:10BD100081473E858280B957EDBF1763FFFFE70279
:10BD2000033C97800000E780A07497800000E780C4
:10BD300000771763FFFF6700C33C1763FFFFE7024D
:10BD400063382A849304140201112E85B289A685D2
:10BD5000214636C63A8997300100E780803C0DE9DC
:10BD6000B24638082686CE85130594049750000005
:10BD7000E780A04021462C084A8597300100E780E3
:10BD8000403A1335150005611763FFFF6700C3369E
:10BD90000145D5BF1763FFFFE702633493054506EE
:10BDA00017A5FF1F1305450597100100E780606880
:10BDB0001763FFFF6700E3341763FFFFE7022332D7
:10BDC00041112EC697F0FFFFE780C017B24588C12A
:10BDD00041011763FFFF6700C3321763FFFFE702EC
:10BDE000632EAA842E8497800000E780406BAA8986
:10BDF0008545228597000000E780E07D83C7E40148
:10BE00001389940899E313890403CE85228597004A
:10BE10000000E780407C21469305190222859700A7
:10BE20000000E780607897A7FF1F9387A71F8C43C8
:10BE3000228597100000E780C08221469385840206
:10BE4000228597000000E78020761763FFFF6700D8
:10BE5000A32A1763FFFFE7020326397197F000005A
:10BE6000E78020B49305400661E997800000E780F1
:10BE7000405F6302051497A7FF1F83C7A7F913B795
:10BE8000170097A6FF1F2387E6F8014499CFC164E6
:10BE900017A9FF1F130909199309400EFD149700F4
:10BEA0000000E78020836342A40A97F0FFFFE78049
:10BEB00060094169B7290900096AFD7A2A8B814422
:10BEC0007D199389F97B130A0A71938A8AC79700AF
:10BED0000000E780208063D7A4041304400EB387DA
:10BEE000840217A7FF1F1307E7130324070B3E94D1
:10BEF0008357C4016382270B18403307EB4063EA82
:10BF0000E900834744008507B3874703D6976365F5
:10BF1000F70801468145094597F0FFFFE780C04AD1
:10BF2000AA8B29E597400000E780C0828547631708
:10BF3000F50689659385057117A5FF1F1305C5EBE8
:10BF400097100100E780E04E95A0B3073403032764
:10BF5000090BBA9703D7C7016308970003C75700B7
:10BF6000A38207002382E700050415BF9305C500DF
:10BF7000228597000000E78080E65E85228697652F
:10BF80000100938565E597F0FFFFE780404F5E85F0
:10BF900097100000E780608A850415BF97A7FF1FF0
:10BFA000938747089C478D83858BC1F72161176371
:10BFB000FFFF6700C31301468545094502D002D241
:10BFC00002D402D697F0FFFFE7800040AA8479DD13
:10BFD00097F00000E780209C1389C4002A848145E3
:10BFE0004A8597000000E780005F0C4041464A8583
:10BFF00097000000E780405B832944006385090CBB
:10C000004E8502D802DA02DC02DE97300100E780BA
:10C0100020382ACE141005462C0808184ECC97500C
:10C020000000E780200A1375F50F51ED8355840059
:10C0300093E525004A8597000000E780E05E114601
:10C040000C104A8597000000E7800056014697656E
:10C0500001009385E5D8268597F0FFFFE780204211
:10C06000268597000000E780407D5C40A1D3014613
:10C0700085450D4597F0FFFFE7800035AA841DD563
:10C0800048401389C40097300100E78060302AC619
:10C090004A8597000000E780404C3246636FC50038
:10C0A0004C404A8597000000E780005001468145DA
:10C0B000268597F0FFFFE780803C268597000000EB
:10C0C000E780A077E5B583558400ADB71763FFFF20
:10C0D000E702E30097A7FF1F9387C7F49C471DC1A2
:10C0E00093E7870017A5FF1F130505D117A7FF1FAB
:10C0F000232EF7F297100100E78080311763FFFFCE
:10C1000067002300DD9B17A7FF1F2321F7F297305D
:10C110000000E78020647DF117A5FF1F1305C5CD42
:10C1200097100100E7802033D1BF1763FFFFE702BC
:10C1300083F84169AA892E8AB28A368BBA8B8144E8
:10C1400017ACFF1F130C0CEE930C400E7D1997F0EB
:10C15000FFFFE780205863C4A40001443DA033845E
:10C16000940383270C0B3E948357C40163862705F1
:10C170005A87D6865286CE851305040397000000A1
:10C18000E780E0BB01C923800B0022851763FFFF16
:10C190006700E3F58347F40185C35A87D686528644
:10C1A000CE851305940897000000E78040B909C5C3
:10C1B00085472380FB00D1BF850451BF83574500CD
:10C1C0006380071E1763FFFFE702C3EF01112A8494
:10C1D00097000000E780C04D09C985476309F5064F
:10C1E00005611763FFFF670023F197E00000E78018
:10C1F000407B7DF5835744004947ED9BE392E7FE82
:10C20000C145228597000000E7804033AA8422853B
:10C2100097000000E780204F0357440002CE91476B
:10C220002A89631AF700228597000000E780A05151
:10C230003C082ACC3ECE97E00000E780C0755C55F4
:10C24000C5D374084A86A6850545829751BF035712
:10C250004400D147E3F6E7F8032A0400C169014925
:10C2600097AAFF1F938A0ADC130B400EFD1997F063
:10C27000FFFFE7802046634FA90E2285032A0400B2
:10C2800097000000E780C042A1452A8922859700D7
:10C290000000E780A02AAA84228597000000E7809A
:10C2A000804A14402A86AA8978082685CA8597007C
:10C2B0000000E780C0E7AA8405D503C7F4018947D9
:10C2C0006315F7008347C10181DF5546D285138589
:10C2D000640097300100E78020E701459780000067
:10C2E000E780001901C583D7C401A5E797A7FF1F01
:10C2F000938747D39C4793551900858913D73700F7
:10C30000058B01CF8983858B6399B70001452EC6C4
:10C3100097000000E780C0DBB2454E8597800000A3
:10C32000E780A01E0346C1012A8493751900268563
:10C3300097900000E780203935C12685978000005E
:10C34000E7802018268511C0014597800000E7800E
:10C35000404B97300000E780E03F8547E312F5E867
:10C3600083C754001307F00FE38CE7E68507A38229
:10C37000F400BDB5B304690383A70A0BBE9483D749
:10C38000C401638B37015546D2851385640097300D
:10C390000100E78000D955DD0509D1BD5DD86DB735
:10C3A00082801763FFFFE702E3D197800000E780F8
:10C3B000400B05C1C164014417A9FF1F130989C6B9
:10C3C0009309400EFD1497F0FFFFE780A030634E05
:10C3D000A40017A5FF1F130525A297100100E780F1
:10C3E00020031763FFFF670023D13305340383273E
:10C3F000090B3E958357C5016388970023120500FA
:10C4000097800000E780E00B050475BF97A7FF1F2A
:10C41000938747C19C478D83858B8DE31763FFFF0F
:10C42000E702E3CB17A5FF1F1305059D9710010039
:10C43000E78060021763FFFF6700A3CC8280176369
:10C44000FFFFE702C3C9970500009385C5A017A5A4
:10C45000FF1F1305659A97100100E78060ED1763D1
:10C46000FFFF670003CA1763FFFFE70243C7884166
:10C47000B7E70400BC5B050542054181829709C509
:10C4800085472300F50005051763FFFF670063C7B5
:10C4900083C7F5FF2E858507A38FF5FE828083C7AE
:10C4A000F5FFFD1793F7F70FA38FF5FE99EF1763CD
:10C4B000FFFFE702C3C2B7E70400BC571385F5FFCF
:10C4C00082971763FFFF6700C3C382801C41035735
:10C4D00045008D8FBA951CC12312B5003E85828020
:10C4E00093D78500A2051441DD8D8357450013873E
:10C4F000E6FF18C189072312F50013D68500411104
:10C50000238FB6FEA38FC6FE410182801841930798
:10C51000F7FF1CC18357450085072312F500A30FC1
:10C52000B7FE8280835745008D8F2312F5001C4192
:10C53000BE950CC12E858280AA8703D7470008418B
:10C540000D8FAA952392E7008CC38280184108457D
:10C550003305A740828083574500035765001D8F30
:10C560001C4108453385A7403305A74082801763E7
:10C57000FFFFE702C3B641112EC62A8497000000D0
:10C58000E780A0FDB2456373B50001A08357440066
:10C590000840BE952312B4003E9541011763FFFF8A
:10C5A000670023B61763FFFFE70263B341112E84D0
:10C5B000B28532C697000000E780A0FB3246A28514
:10C5C00097300100E78040B841011763FFFF670023
:10C5D00043B31763FFFFE70283B02E8485459700BE
:10C5E0000000E78000F9230085001763FFFF670064
:10C5F00043B11763FFFFE70283AE41112317B10078
:10C60000894597000000E780C0F68347E1002300DA
:10C61000F5008347F100A300F50041011763FFFF18
:10C62000670023AE1763FFFFE70263AB93D7850074
:10C63000A2054111DD8D2317B10089459700000047
:10C64000E78020F38347E1002300F5008347F100F2
:10C65000A300F50041011763FFFF670083AA17637A
:10C66000FFFFE702C3A71397850193D78501C16632
:10C67000938606F0D98F13D78500758FD98FA205C1
:10C680003707FF00F98D4111DD8D2EC691459700CA
:10C690000000E78000EE6C00114697300100E78053
:10C6A000A0AA41011763FFFF6700A3A51763FFFF5F
:10C6B000E702E3A21C41854503C407009700000080
:10C6C000E78080E622851763FFFF670083A3176377
:10C6D000FFFFE702C3A01C414111894503C70700C2
:10C6E00083C717002307E100A307F10097000000AC
:10C6F000E78080E30355E10041011763FFFF670016
:10C7000043A01763FFFFE702839D1C414111894548
:10C7100003C7070083C717002307E100A307F10041
:10C7200097000000E78040E08357E100410113D506
:10C730008700A2075D8D420541811763FFFF6700F7
:10C74000439C1763FFFFE70283990C4141112A8440
:10C750001146680097300100E780009F91452285CF
:10C7600097000000E78040DCB247C166938606F080
:10C770001397870113D58701598D13D78700758FBC
:10C78000598DA2073707FF00F98F5D8D41011763AF
:10C79000FFFF670003971C45BE950CC18280AE87E2
:10C7A000944391E6584101EF0CC15CC1828003C7FC
:10C7B000570013671700A382E700B687D5B70CC3ED
:10C7C000EDB7AA87084119CD1841D44398C3631324
:10C7D000D500D8C32A87034657009376160081E612
:10C7E000232007008280944381CA8C4203A847001B
:10C7F0008CC363930601CCC3799A14C3A302C70008
:10C800003687D1BF1C45DC471D8DB777DBB69387D4
:10C8100077DB09853305F502420541818280F147C6
:10C82000B385F50248452E958280834745008507EC
:10C830002302F50082801763FFFFE702438A2A8400
:10C8400009E41763FFFF6700C38B83474400F5DBF0
:10C85000FD1793F7F70F2302F400E5F71C4403D705
:10C86000270005072391E700DC4399C322858297BF
:10C870004C4889CD83475400898B99E71C44228515
:10C880009C479C439C478297232A04000040232016
:10C8900004007DB71763FFFFE70263848357250019
:10C8A00041112EC681EB0144228541011763FFFF30
:10C8B00067002385035705008147F146E305F7FE2E
:10C8C000B385D702404585072E948345440008C4AC
:10C8D000F5F5B247AA8481E7232A040009A81C457C
:10C8E0006C0022859C439C43829748C84DDD854758
:10C8F0002312F400B2472320040023180400231954
:10C90000F4005C485CC483D72400FD172391F40035
:10C9100061BF1753FFFFE702837C9797FF1F938741
:10C92000A74F8843232605002324050041059710BF
:10C930000100E78040B21753FFFF6700837C175365
:10C94000FFFFE702C3791794FF1F1304E44C1C4058
:10C95000411199CF9C472300B5002AC65CC19700BE
:10C960000000E78040FB1C40DC4399C332458297BE
:10C9700041011753FFFF6700C3780347450029E3D0
:10C98000584DAA877D551DCF1753FFFFE70223752A
:10C990001CC3DC479796FF1F23A0E648F1561305FA
:10C9A00007012390D7009705000093850502971093
:10C9B0000100E780E09701451753FFFF67006374AC
:10C9C0007D55828082801753FFFFE702437101117A
:10C9D0006146814528009750FFFFE7804073979795
:10C9E000FF1F938767439C4328009305F00FDC47A4
:10C9F0003EC697000000E780C0F405611753FFFFB3
:10CA0000670023709797FF1F938707419C43D84780
:10CA1000A1679387C702631EF70A397106DE22DC1D
:10CA200026DA80004AD84ED652D456D23285B28405
:10CA300097000000E780C0C7AA89268597000000FC
:10CA4000E78020C92318A4FC268597000000E78012
:10CA500040C82319A4FC268597000000E78060C722
:10CA600083D744000A8A231AA4FC858393F7F70F1F
:10CA7000230EF4FC8607BD0793F7073F3301F1400F
:10CA80008A8A01498347C4FD6367F902CE8513058D
:10CA900084FC232C54FD97000000E78080EA52813B
:10CAA000130104FCF2506254D2544259B259225A32
:10CAB000925A21618280268597000000E78060C13C
:10CAC00093171900D69705092390A7001379F90F3A
:10CAD00055BF82809797FF1F938707349C43D847A1
:10CAE000A1679387A702631AF70A397106DE22DC71
:10CAF00026DA80004AD84ED652D456D23285B28435
:10CB000097000000E780C0BAAA8926859700000038
:10CB1000E78020BCFD572318A4FC26852319F4FCCC
:10CB200097000000E780E0BA83D744000A8A231AFE
:10CB3000A4FC858393F7F70F230EF4FC8607BD074B
:10CB400093F7073F3301F1408A8A01498347C4FDC7
:10CB50006367F902CE85130584FC232C54FD9700EE
:10CB60000000E78000DE5281130104FCF2506254A1
:10CB7000D2544259B259225A925A21618280268552
:10CB800097000000E780E0B493171900D6970509D5
:10CB90002390A7001379F90F55BF82809797FF1F45
:10CBA000938787279C43D847A16789076310F70AB3
:10CBB000397106DE22DC26DA80004AD84ED652D4FD
:10CBC00056D23285328997000000E78060AEAA898C
:10CBD0004A8597000000E780C0AF835749000A8A62
:10CBE0002318A4FC858393F7F70F230CF4FC860726
:10CBF000BD0793F7073F3301F1408A8A8144834799
:10CC000084FD63E7F402CE85130584FC232A54FDDA
:10CC100097000000E780E0D25281130104FCF2503B
:10CC20006254D2544259B259225A925A2161828096
:10CC30004A8597000000E780C0A993971400D69713
:10CC400085042390A70093F4F40F55BF8280979733
:10CC5000FF1F9387671C9C43D847A1679387E7040E
:10CC6000631EF70A397106DE22DC26DA80004AD814
:10CC70004ED652D456D23285B28497000000E78057
:10CC800020A3AA89268597000000E78080A42318A6
:10CC9000A4FC268597000000E780A0A3231AA4FC2B
:10CCA000268597000000E780C0A283D744000A8A47
:10CCB0002319A4FC858393F7F70F230EF4FC860752
:10CCC000BD0793F7073F3301F1408A8A0149834743
:10CCD000C4FD6367F902CE85130584FC232C54FD43
:10CCE00097000000E780E0C55281130104FCF25078
:10CCF0006254D2544259B259225A925A21618280C6
:10CD0000268597000000E780C09C93171900D697EE
:10CD100005092390A7001379F90F55BF82809797D3
:10CD2000FF1F9387670F9C43D847A1679387C7046A
:10CD3000631AF70A397106DE22DC26DA80004AD847
:10CD40004ED652D456D23285B28497000000E78086
:10CD50002096AA89268597000000E7808097FD57D6
:10CD60002318A4FC2685231AF4FC97000000E78012
:10CD7000409683D744000A8A2319A4FC858393F73D
:10CD8000F70F230EF4FC8607BD0793F7073F330127
:10CD9000F1408A8A01498347C4FD6367F902CE8561
:10CDA000130584FC232C54FD97000000E78060B934
:10CDB0005281130104FCF2506254D2544259B259C8
:10CDC000225A925A21618280268597000000E780CE
:10CDD000409093171900D69705092390A70013795F
:10CDE000F90F55BF82809797FF1F9387E7029C43F7
:10CDF000D847A167DD076317F7041753FFFFE70262
:10CE0000032E79713285328497000000E780408AD2
:10CE10002AC6228597000000E780A08B2311A1027B
:10CE2000228597000000E780A088B2452300A10278
:10CE3000280897000000E780C0B045611753FFFF46
:10CE40006700232C82809797FF1F9387E7FC9C4302
:10CE5000D847A167938787046317F7041753FFFF29
:10CE6000E702E32779713285328497000000E7807A
:10CE700020842AC6228597000000E7808085231140
:10CE8000A102228597000000E7808082B24523003E
:10CE9000A102280897000000E780A0AA4561175367
:10CEA000FFFF6700032682809797FF1F9387C7F6CF
:10CEB0009C43D847A1679387A7046312F7021753CF
:10CEC000FFFFE702C3210111280081459700000000
:10CED000E78020A705611753FFFF67008322828048
:10CEE0009797FF1F938747F39C43D847A167938782
:10CEF00057026319F7021753FFFFE702431E0111A0
:10CF0000328597F0FFFFE780A07A2308A1008145D2
:10CF1000280097000000E780C0A205611753FFFFBB
:10CF20006700231E82809797FF1F9387E7EE9C433D
:10CF3000D847A1679387E702631BF7041753FFFFE6
:10CF4000E702E31901113285328497F0FFFFE78091
:10CF50004078AA84228597F0FFFFE7808077854795
:10CF600009E9228597F0FFFFE78080744205B33717
:10CF7000A00028008145231891003ECA97000000B8
:10CF8000E780209C05611753FFFF670083178280AD
:10CF90009797FF1F938747E89C43D84799476313A8
:10CFA000F7081753FFFFE702831379713285328444
:10CFB00097F0FFFFE780C06F2AC6228597F0FFFF3A
:10CFC000E78020712310A102228597F0FFFFE78000
:10CFD000206E2301A102228597F0FFFFE780406DBC
:10CFE000A301A102228597F0FFFFE780606C230276
:10CFF000A102228597F0FFFFE780806B2313A10237
:10D00000228597F0FFFFE780A06AB2452314A102B2
:10D01000280897000000E780C09245611753FFFF82
:10D020006700230E82809797FF1F9387E7DE9C435C
:10D03000D847A1679387C7036313F7081753FFFF08
:10D04000E702E30979713285328497F0FFFFE780C8
:10D0500020662AC6228597F0FFFFE78080672310AD
:10D06000A102228597F0FFFFE780A0662311A102AD
:10D07000228597F0FFFFE780A0632302A1022285AB
:10D0800097F0FFFFE780C062A302A102228597F01C
:10D09000FFFFE780E0612303A102228597F0FFFFF5
:10D0A000E7800061B245A303A102280897000000B1
:10D0B000E780208945611753FFFF67008304828062
:10D0C0001753FFFFE702A30101112A8497F0FFFF26
:10D0D000E780005EAA84228597F0FFFFE780605F0B
:10D0E000228597F0FFFFE780C05E035744008D471D
:10D0F00063F7E700228597F0FFFFE780805D2285D8
:10D1000097F0FFFFE780E05C2800A685970000000D
:10D11000E780208305611753FFFF670083FE979721
:10D12000FF1F938767CF9C43D847A167FD07631F05
:10D13000F7001753FFFFE70283FA328597000000DC
:10D14000E78040F81753FFFF6700A3FB82809797A3
:10D15000FF1F938767CC9C43D847A167E5076315FA
:10D16000F7081753FFFFE70283F77971328532849E
:10D1700097F0FFFFE780C0532AC6228597F0FFFF94
:10D18000E7802055228597F0FFFFE7808054231029
:10D19000A102228597F0FFFFE780A053520551813D
:10D1A0002311A10222852302010297F0FFFFE780ED
:10D1B0002050A302A102228597F0FFFFE780404F95
:10D1C0002303A102228597F0FFFFE780604EB2455E
:10D1D000A303A102280897F0FFFFE780807645614E
:10D1E0001753FFFF6700E3F182809797FF1F938734
:10D1F000A7C29C43D847A1679387E703631FF70043
:10D200001753FFFFE702A3ED328597000000E78088
:10D2100060EB1753FFFF6700C3EE82809797FF1FF5
:10D22000938787BF9C43D847A16793874704631EB2
:10D23000F7021753FFFFE70283EA797132853284E0
:10D2400097F0FFFFE780C0462AC6228597F0FFFFD0
:10D25000E7802048B245280897F0FFFFE780606E1E
:10D2600045611753FFFF6700C3E982809797FF1F4F
:10D27000938787BA9C43D847A16793878702631037
:10D28000F7041753FFFFE70283E579713285328493
:10D2900097F0FFFFE780C0412AC6228597F0FFFF85
:10D2A000E7800041B2452300A102280897F0FFFF64
:10D2B000E780206945611753FFFF670083E48280A0
:10D2C0001753FFFFE702A3E1011197F0FFFFE7808B
:10D2D000203EAA85280097F0FFFFE7808066056161
:10D2E0001753FFFF6700E3E19797FF1F9387C7B2CC
:10D2F0009C43D847A167D107631FF7001753FFFF6F
:10D30000E702E3DD328597000000E780A0FB1753BA
:10D31000FFFF670003DF82809797FF1F9387C7AFE8
:10D320009C43D847A167C507631FF7001753FFFF4A
:10D33000E702E3DA328597000000E780A0F8175390
:10D34000FFFF670003DC82809797FF1F9387C7ACBE
:10D350009C43D847A167B907631FF7001753FFFF26
:10D36000E702E3D7328597000000E780A0F5175366
:10D37000FFFF670003D982809797FF1F9387C7A994
:10D380009C43D847A167AD07631FF7001753FFFF02
:10D39000E702E3D4328597000000E780A0F217533C
:10D3A000FFFF670003D682809797FF1F9387C7A66A
:10D3B0009C43D84789476318F7021753FFFFE702DA
:10D3C00003D20111328532C897F0FFFFE780402E6B
:10D3D000AA85280097F0FFFFE780A0560561175344
:10D3E000FFFF670003D282809797FF1F9387C7A232
:10D3F0009C43D847A1678D076311F7041753FFFFBC
:10D40000E702E3CD01113285328497F0FFFFE78018
:10D41000202A13066100AA844C0022859730000060
:10D42000E78000232800A68597F0FFFFE780605182
:10D4300005611753FFFF6700C3CC82809797FF1FDA
:10D440009387C79D9C4381CFDC4391CB1753FFFF4C
:10D45000E702E3C882971753FFFF670083CA828001
:10D460001753FFFFE702A3C779713C08AE843ED291
:10D47000A165B7070A002A843ED448103C08DD05A0
:10D480003ED636C432C63AC297D0FFFFE780402C62
:10D4900012474810BA8597F0FFFFE780C013324665
:10D4A0004810B28597F0FFFFE780E014A2464810CD
:10D4B000B68597F0FFFFE7800012501001478146C4
:10D4C000A685228597D0FFFFE780E04D4561175381
:10D4D000FFFF670003C31753FFFFE70243C00111BB
:10D4E0007C000329C501AE843ECAA165B7070700C9
:10D4F0002A843ECC48087C00C5053ECE97D0FFFF6D
:10D50000E78000258345D900480897F0FFFFE780B2
:10D51000800C500801478146A685228597D0FFFFE1
:10D52000E780604805611753FFFF670083BD17530D
:10D53000FFFFE702C3BA83C7950093F7F707A384F9
:10D54000F50097000000E78040F91753FFFF6700E0
:10D5500043BB1753FFFFE70283B879713C08AE84E1
:10D560003ED2A165B70709002A843ED448103C0882
:10D57000938545043ED632C636C497D0FFFFE78078
:10D58000201DA2464810B68597F0FFFFE780A00453
:10D5900032464810B28597F0FFFFE780C005501073
:10D5A00001478146A685228597D0FFFFE780A03FEF
:10D5B00045611753FFFF6700C3B41753FFFFE7022E
:10D5C00003B283C7950041112A8493F7F707A38418
:10D5D000F50032852EC697F0FFFFE780800F856744
:10D5E0002AC46370F50297700000E78060E8224665
:10D5F000B24509ED11478146228597000000E7807A
:10D6000060E641011753FFFF6700A3AF0147834660
:10D61000F501DDB71753FFFFE702C3AA01113C0074
:10D620003ECAB7070A003ECC3C003ECE83C79500F9
:10D63000AA89328593F7F707A384F5002E8497F023
:10D64000FFFFE78000098567637DF504A165AA8473
:10D6500093858504480897D0FFFFE780600F2685F3
:10D6600097700000E780C0E02A8929E191454808C9
:10D6700097F0FFFFE78020F6A685480897F0FFFFA8
:10D68000E78060F7CA85480897F0FFFFE780A0F4BD
:10D69000014781465008A2854E8597D0FFFFE7805D
:10D6A000803005611753FFFF670003A581454808D7
:10D6B00097F0FFFFE78020F20349090275BF175377
:10D6C000FFFFE70223A079711C103ECAB7070F00C5
:10D6D0003ECC404D1C10AA84AE894808994532C6FC
:10D6E00036893ECE97D0FFFFE78080063246480855
:10D6F000B28597F0FFFFE78000EE630C0902A545B5
:10D70000480897F0FFFFE780C0E62546CA859720C6
:10D710000100E78060A3500801478146CE85268539
:10D7200097D0FFFFE780202845611753FFFF670070
:10D73000A39C8355C402480897F0FFFFE780A0EB45
:10D740000355E402814505C5854785456301F5021A
:10D75000C167FD179305F00F630BF5007D159770FA
:10D760000000E780608D9305150093F5F50F4808DC
:10D7700097F0FFFFE78020E683450403480897F011
:10D78000FFFFE78040E583451403480897F0FFFF5B
:10D79000E78060E483552403480897F0FFFFE780A3
:10D7A00080E583554403480897F0FFFFE780A0E435
:10D7B0009DB71753FFFFE702839283C79500814609
:10D7C000014693F7F707A384F50097000000E78070
:10D7D00040EF1753FFFF6700C3921753FFFFE702A5
:10D7E000039079713E841C103ECA2E89B7070F0042
:10D7F000A1653ECCFD051C10AA84480842C03AC26F
:10D800003ECE36C432C697D0FFFFE78060F4324682
:10D810004808B28597F0FFFFE780E0DBA2464808A2
:10D82000B68597F0FFFFE78000DD12474808BA850C
:10D8300097F0FFFFE78020DC0248630C0802914567
:10D84000480897F0FFFFE780C0D21146A2859720D5
:10D850000100E780608F500801478146CA85268510
:10D8600097D0FFFFE780201445611753FFFF670043
:10D8700043898945480897F0FFFFE78080CF8347B9
:10D8800004002300F50083471400A300F500E1B76E
:10D890001753FFFFE702038383C7950001112A8A0C
:10D8A00093F7F707A384F5003285AE8432C697F06C
:10D8B000FFFFE78000E232462A89328597F0FFFFBA
:10D8C000E78000DF85676373F902AA894A8597704C
:10D8D0000000E780E0B92A8419ED114781464A86A5
:10D8E000A685528597000000E780C0B705611753F1
:10D8F000FFFF670063809387E9FF93F7F70F054702
:10D90000E366F7FE8347F50195EB8947E380F9FE6F
:10D910008346F401528501474A86A6859700000098
:10D92000E78040B4A167D90748083ECC230A01002C
:10D9300002CE97000000E780A0B04DBF639EE700D5
:10D940008947639EF90093071020231FF500977005
:10D950000000E78000B76DBF0947E39BE7FA8D47FA
:10D96000E398F9FA228597700000E780C0DE978778
:10D97000FF1F9387A7699C4399E79787FF1F9387AA
:10D98000A7529C4399C703D5040097800000E78005
:10D99000E0CD231F040022855DBF1743FFFFE70290
:10D9A000037401113C003ECAB7070B003ECC3C009B
:10D9B0003ECE83C795002A89328593F7F707A38463
:10D9C000F500AE8497F0FFFFE780A0D09317050124
:10D9D000C187635AF006A1652A849385E502480849
:10D9E00097D0FFFFE780C0D6A285480897F0FFFFD9
:10D9F000E78060C09787FF1F9387074B9C43A9EB85
:10DA000001449375F40F480897F0FFFFE780A0BC2E
:10DA10009355844093F5F50F480897F0FFFFE78092
:10DA200080BB9355044193F5F50F480897F0FFFF2D
:10DA3000E78060BA014781465008A6854A8597D09D
:10DA4000FFFFE78040F605611743FFFF6700636B48
:10DA5000416585460546A2857D1597500000E78003
:10DA6000A0BC59DD510597000100E780C08E13046A
:10DA700040063344850271B71743FFFFE702236670
:10DA80000111B70706003EC683C7950021642A89A5
:10DA900093F7F707A384F500AE8428009305A40448
:10DAA0000AC40AC897D0FFFFE78080CA3000014748
:10DAB0008146A6854A8597D0FFFFE780C0EE97E0B4
:10DAC000FFFFE780E01113049404480822CC230AE6
:10DAD000010002CE97000000E780809605611743A1
:10DAE000FFFF670003621743FFFFE702A35DC16406
:10DAF0002A8901449789FF1F9389C952130A80021A
:10DB0000FD1497E0FFFFE780E0BD6347A4000145F7
:10DB10001743FFFF6700435EB307440303A7C90A27
:10DB2000BA9703D707006306970083D7270063845B
:10DB300027010504F9B70545E1BF1743FFFFE702D9
:10DB400063582A8A2E8999C123A0050081498144FE
:10DB5000978AFF1F938ACA2C614B97E0FFFFE780EB
:10DB6000A0BE63C7A4004E851743FFFF6700C358DC
:10DB70003384640383A70A003E948357040099E723
:10DB800063040900232089008504C1BF4146D28572
:10DB90001305440097100100E780A05875F5A2898D
:10DBA000E5B71743FFFFE702E35139717C083ED424
:10DBB000B7070A003ED67C083ED883C795002A8A5C
:10DBC000328593F7F707A384F5002E8932C697F0C4
:10DBD000FFFFE78000B085676373F5083246AA84CB
:10DBE000328597F0FFFFE780A0AC8547AA8963E8FC
:10DBF000A706A16593858504281097D0FFFFE780CD
:10DC000020B5268597700000E78080862A8429ED5C
:10DC10009145281097F0FFFFE780E09BA68528102C
:10DC200097F0FFFFE780209DCE85281097F0FFFF3B
:10DC3000E780609A014781463010CA85528597D0A7
:10DC4000FFFFE78040D6A1679387770448183EDC42
:10DC5000230A010202DE97F0FFFFE780607E216168
:10DC60001743FFFF670043498145281097F0FFFFE6
:10DC7000E7806096A685281097F0FFFFE780A097C1
:10DC80009787FF1F9387C7709C4381CB2285638949
:10DC9000090097D00000E78080238345040271B714
:10DCA00097D00000E7800022CDBF1743FFFFE702B7
:10DCB000634183C795004111AA8993F7F707A384AD
:10DCC000F5003285AE84328A97F0FFFFE78060A0CE
:10DCD0008567637FF5022A8997600000E7804079B5
:10DCE0002A84914631C58347F50105476387E702DA
:10DCF00091C70D476366F704AD461DA8930505035C
:10DD000003250A00414697100100E78080410DE994
:10DD100041011743FFFF6700233E93059508032544
:10DD20000A00414697100100E780A03F814669F54F
:10DD30004A86A6854E8597000000E780C081C9BF4E
:10DD400083250A001305940897700000E780E028F7
:10DD500019C1C146F1BF9787FF1F9387272B9C43AB
:10DD600099E79787FF1F938727149C4399C72285BC
:10DD700097800000E780608969FD8547A30FF40064
:10DD8000228597B00000E780A0832285976000007D
:10DD9000E78020734E8581464A86A68597F0FFFF6F
:10DDA000E780607BA1679387570448003EC4230245
:10DDB000010002C697F0FFFFE780806891BF17431C
:10DDC000FFFFE702432F83C795004111AA8993F70C
:10DDD000F707A384F50032852E89B28A97F0FFFFFA
:10DDE000E780208F85676374F50EAA849760000032
:10DDF000E78000682A840DED416B014A978BFF1F75
:10DE0000938B4B22130C400E7D1B19A833048A03FD
:10DE100083A70B0B3E948357C40163836705050AF0
:10DE200097E0FFFFE780008BE342AAFE95460DA036
:10DE30008357C501639697029305050303A50A005E
:10DE4000414697100100E780C02D994611E18146B7
:10DE50002686CA854E8597F0FFFFE780C06F85A8AC
:10DE600083A50A001305040397700000E780E016FD
:10DE7000C14679FD2285231E940097A00000E7800B
:10DE80002074228597600000E780A0639787FF1FBA
:10DE9000938707509C43A9C323000402228597D08F
:10DEA0000000E78080EF4E8581462686CA8597F080
:10DEB000FFFFE780406AA1679387070448003EC4DC
:10DEC0002302010002C697F0FFFFE780605741017F
:10DED0001743FFFF6700A32189472300F402E1B73E
:10DEE000397106DE22DC4AD8800052D456D25AD08C
:10DEF00026DA4ED65ECE2E8A32892A8B97D0FFFF45
:10DF0000E780407A0605710541998A8A3301A1406C
:10DF1000232224FC231404FC97D0FFFFE7808078A1
:10DF200083479A000605350593F7F7072315A4FCE8
:10DF3000A304FA004A85232624FC97E0FFFFE7802C
:10DF4000407993170501C1876340F00256811301A0
:10DF500004FCF2506254D2544259B259225A925A95
:10DF6000025BF24B21618280AA844A8597E0FFFF21
:10DF7000E7802076AA894A8597E0FFFFE7806075F1
:10DF8000A1659385C5022A89130544FC97C0FFFF4C
:10DF9000E780007C268597C0FFFFE78040708545BD
:10DFA00011C94A86CE8597C0FFFFE780C069AA8B5A
:10DFB00021E98945130544FC97E0FFFFE780A06154
:10DFC000A685130544FC97E0FFFFE780C062CE857D
:10DFD000130544FC97E0FFFFE780E061CA85130565
:10DFE00044FC97E0FFFFE78000610147814613068C
:10DFF00044FCD2855A8597D0FFFFE780C09AB9B715
:10E000008145130544FC97E0FFFFE780C05CA685CF
:10E01000130544FC97E0FFFFE780E05DCE85130524
:10E0200044FC97E0FFFFE780005DCA85130544FCD0
:10E0300097E0FFFFE780205C814497D0FFFFE780F7
:10E040006066E3D4A4FA83A70B0113971400BA9770
:10E0500083D5070099C5130544FC97E0FFFFE780CF
:10E0600080598504D9BF797106D622D44AD00018C8
:10E070004ECE52CC56CA26D25AC8AE893289AA8A06
:10E0800097D0FFFFE78000620605690541990A8A7B
:10E090003301A140232A24FC231C04FC97D0FFFF5A
:10E0A000E780406083C7990006052D0593F7F707C1
:10E0B000231DA4FCA384F9004A85232E24FC97E0A9
:10E0C000FFFFE780006193170501C187634FF000F0
:10E0D0005281130104FDB250225492540259F24964
:10E0E000624AD24A424B45618280AA844A8597E0BF
:10E0F000FFFFE780005EA1659385A5022A891305CD
:10E1000044FD97C0FFFFE780A064268597C0FFFF0E
:10E11000E780E058854509C9CA8597C0FFFFE780B9
:10E1200080552A8B29E18945130544FD97E0FFFFBF
:10E13000E780604AA685130544FD97E0FFFFE7806E
:10E14000804BCA85130544FD97E0FFFFE780A04A96
:10E1500001478146130644FDCE85568597D0FFFFC3
:10E16000E7806084B5B78145130544FD97E0FFFF64
:10E17000E7806046A685130544FD97E0FFFFE78032
:10E180008047CA85130544FD97E0FFFFE780A0465E
:10E19000814497D0FFFFE780E050E3DBA4FA8327B8
:10E1A0000B0113971400BA9783D5070099C513057F
:10E1B00044FD97E0FFFFE78000448504D9BF174383
:10E1C000FFFFE702C3F183474500404DD5EFFD5700
:10E1D0005DC48346940009476363D70A0346B400CD
:10E1E000854663EEC6088306E40063CA06085C45FC
:10E1F000F9562390D7009787FF1F83C7A7C299E3DB
:10E20000A304E4009787FF1F938707CA9C4381E715
:10E210008947A306F4009787FF1F938767179C43DE
:10E2200081E789472306F40097050000938545069A
:10E23000AA841305040197F00000E780600FFD57E2
:10E24000231AF40281471CDC01489787FF1F23A78C
:10E2500087BC9787FF1F9387A7BC232E040304C0A6
:10E26000804397D0FFFFE780204E61463306C5020A
:10E27000814522859740FFFFE78060E981473E8521
:10E280001743FFFF6700E3E7FD57D5BF1743FFFFC5
:10E29000E702E3E42A840355450297600000E78023
:10E2A000201D19E5231E04001743FFFF670063E5E7
:10E2B0008357E401F5DB930504FF174501001305BF
:10E2C000E5EB97E00000E7802014F9BF1743FFFF5C
:10E2D000E702E3E02E89A16541119385E5032A84D5
:10E2E00036C432C6BE843AC297C0FFFFE7804046BC
:10E2F00012472285BA8597E0FFFFE780C02D32469E
:10E300002285B28597E0FFFFE780E02EA2462285B6
:10E31000B68597E0FFFFE780002E63030902914571
:10E32000228597E0FFFFE780C0241146A68597105D
:10E330000100E78060E141011743FFFF670063DCF4
:10E340008945228597E0FFFFE780A02283C704006C
:10E350002300F50083C71400A300F500E9BF1743AD
:10E36000FFFFE702C3D783C79500444D054793F7E6
:10E37000F707A384F5001C42411183C707006367B8
:10E38000F7062E842A89B1C003C7D400630FF702B1
:10E390001787FF1F130747B1184305C3A386F4006F
:10E3A00097A00000E780804983C7D40099E74165C2
:10E3B0007D1597400000E780802F83D72403918B41
:10E3C00089C797E00000E78000134A85A28597F08F
:10E3D000FFFFE7808010A167C10748003EC4230209
:10E3E000010002C697F0FFFFE78080054101174357
:10E3F000FFFF670003D11743FFFFE70243CE03D7B8
:10E4000045008D47AA8441112E8432892E8563E30D
:10E41000E70297E0FFFFE780C02BAA8523000900F1
:10E42000268597C0FFFFE780002541011743FFFFC6
:10E43000670023CD97E0FFFFE780A0292AC6228549
:10E4400097E0FFFFE780E028B24585472A86230052
:10E45000F900268597C0FFFFE780E01EF9B7397104
:10E4600006DE22DC26DA80004ED652D456D24AD8B6
:10E470005AD05ECEAE89B284AA8A97D0FFFFE780D9
:10E48000602106051305250241990A8A3301A1403E
:10E49000232224FC231404FC97D0FFFFE780801F75
:10E4A00083C7990006054D0593F7F7072315A4FCCC
:10E4B000A384F9002685232624FC97E0FFFFE7804C
:10E4C000402193170501C1876340F0025281130177
:10E4D00004FCF2506254D2544259B259225A925A10
:10E4E000025BF24B21618280AA8B03AB040097C0D0
:10E4F000FFFFE780C01A51E583D7440001498544F6
:10E50000F11793B71700A301F4FC834734FCA1650E
:10E51000C9C79385E504130544FC97C0FFFFE78056
:10E520002023A685130544FC97E0FFFFE780A00A9F
:10E53000DE85130544FC97E0FFFFE780C00B8347AF
:10E5400034FC114691E30946DA85130544FC97E053
:10E55000FFFFE78060058144630A0900416B7D1B72
:10E5600097D0FFFFE780001363CCA40201478146E8
:10E57000130644FCCE85568597C0FFFFE780A04276
:10E58000B1B7A685130634FC97000000E780E0E6EB
:10E59000933415002A8986048DBF9385C504A5BFD1
:10E5A0008327C90013971400BA9783D5070063889F
:10E5B0006501130544FC97E0FFFFE780C003850475
:10E5C00045B71743FFFFE70203AF79711C103EC444
:10E5D000B7070F003EC61C103EC883C79500AA8A25
:10E5E000328593F7F707A384F500AE89328497E06C
:10E5F000FFFFE780000E93170501C187635AF006FD
:10E600002A8A228597E0FFFFE780A00C2A8952859D
:10E61000032B040097C0FFFFE780600839ED8357A4
:10E62000440081440544F11793B71700A303F10098
:10E6300083457100DA872287CA86528628009700B0
:10E640000000E780E0C8014781463000CE8556854E
:10E6500097C0FFFFE7802035A1679387D70348085D
:10E660003ECC230A810026CE97F0FFFFE78040DDF5
:10E6700045611743FFFF670083A7A285130671005A
:10E6800097000000E78060D7AA84094455D135443B
:10E69000E30055FB4A8597F0FFFFE78000450D44F6
:10E6A00041D9014497D0FFFFE780C0FE634DA4002D
:10E6B000C16B0144FD1B97D0FFFFE780A0FD634EB7
:10E6C000A4001544B5B7DC4413171400BA9783D7D8
:10E6D0000700638327030504F1B7D8449317140098
:10E6E000BA9703D70700631B77012390270126857C
:10E6F00097A00000E780C0DA01441DBF050465BF94
:10E700001743FFFFE702039C83C7950041112A8A44
:10E7100093F7F707A384F50032852E89328497E0BA
:10E72000FFFFE78000FB93170501C1876353F006E5
:10E73000AA89228597E0FFFFE780A0F92311A100B5
:10E740004E85832A040097C0FFFFE78040F539E536
:10E750008357440085440144F11793B71700A30081
:10E76000F1000348110003572100D6875285CE8659
:10E770002686CA8597F0FFFFE7806006A167F1074C
:10E7800048003EC42302910022C697F0FFFFE780B5
:10E7900020CB41011743FFFF67000396A2851306B4
:10E7A000110097000000E78040C52A84894455D9AC
:10E7B0008357210011678544BA97C2071167C18347
:10E7C0001307F7EFE36FF7F89787FF1F9387078427
:10E7D0009C4381CB85451305210097500000E780BD
:10E7E0006074835521002285814497C0FFFFE78034
:10E7F000A0E125D923100500228597A00000E7801D
:10E8000080CC85B71743FFFFE702E38A83C79500F3
:10E8100041112A8B93F7F707A384F50032852E8ADE
:10E82000328497E0FFFFE780C0EA93170501C187B4
:10E830006351F006AA8A228597E0FFFFE78060E92E
:10E840002A895685832B040097C0FFFFE78020E5C7
:10E8500031E58357440081440544F11793B717000D
:10E86000A301F10003483100DE875A854A87D68626
:10E870002286D28597F0FFFFE78060F6A167ED075B
:10E8800048003EC42302810026C697F0FFFFE780C0
:10E8900020BB41011743FFFF67006385A285130674
:10E8A000310097000000E78040B5AA8409445DD993
:10E8B0009167CA97C2071167C1831307F7EF054431
:10E8C000E362F7FACA8597C0FFFFE780E0D301440F
:10E8D00051F9814997D0FFFFE780C0DC63DBA900D5
:10E8E000984893971900BA9703D7070005EF23902C
:10E8F000270197D0FFFFE780E0DA1544E384A9F60B
:10E90000268597A00000E78000BC9777FF1F9387BC
:10E91000E76F9C430144B9D74A8597500000E780D0
:10E92000005889B785097DB71733FFFFE702837960
:10E9300079713E847C083EC82E8AB7071400A16511
:10E940003ECAE5057C08AA89080836C4428932C651
:10E95000BA8AC6843ECC97C0FFFFE78060DFCA85D5
:10E96000080897E0FFFFE78000C732460808B28535
:10E9700097E0FFFFE78020C8A246630A09049D458F
:10E98000080897E0FFFFE780C0BE1D46814597302D
:10E99000FFFFE780C07763890A089145080897E080
:10E9A000FFFFE78000BD1146A68597000100E780C4
:10E9B000A079100801478146D2854E8597C0FFFF98
:10E9C000E78060FE45611733FFFF6700E372B6859D
:10E9D000080897E0FFFFE78000C21C400808D84302
:10E9E0009355C701858912075183B205D98D97E0E8
:10E9F000FFFFE78040C01C40080883C5870097E000
:10EA0000FFFFE78040BD1C40080883C5A70097E0D2
:10EA1000FFFFE78040BC1C40080883C5970097E0D3
:10EA2000FFFFE78040BB85BF8945080897E0FFFFEF
:10EA3000E78020B483C704002300F50083C71400D7
:10EA4000A300F500BDB71733FFFFE702A36783C735
:10EA500095004111AA8993F7F707A384F500328541
:10EA6000AE84328497E0FFFFE780A0C693170501CC
:10EA7000C187635DF0042A89032A040097C0FFFF61
:10EA8000E780E0C119E9835744000548F11793B7BF
:10EA90001700A307F100814631A81306F100A285F3
:10EAA00097000000E78060951DC51C459DC783D673
:10EAB000470001480347F10093078500D2884A8642
:10EAC000A6854E8597000000E78040E64101173398
:10EAD000FFFF6700636209487DBF1D486DBF1733A4
:10EAE000FFFFE702235E65715C083EC4B7077B0148
:10EAF0003EC65C083EC883C795002A8A328593F7D4
:10EB0000F707A384F500AE8997E0FFFFE78040BADE
:10EB10008357E100E1C78945280097C0FFFFE780E0
:10EB200020C38145280097E0FFFFE780C0AA97C077
:10EB3000FFFFE78000C99787FF1F938767859C4386
:10EB40001774FF1F0344042EAA843334800099C332
:10EB5000136424009777FF1F938707359C4399C35D
:10EB6000136444009777FF1F9387474A9C4399C3D8
:10EB70001364840083D504002800014997E0FFFF57
:10EB8000E78060A783D52400280097E0FFFFE78097
:10EB900080A683D54400280097E0FFFFE780A0A56A
:10EBA00097D0FFFFE78000AB93150501C1812800D6
:10EBB00097E0FFFFE78020A4A285280097E0FFFFF1
:10EBC000E78060A39C446360F902014781463000FE
:10EBD000CE85528597C0FFFFE780E0DC596117338F
:10EBE000FFFF67006351DC441314490028003E9482
:10EBF00097E0FFFFE7806096834744000347540097
:10EC000089070607BA978607E36AF5FC835524004F
:10EC10002800814A97E0FFFFE780E09D834544009C
:10EC2000280097E0FFFFE780009B83455400280001
:10EC300097E0FFFFE780209A8347440063C9FA000A
:10EC4000814A8347540063C1FA020509A5BF1C44E9
:10EC500013975A002800BA9783D50700850A97E0D2
:10EC6000FFFFE7804099C9BF032BC40093975A0068
:10EC700028003E9B83552B00850A97E0FFFFE78025
:10EC8000809783550B00280097E0FFFFE780A09650
:10EC90004DBF1733FFFFE70283445C4993E717003A
:10ECA0005CC997A00000E78060B51733FFFF6700DD
:10ECB00043451733FFFFE70283422E84814597F0D7
:10ECC000FFFFE780C0E705C583570500FD17231048
:10ECD000F50009C4835725002310F40097000000B5
:10ECE000E78060FB01451733FFFF67008341314533
:10ECF0007DD823100400C5BF1733FFFFE702833C14
:10ED000083C7950041112A8A93F7F707A384F5007A
:10ED100032852E89328497E0FFFFE780809B93172E
:10ED20000501C1876356F006AA89C145228597E08F
:10ED3000FFFFE780A0802A8B4E85832A040097C0BE
:10ED4000FFFFE780C09531E983574400231101009C
:10ED50000544F11793B71700A300F100814403485D
:10ED6000110003572100D6875285CE862286CA8598
:10ED700097F0FFFFE780A0A6A167938717024800DE
:10ED80003EC42302810026C697E0FFFFE780406B68
:10ED900041011733FFFF6700233613061100A285D8
:10EDA00097F0FFFFE7806065AA8409E52311010061
:10EDB000094475B7930521005A8597000000E78044
:10EDC00080EF835721002A84D9DB9777FF1F938731
:10EDD000E7239C4381CB8545130521009750000014
:10EDE000E7804014835521002685314497C0FFFFFA
:10EDF000E78080812DD5231005002685979000009F
:10EE0000E780606C0144A1BF1733FFFFE702232DA9
:10EE100041112E896C00AA8402C697F0FFFFE7809B
:10EE200000D20DC10357050005072310E500970028
:10EE30000000E78040E681473E8541011733FFFF30
:10EE40006700232C3247954765DBCA8526859730B6
:10EE50000000E780800CC147E34005FE324485474F
:10EE600041462310F40083570900A685130544008A
:10EE70002311F40097000100E780002D228545BF93
:10EE80001733FFFFE702032483C795004111AA8AC5
:10EE900093F7F707A384F5003285AE89328497E0B3
:10EEA000FFFFE780008393170501C1876356F006D3
:10EEB0002A8AC145228597D0FFFFE7802068AA846F
:10EEC0005285032B040097B0FFFFE780407D31E9B6
:10EED00083574400231101008544F11793B71700AD
:10EEE000A300F10001440348110003572100DA8711
:10EEF0005685D2862686CE8597F0FFFFE780208E46
:10EF0000A1679387070248003EC42302910022C6EE
:10EF100097E0FFFFE780C05241011733FFFF670012
:10EF2000A31DA2851306110097F0FFFFE780E04CB8
:10EF30002A8409E523110100894475B726859305C4
:10EF4000210097000000E78060ECAA8449FD83550A
:10EF50002100228597B0FFFFE780006B49F501494A
:10EF600097C0FFFFE7800074635DA90018489317FE
:10EF70001900BA9703D707000DEF0357210023901C
:10EF8000E70097C0FFFFE780E071630625039777EE
:10EF9000FF1F9387A7079C4399C7035521009750EC
:10EFA0000000E780C0EF228597900000E780A05125
:10EFB0001DBF050975B795443DB705C19307F00F0F
:10EFC000630FF500C547630CF5009307F5FF054592
:10EFD0003315F500420541818280014582804165FB
:10EFE0007D158280B9E91733FFFFE702430F034520
:10EFF0000603328497000000E78060FC9305803EA2
:10F00000B305B502C205C18181CD0357E40285472E
:10F0100063F8E7001305040197E00000E780604112
:10F020008357E40241677D176385E700FD172317C7
:10F03000F4021733FFFF6700C30C82801733FFFF12
:10F04000E7026307004283C79500444D034914005B
:10F0500093F7F707A384F50083470400220911679B
:10F060003369F900A167B347F90041112A8BAE8AD1
:10F0700063ECE70E834724001307C00EB91793F71C
:10F08000F70F6373F71003473400C14763EEE70ED1
:10F09000834744001307E00793C707086371F70C21
:10F0A0008349840083477400A209B3E9F9008567A6
:10F0B00063F7F90A034A6400834754004E85220A25
:10F0C000336AFA0097500000E780803A61C12396C6
:10F0D0002403834B3400137AFA00239A34032388E1
:10F0E00074032399440393890401631C090023A634
:10F0F0000402239804024E8597E00000E780A035C3
:10F100003DA0034924004A8597000000E78020EBDA
:10F110002397A402834744004E85A388F402E38D1D
:10F120000BFCE30B09FC97E00000E780602E979052
:10F130000000E780407281460146D6855A8597E0F7
:10F14000FFFFE7800058A167938797033EC423021F
:10F150000100480002C697E0FFFFE780602E4101F2
:10F160001733FFFF6700A3F88544A2862686D6855D
:10F170005A8597E0FFFFE780C054A1679387970304
:10F180003EC423029100F1B7BD44C5B79144F1BF1D
:10F190001733FFFFE70203F301111C08404D3EC285
:10F1A000B7070F003EC41C083EC62A89AE8997C027
:10F1B000FFFFE78000D7585C1C5C6346B70E639482
:10F1C000E50063E2A70E3385A740B3B7A700B305F8
:10F1D000B7401306803E81469D8D97000100E78071
:10F1E000C0B693140501C180A1659385C50348008D
:10F1F00097B0FFFFE780C0558145480097D0FFFFDB
:10F20000E780603D83550404480097D0FFFFE78006
:10F21000803E83552404480097D0FFFFE780A03D3F
:10F22000814589CCC167FD179305F00F6388F40011
:10F23000268597500000E78020E0AA85480097D0F7
:10F24000FFFFE780403903554404814501CDC16784
:10F25000FD179305F00F6307F50097500000E78056
:10F26000A0DDAA85480097D0FFFFE780C036834520
:10F270006404480097D0FFFFE780E03583457404BD
:10F28000480097D0FFFFE7800035500001478146D6
:10F29000CE854A8597B0FFFFE780E07005611733A0
:10F2A000FFFF670063E5814481B71733FFFFE70283
:10F2B00003E383C7950093F7F707A384F50097004E
:10F2C0000000E78020ED1733FFFF670083E317336B
:10F2D000FFFFE70223DF83C795004111404D93F7FD
:10F2E000F707A384F5002A8A3285B284AE8997D0C5
:10F2F000FFFFE780003E2A8B268597D0FFFFE7803F
:10F30000403D2A89268597D0FFFFE780603A931712
:10F310000B0163CA0702E177CA97C207C18311676D
:10F3200063E3E70293070910C207C1831307B00F15
:10F33000637BF70093170901C187AA8A634AF0002B
:10F34000C54763FE570141011733FFFF6700C3DA6A
:10F3500097B0FFFFE7802025E31725FFD5B76308A7
:10F360000B0263060902814463890A02B7077F0022
:10F3700023106405231124057CC0568597000000E6
:10F38000E780E0C39304803EB304950239A0B70739
:10F390007F00232004047CC081440355240497E0AB
:10F3A0000000E780E0A2A1C497C0FFFFE78060B73C
:10F3B000269593D7F44133379500AE97BA9708DC7A
:10F3C0005CDCCE85528597000000E780A0DC99E0E8
:10F3D00023220404A1679387B70348003EC4230295
:10F3E000010002C697E0FFFFE7808005A9BF8147C3
:10F3F00001481CDC232E0403E9B71733FFFFE702A3
:10F4000003CE97C0FFFFE7802034E1473305F502C4
:10F41000914597500000E78040C4E55711C59777A4
:10F42000FF1F23AFA79E81473E851733FFFF67006D
:10F4300043CD1733FFFFE70283CA9777FF1F9387F8
:10F44000E79D80433DC0835704046390A70683571C
:10F450002404639CB7043689B28497C0FFFFE78019
:10F4600040AC5C5C63C3B7046395B7001C5C63EE9F
:10F47000A7028347640463F3F400A6872303F4041C
:10F480008347740463F39700A687A303F4048357A8
:10F49000440441677D176385E70085072312F40460
:10F4A0003C4481C7CA85268582971733FFFF6700D2
:10F4B00043C59777FF1F938767969C43014599C380
:10F4C00003C5870082801733FFFFE70243C10111A4
:10F4D000B70707003EC683C79500584D0AC493F787
:10F4E000F7070AC8A384F5002A89AE8411CB1C4211
:10F4F00083C707002304F70097900000E7800034DB
:10F50000216493055402280097B0FFFFE780402450
:10F5100097000000E78020FAAA85280097D0FFFF17
:10F52000E780600B300001478146A6854A8597B089
:10F53000FFFFE780404713044402480822CC230A17
:10F54000010002CE97E0FFFFE78080EF05611733EF
:10F55000FFFF670003BB1733FFFFE70243B801114A
:10F560007C003ECAB70707003ECC7C003ECE83C776
:10F5700095002E84AA8493F7F707A384F500A1656C
:10F5800093855502480897B0FFFFE780601C9700FD
:10F590000000E78040F2AA85480897D0FFFFE78087
:10F5A0008003500801478146A285268597B0FFFF5A
:10F5B000E780603F05611733FFFF670083B49777EB
:10F5C000FF1F9387A7859C43094599C303C59700EF
:10F5D00082809777FF1F938767849C43094599C36F
:10F5E00003C5D70082809777FF1F938727839C43AB
:10F5F000014599C303C5A70082801733FFFFE702C7
:10F6000063AC0111B70708003EC683C79500404DA3
:10F610000AC493F7F7070AC8A384F5002A89AE84C1
:10F6200029C41442854703C7060063E0E70A8347FD
:10F630009400094681496380C702B307F740A304D9
:10F64000E400B339F00083C716002305F400979057
:10F650000000E780A01E03572403058B19C76386AB
:10F66000090097D00000E78000E921649305840237
:10F67000280097B0FFFFE780A00D97000000E7800B
:10F6800040F4AA85280097D0FFFFE780C0F49700D8
:10F690000000E78080F5AA85280097D0FFFFE7806B
:10F6A00080F3014781463000A6854A8597B0FFFF69
:10F6B000E780602F13047402480822CC230A01005B
:10F6C00002CE97E0FFFFE780A0D705611733FFFF69
:10F6D000670083A21733FFFFE70263A001117C00DC
:10F6E0003ECAB70708003ECC7C003ECE83C79500DB
:10F6F0002E84AA8493F7F707A384F500A165938568
:10F700008502480897B0FFFFE7808004970000005B
:10F71000E78020EBAA85480897D0FFFFE780A0EBA1
:10F7200097000000E78060ECAA85480897D0FFFFAB
:10F73000E78060EA500801478146A285268597B098
:10F74000FFFFE780402605611733FFFF6700639BDB
:10F750009767FF1F9387876C9C43014599C303C537
:10F76000B70082801733FFFFE70263970111B707E5
:10F7700007003EC683C79500404D0AC493F7F707BC
:10F780000AC8A384F5002A89AE8405C81C4205472F
:10F7900083C707006368F7060347B400630FF700E9
:10F7A000A305F40097900000E78040098347B40068
:10F7B000B9CF97D0FFFFE78000BF21649305B40065
:10F7C000280097B0FFFFE780A0F897000000E780CF
:10F7D00060F8AA85280097D0FFFFE780C0DF0147C7
:10F7E00081463000A6854A8597B0FFFFE780A01BC1
:10F7F0002904480822CC230A010002CE97E0FFFF2B
:10F80000E78000C405611733FFFF6700838F97D03F
:10F81000FFFFE780E0BF55B71733FFFFE702238CF8
:10F8200001117C003ECAB70707003ECC7C003ECEEB
:10F8300083C795002E84AA8493F7F707A384F50065
:10F84000A165AD05480897B0FFFFE78060F097001D
:10F850000000E78020F0AA85480897D0FFFFE780E6
:10F8600080D7500801478146A285268597B0FFFFC3
:10F87000E780601305611733FFFF67008388976790
:10F88000FF1F9387A7599C43094599C303C5C70028
:10F8900082801733FFFFE702838401117C00AE846E
:10F8A0003ECAA165B70707002A843ECCD1057C007B
:10F8B00048083ECE97B0FFFFE78080E99700000040
:10F8C000E78020FCAA85480897D0FFFFE780A0D0FA
:10F8D000500801478146A685228597B0FFFFE78043
:10F8E000800C05611733FFFF6700A3811723FFFF1B
:10F8F000E702E37E83C7950093F7F707A384F5003B
:10F9000097000000E78020F91723FFFF6700637F5F
:10F910001723FFFFE702037B83C795000329C50177
:10F92000411193F7F707A384F5001C4283C9070030
:10F93000854763E637079777FF1F938767A59C4343
:10F940002E84AA8485CF97000000E78080F3894742
:10F950006306F502630409028347C9006380370325
:10F960002306390197900000E78040ED8357290373
:10F97000898B89C797D00000E780E0B72685A285EC
:10F9800097000000E78020F1A167CD0748003EC442
:10F990002302010002C697E0FFFFE78060AA410151
:10F9A0001723FFFF670043759767FF1F938707477C
:10F9B0009C431D4599C303C5E70082801723FFFFC1
:10F9C000E702E3710111B70707003EC683C7950040
:10F9D000584D0AC493F7F7070AC8A384F5002A898B
:10F9E000AE8415C71C4283C7070093968701E18642
:10F9F00063C4060685466381D7068346E7006388AD
:10FA0000F6002307F70097900000E78020E32164C9
:10FA10009305E400280097B0FFFFE78060D39700CC
:10FA20000000E780A0F8AA85280097D0FFFFE780B4
:10FA300080BA014781463000A6854A8597B0FFFF0E
:10FA4000E78060F63504480822CC230A010002CE84
:10FA500097E0FFFFE780C09E05611723FFFF670067
:10FA6000436A1723FFFFE702836701117C003ECA48
:10FA7000B70707003ECC7C003ECE83C795002E849E
:10FA8000AA8493F7F707A384F500A165B905480890
:10FA900097B0FFFFE780C0CB97000000E78000F140
:10FAA000AA85480897D0FFFFE780E0B250080147D9
:10FAB0008146A285268597B0FFFFE780C0EE0561ED
:10FAC0001723FFFF6700E3631723FFFFE702835F4E
:10FAD000AA8401441769FF1F13098934E14997C0BB
:10FAE000FFFFE78060C66344A400014519A8330501
:10FAF0003403832709003E958357250063979700B9
:10FB000011051723FFFF6700235F0504C9BF032EFC
:10FB10008500630A0E121763FF1F1303234F03238D
:10FB200003006315030029436390061203234E016B
:10FB3000631503001D43639907101723FFFFE702B6
:10FB40008357C689428A3E89BA8AB684328BAE8B85
:10FB50002A84B5E103554E0019E501431A851723A0
:10FB6000FFFF6700C358A167A98F116763FBE70018
:10FB700097000000E78080F5814597F0FFFFE78060
:10FB800080130844B70700E05841F98F18455CC15D
:10FB9000B707001FF98F1CC55C4991C7610597E045
:10FBA0000000E780408BE38A09FA228597900000E5
:10FBB000E78060C65DB7328597C00000E7804043AC
:10FBC0000D4349DD1C44116703D54700A167A98F88
:10FBD00063FBE70097000000E78040EF814597F066
:10FBE000FFFFE780400D0323840093164B01D18271
:10FBF0008347B300035663008588FD8BA305F3009C
:10FC0000FD777D8E558EFD76FD16B204F18E83272D
:10FC10004301C58E231273012313D3002304530120
:10FC200023052301A3044301BDDF228597B0FFFF15
:10FC3000E78040CAAA850844B5D1610597D0000085
:10FC4000E780207F8DB71D431A8582801723FFFF31
:10FC5000E70243470569AA84AE89328A0144FD5A06
:10FC60007D1997C0FFFFE780E0A26347A40001452C
:10FC70001723FFFF67004348D84493171400BA972F
:10FC800003D70700631F37032390570163070A0058
:10FC9000268597900000E780A0809C449DC383D771
:10FCA0006700B3F72701639E3701D2880148814777
:10FCB0000147814601468145268597000000E7807F
:10FCC00040E5050479BF1723FFFFE702A33F7971E1
:10FCD0001C103EC4B7070F003EC61C103EC883C7A9
:10FCE0009500AA8A328593F7F707A384F5002E8939
:10FCF000328497D0FFFFE780C09D93170501C1872D
:10FD0000635AF006AA89228597D0FFFFE780609C9E
:10FD10002A8A4E85032B040097B0FFFFE7802098C6
:10FD200039ED8357440081440544F11793B7170018
:10FD3000A303F10083457100DA872287D2864E86BD
:10FD4000280097E0FFFFE780A05801478146300078
:10FD5000CA85568597B0FFFFE780E0C4A167938707
:10FD6000F70348083ECC230A810026CE97D0FFFF38
:10FD7000E780006D45611723FFFF6700E337A28529
:10FD80001306710097E0FFFFE7802067AA8409440B
:10FD900055D1528597E0FFFFE78020D50D4459D912
:10FDA0000546D285268597000000E78060EA2A8410
:10FDB00051B71723FFFFE70283328355070003463D
:10FDC000270041112A842E8532C62EC497E0FFFFFA
:10FDD000E780A0D101C93246A245228597000000E4
:10FDE000E78000E741011723FFFF670083311723F6
:10FDF000FFFFE702432C83C795004111AA8A93F7BE
:10FE0000F707A384F5003285AE89328497D0FFFFCF
:10FE1000E780208C93170501C1876357F00AC1451D
:10FE20002A8A228597C0FFFFE78040712A8D2285AC
:10FE300097D0FFFFE780E0892A89228597D0FFFFCE
:10FE4000E7800087930705F893F7F70F1307E0079C
:10FE5000AA8B637BF706228597D0FFFFE78040855A
:10FE60002A8C228597D0FFFFE7808084AA8C528558
:10FE7000032B040097B0FFFFE780608239E98357C6
:10FE80004400231101008144F11793B71700A30028
:10FE9000F100054403471100835621009387840035
:10FEA0005685DA8822885286CE8597F0FFFFE78054
:10FEB000E0A7A167E90748003EC42302810026C6E7
:10FEC00097D0FFFFE780C05741011723FFFF67006E
:10FED000032213061100A28597E0FFFFE780E0519F
:10FEE000AA8409E52311010009446DB79305210097
:10FEF0006A8597F0FFFFE78060F12A8441FD835512
:10FF000021009356C9001316490185486688E28787
:10FF10005E87858A5182268597000000E78060BF52
:10FF20002A848DBF1723FFFFE702E31883C79500DC
:10FF300041112A8B93F7F707A384F5003285AE8928
:10FF4000328497C0FFFFE780C07893170501C1870F
:10FF50006352F00A2A8A228597C0FFFFE780607704
:10FF6000AA8A228597C0FFFFE780A0762A8922858A
:10FF700097C0FFFFE780C073930705F893F7F70F6B
:10FF80001307E0072A8C6377F706228597C0FFFFE7
:10FF9000E7800072AA8C228597C0FFFFE78040713E
:10FFA0002A8D5285832B040097A0FFFFE780206FE6
:10FFB00039E58357440085440144F11793B717008E
:10FFC000A301F10003473100930784005A85DE88BE
:10FFD0002688D6865286CE8597F0FFFFE78000956B
:10FFE0008D4748003EC42302910022C697D0FFFFF0
:10FFF000E780004541011723FFFF6700430FA285FB
:020000040001F9
:100000001306310097E0FFFFE780203F2A848944F0
:1000100055D99356C9001316490185486A88E68761
:100020006287858A5182D68597000000E78060AE9E
:10003000AA8449BF1723FFFFE702C3082A89814426
:100040000144617A916A176BFF1F130B2BFC97B069
:10005000FFFFE780206563C7A40022851723FFFF09
:10006000670083098327090093991400CE9703D56D
:10007000070033074501420741836364570305C105
:1000800003270B0019C785453E8597400000E78090
:1000900060E9832709000504CE97239007008504B3
:1000A0007DB797000000E78060A283270900050460
:1000B000CE972390070065D5814597F0FFFFE78035
:1000C00080BFF1BF1723FFFFE702C3FF83C795007F
:1000D00041112A8A93F7F707A384F50032852E8908
:1000E000328497C0FFFFE780C05E93170501C18788
:1000F000635AF004AA89832A040097A0FFFFE780CF
:10010000005A31E58357440085440144F11793B701
:100110001700A301F10003483100D687528501473B
:10012000CE862686CA8597D0FFFFE780406BA16701
:10013000F50748003EC42302910022C697D0FFFF76
:10014000E780003041011723FFFF6700E3FAA28533
:100150001306310097E0FFFFE780202A2A848944B4
:100160005DD99767FF1F938767EA9C4381CF044956
:1001700097B0FFFFE7800053AA85268597400000CF
:10018000E78040DA1305040197000000E780C0EA29
:10019000228597800000E78000338144ADBF17239C
:1001A000FFFFE70243F183C795004111AA8A93F745
:1001B000F707A384F5003285AE893284231101004C
:1001C00097C0FFFFE780E05093170501C187635494
:1001D000F0062A8AC145228597C0FFFFE7800036D6
:1001E000AA8B5285032B040097A0FFFFE780204BCA
:1001F00021E98357440085440144F11793B7170060
:10020000A300F1000348110003572100DA87568547
:10021000D2862686CE8597D0FFFFE780405CA16717
:100220009387270248003EC42302910022C697D03C
:10023000FFFFE780E02041011723FFFF670023EB6A
:10024000A2851306110097E0FFFFE780001B2A84B8
:1002500089444DD99767FF1F938747DB98433E89B1
:1002600001CF044997B0FFFFE780C043AA852685E8
:1002700097400000E78000CB1305040197000000C1
:10028000E78080DB97B0FFFFE780C04195443DD910
:10029000930521005E8597F0FFFFE78020B7AA84D1
:1002A00035F11C480357210022852390E7009780F1
:1002B0000000E780402183270900A9D703552100CA
:1002C00097400000E780A0BD35BF1723FFFFE7027E
:1002D00083DE83C795004111AA8A93F7F707A384A9
:1002E000F5003285AE89328497C0FFFFE780603E1B
:1002F00093170501C1876351F0062A8A228597C0AA
:10030000FFFFE780003D2A895285032B040097A058
:10031000FFFFE780C03831E583574400854401443E
:10032000F11793B71700A301F10003483100DA87F2
:1003300056854A87D2862686CE8597D0FFFFE780EE
:10034000004AA167F90748003EC42302910022C673
:1003500097D0FFFFE780C00E41011723FFFF670022
:1003600003D9A2851306310097E0FFFFE780E0087C
:100370002A8489445DD99167CA97C2071167C183EE
:100380001307F7EF8544E362F7FA9767FF1F938738
:10039000E7C79843BE8B01CF044997B0FFFFE780C2
:1003A0006030AA85268597400000E780A0B7130536
:1003B000040197000000E78020C897B0FFFFE780A6
:1003C000602E95443DD11C4822858144239027010D
:1003D00097800000E780200F83A70B00B9D74A85DC
:1003E00097400000E780A0AB89B71723FFFFE70223
:1003F00003CF2A844105B28497000000E780C0C380
:1004000011C5228597800000E780E00B81460146F8
:10041000A685228597800000E780C04E1C4C89C7C6
:10042000DC4799C3228582971723FFFF670063CDBE
:100430009767FF1F9387879E9C43014599C3138548
:10044000070182809767FF1F9387479D88438280BB
:100450001723FFFFE702A3C89317C600DD8DC2056F
:100460004111C1812A8432C697C0FFFFE780A018DE
:100470003246228511829375F60F97C0FFFFE78001
:10048000801541011723FFFF6700A3C71723FFFF54
:10049000E70243C379713C083ED2B7070C003ED453
:1004A0003C083ED683C79500AE842A8993F7F707A8
:1004B000A384F500A16593853504481097A0FFFF3C
:1004C000E7800029C165FD150144176AFF1F130A63
:1004D0006AB5930A400EAE892E8B2EC697B0FFFFE9
:1004E000E780401F4205931704014181C183B24553
:1004F00063E9A702C167FD176387F500481097C03D
:10050000FFFFE780400F501001478146A6854A85CE
:1005100097A0FFFFE780204945611723FFFF670091
:10052000A3BD3307540383270A0BBA9703D6C70129
:10053000630A3601638A3501481097000000E7809E
:1005400060F1DA85050451BFB285EDBF1723FFFFC7
:10055000E70263B679717C083EC8B70711003ECA4E
:100560007C083ECC83C79500AA89328593F7F707AC
:10057000A384F5002E8997C0FFFFE780801585676B
:100580006378F504A165AA848905080897A0FFFF90
:10059000E780001C268597400000E78060ED13345B
:1005A00015000A04A285080897C0FFFFE780A00293
:1005B000A685080897C0FFFFE780E00325CC014728
:1005C00081461008CA854E8597A0FFFFE780A03DB1
:1005D00045611723FFFF670083B1B3075403032767
:1005E000CA0ABA9703D70700631C970003D62700EF
:1005F00063806505080897000000E780A0E5DE85B8
:1006000005042EC697B0FFFFE780C00D4205931783
:1006100004014181C183B245E3E1A7FCC167FD1735
:10062000E38FF5F8080897C0FFFFE780C0FC41BFE3
:10063000B285F9B7C165FD150144176AFF1F130A9A
:100640006A9E930A80022E8BAE8B65BF1723FFFF35
:10065000E702E3A818418347170083460700A20773
:10066000D58FD207D1832390F50083472700034716
:1006700017008D45A207D98F91832310F60097C0EC
:10068000FFFFE78060EA1723FFFF670083A71723B8
:10069000FFFFE70223A3C16401441769FF1F130989
:1006A000699893098002FD1497B0FFFFE7808003EB
:1006B0006347A40001451723FFFF6700E3A3330549
:1006C00034038327C90A3E9583570500E38597FEC7
:1006D0000504D9BF1723FFFFE702C39E2A8AAE890C
:1006E000B284B68A97400000E78080D819E5914728
:1006F0003E851723FFFF670023A02A894E8597C0F8
:100700000000E780E08E2A84638E0A048D476DD155
:1007100003570500C547E31D47FD0347F90185461B
:10072000AD47E317D7FC8347450081CF4146A685F7
:100730005D0597F00000E780C09E814755D9AD4721
:1007400045BF130965012302E500CA852685971078
:100750000000E780606231C1A547E38B0AF82302FD
:10076000040079B705C183570500E39247F9414674
:10077000A685190597F00000E780A09A81472DD93A
:100780009947BDB74E8597000000E78080F02A8426
:10079000954739DD130955004DBF4146A685231005
:1007A0004401231134011305190097F00000E7807C
:1007B000A099228597800000E780A0EA81470DBFBD
:1007C0001723FFFFE702A39179717C003ECCB707A6
:1007D0000A003ECE7C003ED083C79500B2842E84B2
:1007E00093F7F707A384F5001306A1002A892C00CC
:1007F000268597000000E780A0E5A16528088D0503
:1008000097A0FFFFE780C0F490408355A1000355F7
:100810008100854697000000E78000ECAA84AA8545
:10082000280897C0FFFFE78000DB0356A10083552F
:100830008100280897000000E780C0C13008014708
:100840008146A2854A8597A0FFFFE780C0158547AE
:1008500048103ED42302910202D697D0FFFFE780D2
:1008600020BE45611723FFFF6700A3891723FFFF01
:10087000E702E38679717C003ECCB7070A003ECEE2
:100880007C003ED083C79500B2842E8493F7F7078F
:10089000A384F5001306A1002A892C002685970061
:1008A0000000E780E0DAA16528088D0597A0FFFF2A
:1008B000E78000EA90408355A100035581008146FE
:1008C00097000000E78040E1AA84AA85280897C025
:1008D000FFFFE78040D00356A10083558100280820
:1008E00097000000E78000B7300801478146A285E5
:1008F0004A8597A0FFFFE780000B48102302910272
:1009000002D402D697D0FFFFE78080B3456117136A
:10091000FFFF6700037F1713FFFFE702437C970089
:100920000000E78060DB1713FFFF6700837D9757A8
:10093000FF1F9387E74E884382801713FFFFE7026C
:10094000037A835725004111AE842A842307B1001E
:1009500017F5FFFF130525466C002316F10097A03D
:10096000FFFFE780404691C4228597800000E78022
:10097000E0D6FD572310F40013062002814513052D
:1009800054009710FFFFE780807841011713FFFFA5
:10099000670023771713FFFFE702C37279717C00AA
:1009A0003ECCB7070A003ECE7C003ED083C7950000
:1009B000AA89AE8493F7F7073285A384F50013065E
:1009C000A1002C0097000000E78080C8035581003B
:1009D000114497400000E780A0A915C50355A10068
:1009E000014497B00000E780A06011CD03570500D7
:1009F0008357810045446318F70085459700000040
:100A0000E780E0F30144216993053900280897A0A5
:100A1000FFFFE780E0D3A285280897C0FFFFE780AB
:100A200080BB0356A1008355810028089700000071
:100A3000E78040A2300801478146A6854E8597A0F1
:100A4000FFFFE78040F648104AD42302810202D615
:100A500097D0FFFFE780C09E45611713FFFF670037
:100A6000A3691713FFFFE702E3659757FF1F9387FB
:100A7000E73A2A8488432E8915C5035745038357CF
:100A8000C4016311F702232605022318050241055C
:100A900097D00000E780209C630609009780000043
:100AA000E78060DB81449759FF1F9389A957130A98
:100AB000800297B0FFFFE780E0C263C4A4049757A9
:100AC000FF1F9387673E9C4399C70355C401972036
:100AD0000000E780C0BD6307090022859780000001
:100AE000E780C0A01306400E814522859710FFFFC6
:100AF000E780E061FD57231EF4001713FFFF670036
:100B0000A35F3385440383A7C90A3E9503570500B5
:100B10008357C4016317F700CA8597000000E78078
:100B200000E2850479B71713FFFFE702A35983C7D3
:100B300095004111AA8993F7F707A384F500328540
:100B4000AE8497C0FFFFE780C0B885676378F5047F
:100B50002A8997400000E780A091014401CD83D706
:100B60000400314463882701854597000000E78031
:100B700080EF01444E85A2864A86A68597D0FFFF66
:100B8000E780609DA1679387170448003EC4230255
:100B9000810002C697D0FFFFE780808A41011713CA
:100BA000FFFF670063551713FFFFE702A351975735
:100BB000FF1F9387A726804329C4014597C00000E3
:100BC000E780002181470148C1641CDC232E040317
:100BD000232004041759FF1F1309C9440144930932
:100BE000400EFD1497B0FFFFE780C0AE634FA40036
:100BF000814517F5FFFF1305857F97A0FFFFE7806D
:100C0000801C1713FFFF6700234F3305340383272E
:100C1000090B3E958357C50163879700854597006B
:100C20000000E78040E4050475BF9357050113D722
:100C30008700A380F50093170501C183A18323805A
:100C4000E5002381F500A381A50082801713FFFF33
:100C5000E702E3482300050083C71500A300F50061
:100C600083C725002301F50083C73500A301F500E4
:100C700083C745002302F50083C75500A302F50092
:100C800083C7650093059500A30305002303F500C2
:100C900023040500328597000000E78040F9171310
:100CA000FFFF670003461713FFFFE702A34141114F
:100CB000E9540DCD85CD93F9C5FF2E842A89AA84E8
:100CC000338AA900B7EA040063189A020D888544A4
:100CD00011CCB7E704009C5F82972AC622866C007D
:100CE0003305390197E00000E78000462685410181
:100CF0001713FFFF6700434083A78A03910482977D
:100D000093170501C183A183A38EF4FE93570501B8
:100D1000238FF4FEA183238EA4FEA38FF4FE6DB770
:100D200063E6D5021713FFFFE702633BB287411169
:100D30003686BE8536C697E00000E780E040B246C2
:100D4000410136851713FFFF6700A33B81463685B7
:100D50008280838705001387F5003D05FD8793F7A3
:100D60007708834607007D158606B58FA300F5003A
:100D70006307B7007D17834717009D83DDB7828027
:100D80001713FFFFE702A335B7E7040083A707099E
:100D900032872A863A858297133515001713FFFF8D
:100DA0006700233615C181478DC11713FFFFE70286
:100DB0000333414697E00000E780003985473E85D0
:100DC0001713FFFF6700E33381473E8582801DCD07
:100DD0001713FFFFE702A330414681452A8497108D
:100DE000FFFFE780C0324146814513050403971099
:100DF000FFFFE780C0310147C1672322040438C8E0
:100E00007CC805451713FFFF6700A32F01458280AB
:100E100081473DCDB5CD1713FFFFE702432CB284C8
:100E20002E891306800581452A849710FFFFE780ED
:100E3000002ECA8524C4268597000000E780C0F6EE
:100E40004146814522859710FFFFE780402C3044C2
:100E5000A285228597000000E780C0F29304040178
:100E6000A285268597000000E780E0EEA6851305A1
:100E7000040297000000E78000EE22859700000042
:100E8000E78020F585473E851713FFFF670063273E
:100E90003E8582801713FFFFE702C3224111E95408
:100EA0000DCD85CD93F9C5FF2E842A89AA84338A76
:100EB000A900B7EA0400639844030D88814411CC6B
:100EC000B7E704009C5F82972AC622866C00330530
:100ED000390197E00000E78020272685410117139C
:100EE000FFFF6700632183A78A039104829793170A
:100EF0000501C183A183A38EF4FE93570501238FBF
:100F0000F4FEA183238EA4FEA38FF4FE6DB765CDFE
:100F10001713FFFFE702031BB28411E60545171301
:100F2000FFFF6700631D2A842E890145EDD93C48E7
:100F30007848B3E6E700E5D69386F7FFB3B7F60047
:100F40007D17032A4404BA9734C87CC863050A068F
:100F5000C14913050A03B38949412295637D3601CE
:100F6000B2862E86A68597000000E780A0DB7C4035
:100F7000BE9464C065B7CE862E86CE8597000000ED
:100F8000E78040DAC114D2944E9923220404A28748
:100F90009306040103C7070003C607038507318FC3
:100FA000A38FE7FEE398F6FE3044A28522859700E2
:100FB0000000E78020DD2699C1493306994063ECA3
:100FC0009900A9DCA686A6851305040397000000F6
:100FD000E78040D579BF8147B306F4003307F600B8
:100FE0000347070083C5060085072D8F2380E60091
:100FF000E39437FF3044A285228597000000E78004
:1010000060D8C1145DBF014582800DC11713FFFF79
:10101000E702E30C1306800581459710FFFFE78088
:10102000000F05451713FFFF6700A30D01458280E0
:10103000814749C5C1C51713FFFFE702430AFC41B9
:1010400041462E84AA846399C70413860501A287AA
:101050008146C14503C7070003C507038507298FDC
:101060003305D600034505008506298FA38FE7FECB
:10107000E392B6FE3044A285268597000000E78003
:1010800060D0228597000000E78060F885473E85A4
:101090001713FFFF6700E306138507031D8E8145C5
:1010A00022959710FFFFE78080067C40130700F829
:1010B00013060402A2972388E70251BF3E8582806F
:1010C0001713FFFFE702A3016D712E84B284AA8576
:1010D00090102800368997000000E780A0D309ED22
:1010E000D55725A050400C40280097000000E7800D
:1010F00040E27DD5FD142104F5F42C004A859700CB
:101100000000E78020F3814761DD3E8551611713C0
:10111000FFFF670003FF1713FFFFE70243FC4111C6
:101120002EC432C62C00054697000000E78080F9E7
:1011300041011713FFFF6700C3FC1713FFFFE7020E
:1011400003FA01112A842EC602C802CA02CC02CEBA
:1011500097E00000E780C023B2462A86A2850808EF
:1011600097000000E78060FB1375F50F056117130A
:10117000FFFF670003F91713FFFFE70243F67971DA
:10118000B2872A8421462308B10013051101BE85C8
:101190003AC436C697E00000E78000FBB2469305EC
:1011A0009101368597000000E78060A82285141021
:1011B00035460C0897000000E78020F62A84224775
:1011C00001E921460C103A8597E00000E780C0F75E
:1011D000228545611713FFFF6700A3F21713FFFF76
:1011E000E702E3EF7171AE84AA850A853284970025
:1011F0000000E78060BB11C90A86A685228597009A
:101200000000E78020B8814711E1C5473E854D6168
:101210001713FFFF6700E3EE1713FFFFE70223E951
:101220001D712A8AB289BE8435468547130511018E
:101230002E8CB68A3A8BC28C468D2308F10097E03B
:101240000000E78060F010100C085285231F010099
:1012500097000000E780C0F82A843DEDA1476313A2
:10126000FD089307900591E0E5473546E2851305B3
:10127000110113990A012308F1001359090197E09C
:101280000000E78060EC1357890093978A00D98F9C
:1012900090080C085285231FF10097000000E7809A
:1012A00020F42A8415E9A1E49387FA009183137945
:1012B000F9003EC6631309004149668B8144C14B66
:1012C000854DB247639F970C6A868C0033855C011D
:1012D00097E00000E78040E7228525611713FFFFB4
:1012E0006700A3E093079004C9F0A547BDBF8347FB
:1012F00001050947C14B2308F10083471105A58F5C
:10130000A308F10093872400814463E1FB040147B3
:1013100014083386E6008C08B386E400BA95DA96A2
:1013200083C6060083C505000507AD8E2300D600E1
:10133000E390E7FE4147639CE70490080C08528560
:1013400097000000E780C0E925D181A0B3069B008B
:10135000BA871008B305F60090083E9603C506004C
:101360000346060085078506298E2380C500E39283
:1013700077FF998F90080C085285BE949700000063
:10138000E78000E68947014749D12A84B1B7900830
:101390003E96034606001408BE962380C6008507C5
:1013A00059BFB24785046387971481471808B3066D
:1013B000F70098083E973386F90003470700034675
:1013C00006008507318F2380E600E39177FF9008C0
:1013D0000C08528597000000E78080E05DF53546F7
:1013E000E285130511012308B10197E00000E780B1
:1013F000A0D5139704014183939784002183D98F4B
:1014000010180C085285231FF10097000000E78098
:1014100020DD25FD814710183387F9003E960347EC
:10142000070003460600B306FB008507318F2380C3
:10143000E600E39277FF65A81808B306F70098085E
:101440003E973386F90003470700034606008507E9
:10145000318F2380E600E3E127FFCA87639E770987
:1014600090080C08528597000000E78060D711FDB6
:1014700081479800B306F700900818103E973E96F3
:1014800003470700034606008507318F2380E600E7
:10149000E39177FF3546E285130511012308B10179
:1014A00097E00000E78040CA1397040141839397B7
:1014B00084002183D98F10180C085285231FF10056
:1014C00097000000E780C0D1E31105EC81471018B8
:1014D0003387F9003E960347070003460600B3062C
:1014E000FB008507318F2380E600E3E227FFC10977
:1014F000410BC1BB814785B79408BE9683C60600E1
:1015000018083E972300D700850789BF63800632FD
:101510001713FFFFE702A3B959712A84BE89B28B62
:1015200085473546130511022E8B468C4289BA8AAF
:10153000368A2300F10297E00000E780E0C010182F
:101540000C1022852317010297000000E78040C994
:1015500063180512A147631FFC0693079005639368
:101560000900E5473546DA851305110293140A018F
:101570002300F102C18097E00000E780E0BC9317F0
:101580008A0013D78400D98F90080C102285231766
:10159000F10297000000E780A0C47DE16392090496
:1015A0009307FA00BD88918391E0C144C207C183CB
:1015B000DE8C814A3EC6414DB24763E2FA0E628636
:1015C000B3854B01881097E00000E78080B54DC9D6
:1015D0003D557DA093079004E39609F8A54759B7B8
:1015E000834701050947C14C2300F10283471105D8
:1015F000B3C7F900A300F10293872900814963E191
:10160000FC04814618103306D7008C083387D900B4
:10161000B69556970347070083C5050085062D8FAD
:101620002300E600E390D7FE41476390E706900869
:101630000C10228597000000E78080BA35D189A080
:10164000B3863A01BA871010B305F60090083E96AB
:1016500003C506000346060085078506298E2380FC
:10166000C500E39297FF3387EC4090080C10228569
:10167000BA9997000000E780A0B68947014741D199
:1016800065611713FFFF670043A690083E96034667
:1016900006001410BE962380C600850779B7B247AE
:1016A000850A93990A01939D8A0093D90901639150
:1016B000570F85473546DA85130511022300F102DD
:1016C00093D9890097E00000E78000A8B3ED3D01C1
:1016D00090000C1022852317B10397000000E780CB
:1016E00020B059FD8147A68963EA970626860C0833
:1016F0004A8597E00000E78020A581471810B306CF
:10170000F700100898083E973E96034707000346E7
:1017100006008507318F2380E600E3E197FE639F93
:10172000A90590080C10228597000000E78040ABC7
:1017300021F981479810B306F700900818183E97D2
:101740003E9603470700034606008507318F238036
:10175000E600E391A7FF4109C10CB9BD180890004C
:10176000B306F7003E963387FC00034707000346A5
:1017700006008507318F2380E600B5B798084E979D
:10178000034707001C10CE972380E700850941BF5F
:1017900085473546DA85130511022300F10293D9F6
:1017A000890097E00000E780209AB3ED3D019000AA
:1017B0000C1022852317B10397000000E78040A298
:1017C000E31005EC814718089000B306F7003E9639
:1017D0003387FC0003470700034606008507318F67
:1017E0002380E600E391A7FF41460C084A8597E075
:1017F0000000E780609581471810B306F7001008D5
:1018000098083E973E960347070003460600850763
:10181000318F2380E600E391A7FF90080C1022850A
:1018200097000000E780C09B1DD599BD7D55828043
:101830001713FFFFE702A38A01112A842E8593055F
:101840005100328902C002C202C402C6930474006D
:1018500097F0FFFFE780A03D1D46A6851305910088
:1018600097E00000E780408E10088A854A8597003F
:101870000000E780E09619ED93071400180883C66E
:1018800007000346070085070507B18EA38FD7FE23
:10189000E397F4FE05611713FFFF670083861713B4
:1018A000FFFFE70223822E848C414111AA8983879E
:1018B00015003289914463D30700A1449757FF1F55
:1018C000938707AD9C43A1C7C1CA8D472310F10080
:1018D00083C725004A852301F10083C73500A30192
:1018E000F10083C745002302F10083C75500A3021E
:1018F000F10083C7650093059100A3030100230352
:10190000F1002304010097F0FFFFE78040320C4014
:101910004A860A8597F0FFFFE7808033032804009A
:1019200083564400A6881D0881470147E516428674
:101930008A854E8597000000E780408E2A8919E548
:10194000A685228597B0FFFFE780A0C24A854101A6
:101950001703FFFF6700437A4A860A8597F0FFFF67
:10196000E780002F6DB71703FFFFE702A3752E84F2
:101970008C414111AA89838715003289914463D330
:101980000700A1449757FF1F938787A09C43A1C7D7
:10199000C1C68D472310F10083C725004A85230166
:1019A000F10083C73500A301F10083C7450023027E
:1019B000F10083C75500A302F10083C765009305BA
:1019C0009100A30301002303F1002304010097F019
:1019D000FFFFE780C0250C404A860A8597F0FFFF8D
:1019E000E780002783564400032804008A85858EFB
:1019F000C2061D08C1822312D400A6888147014770
:101A0000E51642864E8597000000E78060B04101F0
:101A10001703FFFF6700436E4A860A8597F0FFFFB2
:101A2000E78000234DBF1703FFFFE702436BB33589
:101A3000B000011185052A891315F60133651501DA
:101A40002308B1009305110136843AC632C03EC462
:101A500042C297F0FFFFE780801DA247124842551F
:101A600093D68700230BF1009305910193578800CB
:101A7000A30AD100A30BF100230C010197F0FFFF93
:101A8000E780E01A3247024603280400B337E0003B
:101A9000835644009207914411C2A1444A85A68806
:101AA00042860C0897F0FFFFE78040772A8919E506
:101AB000A685228597B0FFFFE780A0AB4A85056128
:101AC0001703FFFF6700E3631703FFFFE702835F6E
:101AD00001113EC68647B335B0008505AA891315A6
:101AE000F6015D8D2308B1009305110136843A8912
:101AF000B28442C446C297F0FFFFE78040132248F9
:101B00009248164593578800A30AF1009305910166
:101B100093D78800230B0101A30BF100230C1101C3
:101B200097F0FFFFE780A010324710408356440033
:101B3000B337E000920703280900914891C0A148FB
:101B40000C084E8597000000E780809CAA8401E97C
:101B5000835544004A8597B0FFFFE78080A1268522
:101B600005611703FFFF67002359AA959307F00F3C
:101B700017070100130707646317B50013C5F7FFC4
:101B80001375F50F828005058346F5FFB58FBA976B
:101B900083C70700D5B70357450014419307F00FDB
:101BA0001706010013060661369742074183139515
:101BB00006014181631BE500AD8FB29703C50700A5
:101BC000130515F3133515008280850603C5F6FF4E
:101BD000A98FB29783C70700D9BF1703FFFFE7029A
:101BE0000350B28736842E86BA86AA853E85BA848B
:101BF00097F0FFFFE7806052634F0500228597D082
:101C00000000E780E0782A86A686A285268597F0E0
:101C1000FFFFE78080501703FFFF6700834E170325
:101C2000FFFFE702234A5D712A8BAE8A1705010088
:101C30001305C5552C00B284368ABA893E8997F0BF
:101C4000FFFFE780C04F2A845DE134104146DA850A
:101C5000280097F0FFFFE780404C2A8449E9854738
:101C6000A303F100A6C2930771002408BEC4A68690
:101C700085470D462C18281002DC02DED6C0BEC6F1
:101C800097F0FFFFE78000442A8435E18347710223
:101C9000A6860D4693F7F7072300FA00C1473EDEFC
:101CA0002C188947281026DCA303F10097F0FFFFCA
:101CB000E78040412A8405ED4146A6854E8597D0B0
:101CC0000000E78060488D47A6860D462C18281036
:101CD000A303F10097F0FFFFE780C03E2A8401E9EB
:101CE0004146A6854A8597D00000E780E0452285D9
:101CF00061611703FFFF670023401703FFFFE7023F
:101D0000033E97F700009387E7A1984383C74700F6
:101D100079712A89AE84170501001305A5470C08BF
:101D20003AC42306F10097F0FFFFE78040412A8480
:101D300005ED14104146CA85080897F0FFFFE780BB
:101D4000C03D2A8415E1140815462C00081097F0B0
:101D5000FFFFE780803C2A8401E921462C08268584
:101D600097D00000E780403E228545611703FFFFC2
:101D7000670023391703FFFFE702633697F7000078
:101D80009387479A9C477971AA842E84170501008E
:101D90001305C5400C083EC697F0FFFFE780203AC8
:101DA0000DE914104146A685080897F0FFFFE7806B
:101DB000C03605E1140811466C00081097F0FFFFCB
:101DC000E780A03519E58347F10193F7F703230076
:101DD000F40045611703FFFF6700A3321703FFFFFD
:101DE000E702E32F3688A14881470147E54697F08F
:101DF000FFFFE780A0421703FFFF67008330170350
:101E0000FFFFE702C32D3688A14881470147E54619
:101E100097F0FFFFE780C06F1703FFFF6700632E97
:101E20001703FFFFE702A32B01112A842E850C085C
:101E300032C697F0FFFFE780803009ED3247970602
:101E40000100938626341008C145228597000000C2
:101E5000E780E0D805611703FFFF6700832A1703B7
:101E6000FFFFE702C3274111C1472EC032C48A8554
:101E700009463EC23EC697F0FFFFE780A02441011D
:101E80001703FFFF6700E3271703FFFFE702232580
:101E90004111AE8613061009AA850A8502C002C246
:101EA00002C402C697F0FFFFE78020274101170315
:101EB000FFFF670003251703FFFFE7024322328776
:101EC000970601009386062E2E8693050002970042
:101ED0000000E780C0D01703FFFF670083221703CD
:101EE000FFFFE702C31F7971C1472ACC2ED032D43D
:101EF0002C080D4628003ECE3ED23ED602C402C675
:101F000002C802CA97F0FFFFE780C01B45611703B4
:101F1000FFFF6700031F1703FFFFE702431C0111C8
:101F2000AA842E8417050100130545288A8597F099
:101F3000FFFFE780C02015E514084146A6850A8505
:101F400097F0FFFFE780601D09ED8347E10103473C
:101F5000F101A207D98FCA07C9836177D98F2310EE
:101F6000F40005611703FFFF6700A31915CD1703E0
:101F7000FFFFE702C3169747FF1F9387E7EE9043E3
:101F80009745FF1F938585EE1745FF1F1305C5E98C
:101F900097D00000E78000C51745FF1F1305C5E86F
:101FA0001703FFFF6700E3151745FF1F1305C5E77C
:101FB00082808DCD1703FFFFE70263129747FF1F53
:101FC000938787EA944301112E840A869745FF1F61
:101FD0009385C5E997D00000E78040C60A85029442
:101FE000014505611703FFFF6700A3117D5582803E
:101FF0001703FFFFE702A30E97D00000E78080D110
:102000009747FF1F23A2A7E617F5FFFF1305E5C9B2
:1020100097B00000E780C0741703FFFF6700630EEE
:102020001747FF1F130787E69317150008433E95D0
:10203000FD572310F50082801703FFFFE702230AF4
:102040002A84084009E51703FFFF6700830B1C4142
:1020500058401CC06313E5005CC083475500232033
:102060000500F99BA302F50097A0FFFFE780E07C45
:10207000C9BF1703FFFFE702E3049747FF1F9387DA
:10208000E7E298432A8411CB8347350093F7070290
:1020900089C703550500894502971305440197B088
:1020A0000000E780403B835504000355E40097306F
:1020B0000000E780A00C485819C597A0FFFFE780F3
:1020C000C077232A04021305840397000000E780E9
:1020D000E0F68144B1499790FFFFE780E06A63CB67
:1020E000A402834734002320040493F727FCA301B0
:1020F000F40000489790FFFFE780006A1316150070
:10210000814522859700FFFFE78060001703FFFFEE
:10211000670083FEB38734030329040385043E99D3
:102120004A8597000000E78060F12304090065B745
:102130008347350093F7070299E30145828083576F
:10214000E500E39CB7FEC167FD176316F600054581
:102150008280054599A81703FFFFE70243F893170C
:102160000601C187B2842A8401496359F00283576A
:1021700005009DCB01456367F600034584003E954D
:102180003325A6001375F50F0DA01C481317190071
:10219000BA9783D70700E38E97FA05099790FFFF58
:1021A000E780805FE343A9FE01451703FFFF670057
:1021B00043F51703FFFFE702E3F0AE89AA84979087
:1021C000FFFFE78020532A8497D0FFFFE780A02EEF
:1021D000AA8601471306840197050000938585E4CC
:1021E0001745FF1F1305C5CA9790FFFFE780A01989
:1021F0002A8925C98C441304C50022859E0593F5C0
:10220000050897A0FFFFE780003DCC40838774005E
:10221000E18163DD070493E50508228597A0FFFFB0
:10222000E780603B0D4693854400228597A0FFFF21
:10223000E780803783D50400228597A0FFFFE780E1
:10224000A03E83D52400228597A0FFFFE780C03DF4
:1022500003D6490083A50900228597A0FFFFE780E8
:10226000A0344A851703FFFF670003E993F5F507DC
:102270006DB71703FFFFE70283E601112A84328559
:1022800032C697A0FFFFE780A0289780FFFFE78076
:102290008031835704001747FF1F1307A7D8324622
:1022A000231BF100930700F8A30DF1001C4718430E
:1022B000231AA1008983858BB307F740B2854808AC
:1022C0003ECE231C0100230D010097000000E78093
:1022D00080EE05611703FFFF6700A3E21703FFFF0E
:1022E000E70243DE004101453DC49304C400268556
:1022F0003289AE8997A0FFFFE780802595452A8A1D
:102300002685035B040197A0FFFFE780E021268577
:1023100097A0FFFFE780203F8D45AA8A268597A0DA
:10232000FFFFE7806020268597A0FFFFE780A03DA4
:102330005C48420A135A0A01D2975CC4231864010C
:10234000814763983A0146054D813306254193370D
:10235000160013F5F70F1703FFFF6700E3D9170304
:10236000FFFFE70243D589692A8BAE8B328AB68A92
:1023700081440144314CFD199790FFFFE780C04034
:1023800063CDA4009790FFFFE7800043018D33B534
:10239000AA001703FFFF670083D5338984038327CF
:1023A0000B003E9963170A008347890085043E9419
:1023B000E1B703560A00DE854A8533F6C900970067
:1023C0000000E780E0F16DD10545E1B71703FFFF9D
:1023D000E702E3D001112A847C000355E5003ECAE0
:1023E000B70707003ECC7C003ECE97200000E78078
:1023F00020082A898545480897A0FFFFE780E03933
:102400009945480897A0FFFFE780A016AA844A854F
:1024100097200000E780A0082380A4009747FF1FB3
:10242000938747C09C434166130606F09396870145
:1024300013D78701558F93D68700F18E558FA2074A
:10244000B706FF00F58FD98F11462C0013851400B5
:102450003EC497D00000E78020CF5008A38204003C
:102460008945228597000000E780E0E019C9AA8528
:102470001305840397A0FFFFE780A0323C40850747
:102480003CC005611703FFFF6700A3C71703FFFFE9
:10249000E702E3C49790FFFFE78000322A84050437
:1024A0009790FFFFE78040303305A402F147914544
:1024B0003305F50297200000E78020BA11E5655545
:1024C0001703FFFF6700E3C39747FF1F23A8A79CDD
:1024D0009790FFFFE780402E2A8405049790FFFF26
:1024E000E780802C3305A40289450605972000006B
:1024F000E780A0B669D59747FF1F23A9A7989790B3
:10250000FFFFE780602B2A8405049790FFFFE78098
:10251000A0293304A4029747FF1F239B8796979017
:10252000FFFFE78060292A849790FFFFE780C0279C
:10253000930714003385A7029747FF1F239BA79497
:10254000970701009387478A1747FF1F2326F794B1
:102550000145BDB71703FFFFE702C3B6AA842E8962
:1025600001449749FF1F9389E9AB130A80069790AE
:10257000FFFFE78060236347A40001451703FFFFC7
:10258000670083B73305440383A709024A86A685FB
:102590003E9597000000E780E0B919E10504C1BF4E
:1025A0000545E9BF1703FFFFE702E3B0AA8A2E8BB8
:1025B000B28B368C3A8A814401448149974CFF1F83
:1025C000938C4CA6130D80069790FFFFE780C01DEB
:1025D00063C9A40011E085494E851703FFFF67001A
:1025E00003B13389A40383A70C025E86D6853E9986
:1025F0004A8597000000E780E0B31DC19790FFFF78
:10260000E780801B0544636D4501D2866286DA85CA
:102610001305090397000000E780A0D411C1854984
:1026200085045DB71703FFFFE702C3A9C164411129
:102630002A8901449749FF1F9389C99E130A80067E
:10264000FD1436C632C42EC29790FFFFE780C01536
:1026500092452246B2466348A40001454101170352
:10266000FFFF670063A93305440383A709023E9572
:1026700009C683473500C18B9DC791C68347350086
:1026800093F707028DC3630699008357E500639CA7
:1026900027010357050001CB63E7E5008347850069
:1026A000BA97E3CDF5FA050469BF1703FFFFE70208
:1026B00063A1C1642A8901449749FF1F93898996C0
:1026C000130A8006FD149790FFFFE780E00D634634
:1026D000A4001703FFFF670023A23305440383A769
:1026E00009023E958357E500638A970063049900C9
:1026F0006396270197000000E780E0970504E1B7A3
:102700001703FFFFE702A39A89692A8AAE8A328BF0
:10271000B68B8144174CFF1F130CCC90930C800692
:10272000314DFD199790FFFFE780000863C6A400B4
:102730001703FFFF6700639B3389940383270C0211
:102740008355CA015A863E994A8597000000E78062
:10275000609E31C1814D15A03384AD0383270903E9
:1027600003D60B00D68533F6C9003E942285970028
:102770000000E780E0B609E9850D9790FFFFE7804C
:10278000A000E3CBADFC01A8228597000000E78004
:10279000E08A23040400850471B71703FFFFE702F2
:1027A00083914169AA8A014A174BFF1F130B8B873C
:1027B0007D19C14B054C9790FFFFE780E0FE634613
:1027C000AA001703FFFF6700839293098006B307EF
:1027D0003A0383290B02BE9983D7E900638E270150
:1027E00063842A01639A570103A4890301E84E8593
:1027F00097000000E780C0BD050A75BF835704013C
:10280000639977099304C400268597A0FFFFE780AA
:1028100020D485452A8D2685835C040197A0FFFF7F
:10282000E78080D0268597A0FFFFE78060E86205FB
:102830006185635905048D45268597A0FFFFE780D4
:10284000A0CE8945268597A0FFFFE780E0CD89458A
:10285000268597A0FFFFE78020CD8545268597A098
:10286000FFFFE780A0CD83470500094793F7F707EF
:10287000639AE7009945268597A0FFFFE78000CC83
:10288000A30285014848337D2D01231894016A95E0
:1028900048C40040A1BF1703FFFFE702438437E4A9
:1028A00004008327041D82979737FF1F83C787641F
:1028B0001715FF1F130585C7A300F5008327441CC8
:1028C00082978327841C81461306F00F81450145BA
:1028D00082971703FFFF6700C3821737FF1F130795
:1028E000675118439735FF1F83C5C5609737FF1F92
:1028F0009387C75E83468703034697036397D50094
:102900009737FF1F2388C75E828083C587010347EF
:10291000A7036317B6009737FF1F238DE75C8280FC
:1029200003C687016317C7009737FF1F2384D75C4F
:10293000828083C68701130750026319D70093076B
:1029400060021737FF1F2307F75A828083C687016B
:10295000130660026315D60093077002DDB783C7C4
:10296000870155BF9737FF1F93874757D44B0947B8
:10297000638DE60817F3FEFFE70263761739FF1F42
:10298000130909533E8483470900918B9DCFB7E417
:10299000040083A7041D829783A7441C1735FF1FDB
:1029A00013058551829783A7841C81461736FF1F24
:1029B0000346865281450145829721C58347090018
:1029C000ED9B1737FF1F2305F74E8347040093F74E
:1029D000F70F85CB91471737FF1F232BF750970031
:1029E0000000E78080EB97000000E78040EFB7E74A
:1029F0000400BC4F414691451735FF1F0345854EE6
:102A0000829717F3FEFF6700C36F828017F3FEFF04
:102A1000E702E36C8D4741116306F504C54763087F
:102A2000F50285476310F5029737FF1F2386A74CF1
:102A3000B7E70400BC4B930500101735FF1F034593
:102A4000654A8297410117F3FEFF6700836B854754
:102A50001737FF1F2302F74AB7E70400BC4B930563
:102A60000020E1BF9737FF1F93874747D44B11479B
:102A7000638DE600B7E7040083A7071D8297B7E7D9
:102A80000400BC4B930500044DBF05491737FF1FD9
:102A90002320274783C7070032C62E8493F7F70FFA
:102AA000D5D3B7E4040083A7041D7D141374F40F79
:102AB0008297E37689FCB245994703C61500E3F097
:102AC000C7FCFC4409061735FF1F130525438297F1
:102AD000BC48930500081735FF1F0345A5408297A2
:102AE00079BF17F3FEFFE702835F1737FF1F130756
:102AF000E73E4047184B1C409736FF1F23A6F63E83
:102B00006316E4001737FF1F2322F73E130584FEE8
:102B10009790FFFFE78020A7035564FF9780FFFF92
:102B2000E780A06F97A0FFFFE78020D117F3FEFF9B
:102B30006700235D17F3FEFFE702635A9737FF1F15
:102B40009387C739D84BDC4789C797000000E780D7
:102B500080F985471737FF1F232CF7389737FF1F5A
:102B6000938747299C43930500021735FF1F0345B0
:102B7000653783C787031737FF1F230DF736B7E77E
:102B80000400BC4B829717F3FEFF6700835797370B
:102B9000FF1F23A7A734828017F3FEFFE7028352AB
:102BA00037E404007C4CA1451735FF1F03458533EE
:102BB00082977C48A1451735FF1F0345A5329734FE
:102BC000FF1F9384A4318297DC4489EB97000000B7
:102BD000E78080D917F3FEFF6700035203D567FF34
:102BE0009780FFFFE7806063AA896DD1D84891473D
:102BF0006310F7027C4C91451735FF1F0345852E66
